:10000000C0A0002035260000B71101002126000005
:10001000212600002126000021260000000000000B
:10002000000000000000000000000000AD270000FC
:1000300021260000000000004927000021260000C2
:100040007129000025A70000712900007129000016
:100050007129000071290000712900007129000038
:100060007129000071290000712900007129000028
:100070007129000071290000712900007129000018
:100080007129000071290000712900007129000008
:1000900071290000712900007129000071290000F8
:1000A00071290000712900007129000071290000E8
:1000B00071290000712900007129000071290000D8
:1000C00071290000712900007129000071290000C8
:1000D00071290000712900007129000071290000B8
:1000E00071290000712900007129000071290000A8
:1000F0007129000071290000712900007129000098
:1001000053B94AB9002908BF00281CBF4FF0FF317E
:100110004FF0FF3000F00CB8ADF1080C6DE904CEE3
:1001200000F010F8DDF804E0DDE9022304B07047C8
:10013000704700BF034611F8012B03F8012B002A7A
:10014000F9D170472DE9F04786468C460846089E4F
:10015000154674461946002B40F0C2808542B2FA1B
:1001600082F245D94AB1C2F1200300FA02FC2EFA0C
:1001700003F3954043EA0C0C94404FEA154EA8B2A5
:10018000BCFBFEF8230C0EFB18CC08FB00F943EA7D
:100190000C43994528D9EB1808F1FF3704D299454B
:1001A00002D9A8F102072B44A3EB0903A4B2B3FBC5
:1001B000FEFC0EFB1C330CFB00F044EA0344A0429F
:1001C00014D92C190CF1FF3304D2A04202D9ACF19E
:1001D00002032C44241A43EA07401EB1D4400023F2
:1001E00034607360BDE8F0874746DDE76346F1E7BA
:1001F00092BB431B01214FEA154EAFB2B3FBFEFC8D
:10020000200C0EFB1C330CFB07F840EA0343984517
:1002100062D9EB180CF1FF3004D2984502D9ACF149
:1002200002002B44A3EB0803A4B2B3FBFEFC0EFBBD
:100230001C330CFB07F744EA0344A7424ED92C19A0
:100240000CF1FF3304D2A74202D9ACF102032C44D3
:10025000E41B43EA0040C0E7C2F1200320FA03F1A7
:10026000954090402EFA03F303434FEA154EAFB288
:10027000B1FBFEFC0EFB1C10190C0CFB07F841EA4D
:100280000041884504FA02F422D969180CF1FF30C4
:1002900004D2884502D9ACF102002944A1EB08013F
:1002A0009BB2B1FBFEFC0EFB1C110CFB07F743EAF3
:1002B00001439F420ED9EB180CF1FF3104D29F424B
:1002C00002D9ACF102012B44DB1B41EA004192E769
:1002D0006046E3E76146F7E76046A3E76346B7E7B2
:1002E000834206D916B9002108467BE7C6E900E03B
:1002F000F9E7B3FA83F78FB9834201D3724508D87F
:10030000BEEB020460EB030301209C461EB90021F2
:1003100068E73846FAE7C6E9004CF8E7C7F1200C71
:10032000BB4022FA0CF41C432EFA0CF120FA0CF319
:10033000B84001434FEA14490EFA07F5B3FBF9F848
:100340001FFA84FE09FB18300B0C08FB0EFA43EA77
:1003500000439A4502FA07F240D9E31808F1FF304A
:1003600004D29A4502D9A8F102002344A3EB0A0360
:1003700089B2B3FBF9F809FB183308FB0EFE41EA1A
:1003800003418E452CD9611808F1FF3304D28E4504
:1003900002D9A8F10203214443EA0040A0FB0298DD
:1003A000A1EB0E014145CE46434602D306D14D4551
:1003B00004D2B9EB020E68EB04030138002EA6D07C
:1003C000B5EB0E0261EB030101FA0CFC22FA07F314
:1003D0004CEA0303F940C6E9003198E74046C5E717
:1003E0004346D9E7000000002DE9F843D0E906387C
:1003F000456903EB08042F34A5420F46164619D869
:10040000DFF86C80A3FB080117A3D3E90023FFF7F3
:1004100077FE0346601BA0FB080123F07F4412A374
:10042000D3E90023FFF76CFE20F07F403C60306092
:10043000BDE8F883DFF838900BA3D3E90023A5FBD0
:100440000901FFF75DFE20F07F440A480A2106A358
:10045000D3E90023E8FB0901FFF752FE20F07F40BB
:100460003C603060BDE8F8838D49FD1A070000004C
:1004700000CA9A3B00166BF170B5234C9DF810E052
:1004800094F83AC01CF0020F34D1460816F0040567
:1004900030D139B363F3830C4001237D21854FEACA
:1004A000CE0E0EF0180E00F0200040EA0E0023F0F1
:1004B0003803184394F820302075144884F83AC063
:1004C00066F3020384F820309121A2FB000301FBB4
:1004D00002310BA3D3E90023FFF712FEE062206391
:1004E000284670BD94F8203065F3020384F820306C
:1004F000284670BD0C25284670BD00BFAFF30080B4
:100500008D49FD1A0700000090070020002AE784AB
:100510002DE9F04390F83A30027D3F4D6FF3000330
:10052000044600F12101C3F3800060F386128DB010
:1005300084F83A30227505F0ABFD227D238D3748D3
:10054000246102F079024FF0000922759121A3FB8A
:100550000002C4E9029984F8009001FB03212CA356
:10056000D3E90023FFF7CCFD226B02F10E03984282
:100570008EBF19464A460146294BE2626160651BFF
:10058000A3FB0535064605F045FD4F460DF12C0849
:10059000CDF8208006940397238D00F10E091F48A3
:1005A0009121A3FB000201FB0321636804931D4B0F
:1005B00007931D4B059302230B9315A3D3E9002347
:1005C000FFF79EFD104619464FF47A720023FFF79D
:1005D00097FDC5F307150235EDB2CDE901600321A2
:1005E0004B462A460097384605F020FC414606F067
:1005F00013F940B994F83A3043F0020384F83A30E2
:100600000DB0BDE8F0830C200DB0BDE8F08300BF55
:100610008D49FD1A0700000090070020002AE7849A
:10062000398EE338F96000006D8E00000000000094
:100630002DE9F04F0B7995B0092B0C460A9008D0A4
:100640000D2B00F05D81062B4DD000DE15B0BDE80E
:10065000F08F8B680B931A46A74B15689D4240F0AC
:10066000C082D5F81CB0BBF1000F00F00584A24990
:100670003022084604F034FB0330C3B20D93BBF1C3
:10068000000F00F00E85DBF80060304608F052FEE7
:100690000746002800F0A6830B9B5A7990F83C305F
:1006A00002F007029E0754BFD0F840A04FF0000AA6
:1006B000012A00F01283022AC7D10723667E237124
:1006C0000A9B23600021334661F3C713637694F8D5
:1006D0002130E160002B00F0E38288461092C6F3DF
:1006E00080060C9129E0D1F808B0DBF80830002B27
:1006F00040F09E83DBF8007097F83C3038469B074B
:1007000054BFD7F840A04FF0000A08F0F9FD0230BE
:10071000C3B20D930A9B2360637E002666F3C71362
:10072000637694F82130E660002B00F07783CDE902
:100730000B6601221092B046354694F822209006AE
:1007400000F0258194F8233013F0010004F124090E
:1007500024D0BAF1000F1ED097F83C1001F00C0223
:10076000082A18D094F8202000204B46009001F071
:100770000101C2F38012504609F026FB97F83C3085
:10078000002800F0E982012262F3830387F83C30FD
:1007900094F8233000E0002004F12A09990748BFAB
:1007A00009F106095A0748BF09F1010913F00802C7
:1007B0001CBF4A4609F1020913F0100116BFCDF81B
:1007C00038900E9109F1030999061CD509F112011F
:1007D0000F91BAF1000F00F04082002D00F03D8231
:1007E000002800F03682002A00F03782527839461D
:1007F0001209504609F012FB002840F04883DDF84A
:100800003C9094F8233094F822105A0648BF09F11E
:100810000109C1F3050104F122030131A9EB03032E
:10082000DBB2C9B28B429EBFCB1ADAB20B4694F848
:10083000211088BF0022994286BFC91ACBB200237B
:100840000F9323790D2B00F0C4810E9B43B199784F
:100850005A789C460B0203F4F853134340F0C080CF
:10086000B8F1000F00F03B82D8F800200F98B2F8E2
:10087000B43000211844A083A2F8B410002E40F038
:10088000D681BAF1000F6BD097F83C3003F00C031F
:10089000082B00F0018297F83C306FF3830387F850
:1008A0003C3000237B64002D00F089806B6A002BB4
:1008B00000F0DE8197F83A20D20700F1B182DC60C7
:1008C0006C62EB69002B00F08982EB69002B00F071
:1008D00087822B7803F0FF02002B00F0B481012AFD
:1008E00040F0A282AB68002B40F0A082034BC5E928
:1008F000023515B0BDE8F08F184300201D950000AB
:10090000D1F80880D8F83C30002B40F09382D8F81A
:100910000060304609F02CFAE368E080304698F831
:100920000B500C9309F024FA0A9B2360637E002687
:1009300066F3C713637694F82130E66005F0070587
:10094000BBB99A461F461D46D8F80020B2F8B4003D
:1009500000210344A383A2F8B410BAF1000F93D18D
:100960006DB36B6A002B00F0838107B900DE6B6A00
:10097000A0E70430C2B20D9294F8222010959006A0
:10098000B346B246374635460B967FF4DBAE013BA5
:10099000DBB2B8F1000FD7D1002D40F08181A383E5
:1009A000BAF1000F0BD097F83C3003F00C02082A84
:1009B00005D06FF3830387F83C3000237B640A98EB
:1009C000214605F00FFF0C9A2AB10123106813711C
:1009D000114605F007FF15B0BDE8F04F05F008BF60
:1009E000002E40F015814809022800F2948100F0A1
:1009F00092819CF800C00CF03F02242A00F28B8107
:100A0000109E94F8211006F003020A441CF0800F97
:100A100002F10902C6F340014FEAC20214BF4FF4CB
:100A200096761E26CA4006FB03F303EB060E02F57C
:100A300096718E45FFF425AF1CF0400F14BF322194
:100A40004FF4FA71DFF8F8C203FB01F1ACFB01C10E
:100A5000890C1091012101FA00F95FFA89F0CDE9C2
:100A600011320AF06DF96169129A119B13902F39B6
:100A70008A1A1344109A1B1AB2489B1AA3FB00014E
:100A8000ADA3D3E90023FFF73BFB20F07F43119395
:100A9000A37EDB0740F18581002D00F04D82B8F187
:100AA000000F00F00C82D8F800200F99B2F8B43093
:100AB00019448BB21E2BA2F8B430A38304D9A37EB1
:100AC00013F0010300F071820E9B0B981978828855
:100AD00001F03F0141EA092122F4E76240F23F734D
:100AE00022F007020B4013438380A37EDB0700F153
:100AF0001182BBF1000F00F06081002F00F07D82B9
:100B000097F83A3013F0010340F0AA80DBF8082090
:100B10000B998A4200F056820B9F139B7A79894881
:100B200003F5EA7102F003030933C2F34002DB006C
:100B3000D340854A0B440721E3FB002110467EA3E6
:100B4000D3E90023FFF7DCFA109B2F3306EB4303B6
:100B500020F07F4068600022BB600221012004F089
:100B600025F90D9AFF2A0DD02369119900203B3BEE
:100B70000B44CDE90000012105F0C6F910F0FD0F8E
:100B800040F08D8271493022284604F0A9F870495E
:100B90002369CDE907156F49CDE905156968024656
:100BA0000020CDE90301033211990091CDE9010044
:100BB0003B3BD2B2012105F039F910F0FD0F40F0B6
:100BC0006C8201220221104615B0BDE8F04F04F0FE
:100BD000EDB8002A3FF439AEA079494609F04AFA47
:100BE00033E6284608F0A6FBE3680B93834600280B
:100BF00000F02781D4F808B0002B00F0D0800B9BC8
:100C00001D68EB695B4540F0C880FF230D9336E516
:100C1000B8F1000F00F0B480D8F800200F99B2F8B6
:100C2000B43019440B460021A383A2F8B410002D60
:100C300000F0B0806B6A002B00F0AC80DC606C626E
:100C400015B0BDE8F08F284615B0BDE8F04F08F0AC
:100C5000FDBB796CA9423FF4C6ADDDF83C90D2E50E
:100C6000BAF1000F40F0A6816B6A002B40F0D880EB
:100C7000B8F1000F2DD00A98214605F0BFFDD8F835
:100C8000003093F88A30DB067FF51BAED8F83C3095
:100C9000002B3FF416AED9E4002D7FF407AE8EE6AC
:100CA0002A8D13449BB22B85A383BAF1000F00F069
:100CB000C38097F83C3003F00C02082A53D06FF33E
:100CC000830387F83C3000237B646B6A002B7FF43E
:100CD000F1AD00DE4FF00008CDE70623EEE4002D75
:100CE00046D02B8D0F9A1A4493B22B85A383002EE6
:100CF000A0D1BAF1000F3FF434AE97F83C3003F0C6
:100D00000C02082A3FF4D2AD6FF3830387F83C301E
:100D100000237B64CAE5B8F1000F00F0B080D8F87A
:100D200000200F99B2F8B4301944A183A2F8B4603E
:100D3000A7E500BFAFF300808D49FD1A0700000052
:100D400083DE1B4300CA9A3B8C49FD1A18430020DE
:100D5000B19300000594000060F3830387F83C30F2
:100D600094F8233018E56B6A002B7FF4A3ADB0E74D
:100D70000F9BA38376B9BAF1000F7FF414AE1EE681
:100D800035B12B8D0F9A1A4493B22B85A38351E76B
:100D90000F9BA38300DE6B6A50E700DE35E700DEC1
:100DA0002DE705F037F92369119A243B991805F0CE
:100DB00033F900023FF570AE63E5D8F83C30002B04
:100DC00040F06481D8F8003093F88A30D90600F1F9
:100DD00016810B9BC8F83C302C629DE600DE74E562
:100DE00000DE76E50B9B5B7903F0070380461093EA
:100DF0000D233046237108F0BBFF0A9B2360637EFE
:100E0000E080002666F3C713637694F82130E6602D
:100E1000002B29D0B24637460C968EE40C93BEE5E3
:100E20009C427FF40BAF11E400DE5BE500DE5DE584
:100E300000DE5FE400DE6AE56B6A002B7FF495ADAF
:100E400047E7D4F80880002B37D00B9B1D68EB696F
:100E5000434530D10B9BD8F800605B7903F0070362
:100E60001093FF230D93C3E79A461F460C93B8F1E6
:100E7000000F7FF469AD8FE500DEFFF7F8BB9DB191
:100E80002B8D0F9A1A4493B22B85A38331E7697D8A
:100E90004B4601F0070122463846DDF83C9000F051
:100EA00007F994F82330AEE40F9BA383BAF1000F47
:100EB0007FF479AD83E500DECCE700DEC5E72B8D5E
:100EC0000F9A1A4493B21E2B2B8502D9A37EDA0700
:100ED0007DD56B6A002B78D0DC602B8D6C62A38390
:100EE0000E9B0B981978828801F03F0141EA092195
:100EF00022F4E76240F23F7322F007020B401343F3
:100F00008380A37ED80744D4BBF1000F7FF4F5ADF6
:100F100000DE57E70B9BC8F83C30637E0A9843F02D
:100F200080032146637605F069FC0B9A13796FF311
:100F300086131371FFF78ABB5B4803F0A7FE0028F6
:100F400065D0027D0F9B038565F3C712027500F122
:100F50001003BBF1000F14BF5A4642460570C0E9AA
:100F60000255056245620061C2610B93BAF1000F40
:100F700006D097F83C2002F00C02042A08BF7864DF
:100F80000C9BC3620546B8F1000F65D000230C939B
:100F900089E5DBF80830002B73D10B9BCBF80830C8
:100FA000637E43F080036376BFE7A2F8B430BAF102
:100FB000000F27D097F83C3003F00C03082B7FF488
:100FC0006AAC73E4CBF80830A6E52C6285E7BAF189
:100FD000000F3FF431AF97F83C3003F00C02082AC1
:100FE0003FF4C1AE68F3830387F83C30C7F8448010
:100FF0006B6A002B7FF45EAC6BE600DE80E5BAF135
:10100000000FD7D16B6A002B7FF4AFAC33E6A37E21
:10101000D90703D5637E43F080036376B8F1000FF0
:101020001DD0D8F800100F98B1F8B4300022184441
:10103000A083A1F8B420BAF1000F3FF4C0AC97F838
:101040003C3003F00C0108293FF4B9AC62F3830390
:1010500087F83C307A64B2E4CDF8308039E7BAF1F1
:10106000000F3FF4ACAC97F83C3003F00C02082AB8
:101070003FF4A5AC68F3830387F83C30C7F844809D
:101080009DE40B9A934288D000DE86E7D8F83C3086
:101090000B9A93423FF496AE3AE700DE91E500DE0C
:1010A00070E5DBF80030FFDE144300200000000094
:1010B0002DE9F04F046C94F8346084F835601D46D7
:1010C00007462823062010FB06306B6823502B7A36
:1010D000204403F01F0303718DB0894606EB4606DA
:1010E000052104EB4606904603F0ACFF96F82D3040
:1010F00000F03F0060F30503012886F82D3040F230
:1011000015812046D5F8093040F8143F09F076F9EA
:10111000E084B5F80D30EA7BA2762383E27E237F5C
:10112000298AA18469F302026FF3C303E27623776D
:10113000B5F802A0B4F87A2040F2E2431FFA8AF62A
:1011400003FB06F642F21071731E01FB0233B3FB80
:10115000F6F39BB2A4F87C30B4F87C309BB2062B3B
:1011600000F2E7800023A4F8783094F88A30062251
:1011700062F3471384F88A3095F8089009F032FF3B
:101180004FEA59198346484609F02EFF0BEB00033E
:1011900006FB03F3704A714903F5742303F23F23FE
:1011A000A2FB03239B0CA3637308963BE3636B785A
:1011B00013F0200F0CBF1E234FF49673A36400237B
:1011C00023677B6497F83C30022262F3830387F83D
:1011D0003C30B822204603F083FDD4F8B0300C2216
:1011E000A3F822A0D8809C601A71E27E83F8249034
:1011F000C2F3020283F821200746E07E012100F0BD
:10120000070009F09DFD95F801E02B7894F81BC0CC
:1012100098F82120D8F81410D4F848901EF0400F08
:101220004FEA0E2E0EF4F85E4EEA030E0CF00303A6
:101230001A4402F10902CCF3400C4FEAC202A1F1B8
:101240002F0522FA0CF209FB0E55A5EB0205A5EBC2
:1012500000050CBF00224FF416121544A5EB01093E
:1012600040F28A22914503D8A28C01323544A284EF
:101270000933DB0023FA0CF303F5EA73DFF8E0909F
:1012800018444FF0070A374B5146E0FB0931184626
:10129000A36BF61AA6FB09B30B932DA3D3E9002386
:1012A000FEF72EFF304BC4F8803020F07F4628A395
:1012B000D3E900230B9966605846FEF721FF069498
:1012C0000496D8F81030A3F13B08284B20F07F4457
:1012D000A4FB0331BBEB03000B9B0AFB041163EB84
:1012E00001010022224B03920593224A079240F209
:1012F000824308934FF47A720023FEF701FF14A390
:10130000D3E90023CDE90140A5FB0901FEF7F8FE72
:10131000043720F07F40FFB2009043463A46012157
:10132000002004F083FD10F0FD0F0CD10DB0BDE8DE
:10133000F08FB4F87C30B4F87820063B9BB29A4228
:101340007FF613AF0FE700DEF0E700BFAFF30080DA
:101350008D49FD1A0700000083DE1B438C430020EB
:1013600000CA9A3B8C49FD1A59CB00008D49FD1AE1
:10137000E5970000DD9700002DE9F0418AB00223D7
:101380000C4615462C490993B82203F0A9FCDFF856
:10139000AC8009AB06932A4B0593002724A3D3E91D
:1013A0000023061DA5FB0801CDE90377FEF7A8FE83
:1013B000034623F07F430293A4FB08011CA3D3E957
:1013C0000023FEF79DFEF6B220F07F40CDE90070CD
:1013D0003B4632460321384604F044FD10F0FD0F31
:1013E0000CD0099B022B19D1099B012B14BF6FF064
:1013F0000B006FF001000AB0BDE8F0814FF0FF3242
:101400004FF0FF330F480EF095F9099B012B14BFE5
:1014100038466FF00D000AB0BDE8F0814FF0FF32A2
:101420004FF0FF3307480EF085F9DDE7AFF300809A
:101430008D49FD1A070000008C43002000CA9A3B2A
:10144000BD980000704300202DE9F041C468237965
:101450006FF300038CB023710F4605460BF0C6FDF9
:1014600000200BF0E9FD207C012100F007000BF0CB
:10147000D5FD227C92000820252102F01C020BF0F1
:1014800039FE237C23F018030120237405F058FA59
:10149000002864D020300BF061FE494B0B930BA861
:1014A0000BF014FE474940F25B600BF0D3FE20794D
:1014B000C0F34100253009F00FFC434821460BF0F2
:1014C00069FD23799B062DD596200BF0F3FF0023B1
:1014D0001A46194618460BF021FFD4F800802E68F2
:1014E000404609F0E5FB06446A6806F10E0100205B
:1014F0000BF0ECFF0CF01AF90BF084FF204607F01C
:101500000BFF811CC9B24046324609F0D3FB0546A9
:1015100048BB57B1204609F099FB10BB00200CB026
:10152000BDE8F0810BF05CFFD7E7E369002BF1D059
:10153000264D0795264D059540F2F3150093CDE90C
:101540000377CDE9017706943346012239460895A1
:1015500004F06CFC10F0FD0FDCD000DEDAE700DEFA
:1015600098E700DEDAE71B4A1B491C4840F2E51306
:101570000FF09DFC1A4B0721A5FB030301FB05316E
:101580000DA3D3E90023FEF7BBFD1649024616481A
:101590000FF08DFC002585F31188BFF36F8F0323B7
:1015A000184602DF114821460BF0F4FC0BF0F2FD67
:1015B0006FF08B00B3E700BF00CA9A3B0000000049
:1015C000D6BE898E5555550011B50000F5AF000007
:1015D0006DB000008C2F0100D82F0100042F0100F6
:1015E0008D49FD1A08300100DC2F0100F1B0000028
:1015F0002DE9F041C46882B005460DF10301204693
:1016000008F00AF89DF80330002B7ED023795A4A5F
:101610006FF386132371002616800BF0E7FC30462B
:101620000BF00AFD6079012100F007000BF0F6FCD9
:10163000627992000820FF2102F01C020BF05AFD93
:10164000012005F07DF9002867D020300BF086FDE1
:101650004A4B019301A80BF039FD494940F25B6008
:101660000BF0F8FD207900F03F0009F035FB214632
:1016700044480BF08FFC96200BF01CFF627902F0BF
:1016800007020123104600210BF048FE27682E6850
:10169000384609F00DFB06446A6806F10E01002089
:1016A0000BF014FF05466079D4F8088000F00700BD
:1016B00001210BF061FD0544607900F0070002286C
:1016C000454426D004280CBF4FF4BC7328230121C5
:1016D0001D440BF053FD28440BF0D4FF0CF026F80A
:1016E0000BF090FE204607F08DFFC11C3246C9B2B8
:1016F000384609F0DFFA054688B9204609F0A6FA0F
:1017000048B9002002B0BDE8F08121460BF060FA34
:10171000BCE71823DBE700DEF3E700DE95E71A4AB3
:101720001A491B4840F25A230FF0C1FB194B0721FD
:10173000A5FB030301FB05310DA3D3E90023FEF74D
:10174000DFFC1549024615480FF0B1FB002585F373
:101750001188BFF36F8F0323184602DF104821461C
:101760000BF018FC0BF016FD6FF08B00CAE700BF02
:1017700000CA9A3B00000000F2750020D6BE898E98
:101780005555550089C000001C300100D82F0100BC
:10179000042F01008D49FD1A6C300100DC2F01007F
:1017A000C9B70000000000002DE9F041C4680E46F2
:1017B000D4E90A31228A02FB0333226B1344626BA1
:1017C0008B4294BFD21852188A4228BF0A46217B06
:1017D0006263002363F382014F4A2363217305464A
:1017E00013700BF003FCE07A012100F007000BF00E
:1017F00015FCE27A920002F01C02FF2108200BF097
:1018000079FC201D0BF062FC2389A17A40F25B6019
:1018100043EA01410BF01EFD304609F05DFA01205C
:1018200005F08EF8002846D020300BF097FC276892
:101830002E68384609F03CFA06446A6806F10E0143
:1018400000200BF043FE80460BF038FF636BE07A1C
:1018500003F12F02A36B00F00700012103EB420507
:101860000BF08AFC45440544E07A00F007000228AA
:101870001FD004280CBF4FF4BC73282301211D4442
:101880000BF07CFC28440BF0FDFE0BF04FFF2046D4
:1018900008F074FA011D3246C9B2384609F00AFA56
:1018A000054660B9204609F0D1F930B90020BDE8FD
:1018B000F0811823E2E700DEB6E700DEF6E7174A1C
:1018C0001749184840F2F7130FF0F1FA164B0721A9
:1018D000A5FB030301FB05310DA3D3E90023FEF7AC
:1018E0000FFC1249024612480FF0E1FA002585F379
:1018F0001188BFF36F8F0323184602DF0D4821467E
:101900000BF048FB0BF046FC6FF08B00CFE700BFFD
:1019100000CA9A3B00000000E083002078300100FC
:10192000D82F0100042F01008D49FD1AC430010099
:10193000DC2F01002DC5000070B503788AB0044685
:101940000E4607AD032B20D8DFE803F002191B1D5C
:1019500011492846FEF7EEFB059563780493A378BA
:101960000393E37802932379019363790093A37936
:101970000A4A1E2130460EF083FE0AB070BD0849A7
:10198000E7E70849E5E70849E3E7084A0A21284666
:101990000EF076FEE0E700BFA0310100C931010082
:1019A000A7310100AE310100B8310100C2310100A0
:1019B00070B50C468CB01546064604A92068FFF7A2
:1019C000BBFFA988104A286840F6E5430FF08AFA61
:1019D000304602F02DFFE27994F90530042A0146E1
:1019E00094F9060096BF094C094A54F82220064C87
:1019F0000394AC880090CDE90124064804AA0FF0B6
:101A000049FA0CB070BD00BFF4750020482D0100EC
:101A1000EC310100F431010010B50B4688B0694685
:101A200004461868FFF788FF204602F001FF6A4667
:101A3000014604480FF02EFA03480DF041FE08B0AD
:101A400010BD00BF4C320100A4030020F0B50D46CC
:101A500085B002F0EDFE6B79AA7AAE79042B0146CF
:101A600096BF0F480F4B50F82330E879022815D065
:101A70000ED80D4C0D4F002818BF3C46B5F902009A
:101A80000096CDE901400A480FF004FA05B0F0BD18
:101A9000084C044FFF2818BF3C46EFE7064CEDE723
:101AA000482D0100EC310100943201007C3201002C
:101AB000C6320100B93201009B3201002DE9F04726
:101AC0009CB004460D461E22002114A810F0E4FE2E
:101AD000284614AA2D490FF092FC20680CA9FFF7A4
:101AE0002BFF207B2189E27994F9063094F9057067
:101AF000042896BF264D274E55F82060607B0428A9
:101B000096BF234DDFF88CA055F820A06089257979
:101B10000B9501F0010CC1F3400EC1F38008C1F335
:101B2000C00900EB8005C1F30011CDE90591AD10AE
:101B300014A9CDE90905CDE90071CDE9076ACDE920
:101B400003E81548CDF808C00CA90FF0A3F9134A13
:101B50001378C3B96389B3B103EB830310499B10B6
:101B6000C3EBC3030B60012313700E4B22791A7071
:101B700022680D4B116819609188998092799A7149
:101B80000A480DF09DFD1CB0BDE8F087930B0100E5
:101B90005C2D0100EC31010022330100DB820020CA
:101BA000180B0020D9820020DC8200207403002062
:101BB00030B50C468BB002A905462068FFF7BCFE85
:101BC000284602F035FE0146207AE388042896BFB5
:101BD000084C094854F8200003EB83029210CDE929
:101BE0000020064802AA0FF055F905480DF068FDDF
:101BF0000BB030BD5C2D0100EC310100A8330100B9
:101C00008C0300202DE9FF476F480FF043F96F4820
:101C10000FF040F9002001F0F5FD014610B16C48CD
:101C20000FF038F96B486C4D6C4FDFF8B4A10FF032
:101C300031F96C480FF02EF96B4802F0E1FD6B486A
:101C40000FF028F96A480FF025F96A48002602F0DB
:101C500013FF66480FF01EF9B0462E70B146664A73
:101C60002C7887F800903023CDE9002302965CB9E8
:101C700062480FF00FF92146684602F055FD014613
:101C8000B0B153480FF006F95D480FF003F95D4815
:101C90004FF0FF324FF0FF330DF04CFD044668B1BA
:101CA00001464B480FF0F6F8002004B0BDE8F0877D
:101CB00048480FF0EFF801232B70E5E752480FF08A
:101CC000E9F852480FF0E6F8514B524918689A88E3
:101CD0009B798DF80630504B00901B788DF80730BB
:101CE00068464FF42023ADF804200294039302F0D9
:101CF000F3FD014660B336480FF0CCF847480FF0CB
:101D0000C9F8474BD3F800C04FF40044414640F2B5
:101D1000E7304FF47A720023ECFB0401FEF7F0F990
:101D200002460B463F483B4C0DF004FD014698B17E
:101D300027480FF0AFF83C480FF0ACF8206802F0ED
:101D400083FD01460028ACD122480FF0A3F886E7B6
:101D500026480FF09FF8D1E734480FF09BF8344B3A
:101D600034480193CDF800A00FF094F8694620683C
:101D700002F04AFF0146E8B115480FF08BF82E48F3
:101D80000FF088F802F020FD0446B8B10146104873
:101D90000FF080F829480FF07DF829484FF0FF3206
:101DA0004FF0FF330DF0C6FC014600287FF479AFF9
:101DB0002448CAE724480FF06DF8E0E723480FF005
:101DC00069F82C70E6E700BFF0330100163401001B
:101DD0003234010043340100DA820020DB8200202B
:101DE0000702050C4C340100F800002067340100A4
:101DF0007134010004010020010160009C340100E5
:101E0000AE34010074030020D3340100F934010022
:101E1000DC8200201C0B0020D98200201F3501002D
:101E2000180B00208C0300203D35010063350100B4
:101E30004F36010088350100C3350100DD35010052
:101E4000A403002000360100A4350100D3350100B1
:101E5000014B1B68184700BF20010020014B186090
:101E6000704700BF2001002030B585B004460D4604
:101E700010220021684610F00FFD02238DF8023079
:101E80002A46044B0193214668460EF025FC05B016
:101E900030BD00BF511E000080B505460E461746F6
:101EA00098460EF0EFF8034610F08AFDDFF8189020
:101EB000044649F80030424630463946A84754F8AF
:101EC000090000F02BFC00BF080000002DE9F047DE
:101ED000058B04462807904611D4022905F0070512
:101EE00040F0CC8020460FF038F878B10138218BD3
:101EF000042811D8DFE800F0C2106D859500012993
:101F00000CBF45F0100545F02005258388F31188A6
:101F1000BFF36F8FBDE8F08701F0070AAA4500F014
:101F2000A5800027B9463E46A368002B00F0BC8080
:101F300041F00801218388F31188BFF36F8FA168F6
:101F4000002900F0BA800D68002900F0B680D1F8B1
:101F50000480334652462046C047002D76D02B6879
:101F600029461D46F0E701F007035A1F012A1BD836
:101F7000002221F00701062B276889B2C4E900225C
:101F800009D13B4603E0628B013262831B68002B60
:101F9000F9D141F00201218320460EF0DEFF002836
:101FA0007AD041F0200176E0042B0AD121F007011C
:101FB00089B2218320460EF0D0FF10B141F02001FC
:101FC0002183218B01F0070AAA454FD00027B9468B
:101FD000AAE7236921F0070141F00601062DD3F895
:101FE000009021832DD1B9F1000F3FD041F00801BD
:101FF000218388F31188BFF36F8F3A492046C84781
:1020000029E021F00701236941F0040189B2042D80
:10201000D3F804902183E6D000273E464FF0040A0F
:1020200082E721F00701236941F0050189B2052DFE
:10203000D3F808902183D6D000273E464FF0050AFA
:1020400072E700273E464FF0060A6DE72B4687E70A
:10205000B9F1000FD1D1EFF31188202383F3128857
:10206000BFF36F8F238B23F008032383258BEA06AE
:102070002ED525F01003238305F007056669218B13
:10208000002EBFF670AF00232768C4E9003321F0AB
:10209000070141F001012183218B01F0070AAA45C4
:1020A0004FF000097FF440AF002F9CD041F00801B1
:1020B000218388F31188BFF36F8F002FC8D03D684C
:1020C00039463346524620460EF073FF2F46F4E75A
:1020D000AB067FF51BAF25F02003238305F0070532
:1020E00000E700BFDF0F0100014B036000207047D5
:1020F000702D010008B504480EF0CCFE03480EF028
:10210000C9FE002008BD00BF5B360100903601000B
:1021100008B50348034A0021121A0FF044F808BD1D
:1021200070040020E88300200748084A084908B5E1
:10213000121A0FF03AF80748074A0849BDE8084064
:10214000121A0FF032B800BF000000206C0400200B
:10215000E43C01000000002000000020E43C0100FD
:1021600038B505460C4699B1D1E901230F480968F5
:102170000EF090FED4E90423E1680D480EF08AFECB
:10218000E1690C480EF086FEA1690B480EF082FE54
:10219000012D05D1EFF30581084810390EF07AFEC4
:1021A00021462846BDE838400DF04CB8BE36010047
:1021B000EE3601001E3701002E3701005D370100A9
:1021C00030BFFFF7FDBF00BF2DE9F0410B4EDFF838
:1021D000308006EB0807CC1B0546324609492046ED
:1021E00010F04CFBA01942460021083C10F054FBB3
:1021F000C5F8A84007F10800BDE8F0810000000024
:1022000004000000182D0100054B5A699B689A4292
:102210001FBF044A536843F080535360704700BFA8
:10222000B875002000ED00E02DE9F843324D8046FE
:102230003248894617460EF02DFEAB6ADE0622D5DF
:102240002F480EF027FE1124AB6A1D0703D52D4839
:102250000EF020FE1224284DAB6A980715D52A48A7
:102260000EF018FE6E6BAB6A190642D52748314650
:102270000EF010FEB9F1000F03D0AB6A23F080031B
:10228000AB62132403E01024DEE76FF015061A4D4D
:10229000AB6ADA0703D51E480EF0FCFD1424AB6AC6
:1022A0009B0603D51B480EF0F5FD1524124B9A6AC8
:1022B000D50602D49A6A90070AD55B68190507D536
:1022C0004146304600F00AFB10B180F30988022431
:1022D000094B9A6A920642BF5A6A22F400525A6225
:1022E0009A6A42F0FF029A6200233B702046BDE8E2
:1022F000F8836FF01506C4E700ED00E071370100C8
:1023000088370100BC370100D0370100E9370100F0
:10231000003801002038010010B51D4C1D480EF09A
:10232000B9FDA36A990130D51B480EF0B3FD1E20FC
:10233000A36ADA0103D519480EF0ACFD1F20144C36
:10234000A36A1B0303D516480EF0A4FD2120A36A3F
:10235000590303D513480EF09DFD22200C4CA36AAF
:102360009A0303D510480EF095FD2320A36ADB03E2
:1023700003D50E480EF08EFD2420054A936A6FEABD
:1023800003436FEA1343936210BD1D20D0E700BFE3
:1023900000ED00E050380100693801007D3801008F
:1023A00098380100B7380100DD380100F838010025
:1023B00070B5244C064624480D460EF06BFDA36A0A
:1023C000D90435D521480EF065FD1720A36A1A05FA
:1023D00003D51F480EF05EFD18201A4CA36A9B051A
:1023E0000FD51C480EF056FDA16BA36A180407D543
:1023F00019480EF04FFD1EB1A36A23F40043A362F7
:102400001920104CA36A590503D514480EF042FD5B
:102410001A20A36ADA050DD511480EF03BFD1B20EA
:10242000084A936A43F47F43936200232B7070BD84
:102430001620CBE7A36A9B04F2D50A480EF02AFDCA
:102440001C20EDE700ED00E0243901003B390100DC
:10245000BC3701004D390100673901007D390100A9
:1024600099390100203801002DE9F0415B4B5F688C
:102470008AB00446C7F30806002585F31188BFF328
:102480006F8F02F07F43B3F17F4F06D102F00C0350
:10249000082B13D152480EF0FDFC00252C464FF0BE
:1024A0000008F31E8DF80780092B00F28680DFE814
:1024B00003F00A7A7E7684848484848210074CBF79
:1024C0000C460125EBE74748444E0EF0E3FC8DF83F
:1024D0000780F36A9A0704D543480EF0DBFC00231B
:1024E00030E0F36A002B01DA4048F6E7F36A5B005C
:1024F000F5D53F480EF0CEFC7369A26943F48073B2
:102500007361BFF34F8FBFF36F8F736932F8022C83
:1025100023F480737361BFF34F8FBFF36F8F4DF65A
:1025200002739A4209D0B36ADBB253B30DF10702CA
:1025300001212046FFF778FE33E021682D480EF098
:10254000A9FC23689DF80720C2B902AE04F1200758
:1025500020686168324603C20834BC421646F7D18F
:10256000099AB5B3C2F3080121B96FEA52226FEAA2
:102570004222099202A91846FFF7F2FD0AB0BDE80F
:10258000F081B36A13F47F4F05D00DF107010120EC
:10259000FFF70EFF05E0B36AB3F5803F9FD3FFF767
:1025A000BBFE0346CEE70DF107020021C1E70DF1A6
:1025B00007010020ECE710488FE7104B1049114845
:1025C00017F4F87FA6F1100218BF19460EF062FC4E
:1025D00085E722F4FF7222F00102CAE700ED00E075
:1025E000E03901000C3A0100243A0100463A0100AA
:1025F000553A0100753A0100923A0100C7390100CD
:10260000B2390100B73A0100044B5A6942F0100296
:102610005A615A6922F008025A61704700ED00E0E1
:10262000EFF30880EFF3098101B57246FFF71CFF55
:1026300001BD00BF002080F31488BFF36F8F1148E5
:1026400080F308880020104908700CF0ADFA0020D3
:102650000E490860BFF34F8F00F02EF8202080F362
:1026600011880B484FF40461401880F30988EFF398
:1026700014800221084380F31488BFF36F8F00F0A9
:10268000FDF80000C0A00020E583002094ED00E0EC
:10269000009300200749D1F890200023C2F30722BD
:1026A0001846934200DB7047C1F89830C1F8A0008B
:1026B0000133F6E700ED00E008B572B6002383F3BE
:1026C0001388FFF7E7FF144B4FF0FF32C3F8802069
:1026D000C3F88420C3F88820C3F88C20C3F8902066
:1026E000C3F89420C3F89820C3F89C20C3F8802135
:1026F000C3F88421C3F88821C3F88C21C3F8902142
:10270000C3F89421C3F89821C3F89C2162B6BFF3A3
:102710004F8FBFF36F8F08BD00E100E0084B9B684F
:1027200083420BD1EFF3058343B1064B5A6842F065
:1027300080525A605A6A22F400425A620DF0A8BCD4
:10274000B875002000ED00E015498A684FF03000B0
:102750001044EFF3098C80E8F01F202080F31288EA
:10276000BFF36F8F0F4F4FF000664A698A603E607B
:10277000D2F8A8000C4C2060D2F8AC000023C2F8BC
:10278000AC3080F3118804B5104600F00FF9BDE8B5
:10279000044002F1300090E8F01F8CF30988704784
:1027A000B875002004ED00E0200B00201EF0040F9F
:1027B0000CBFEFF30880EFF30980816911F8021C68
:1027C0000229FFD001B572460EF0F1FC01BD00BF39
:1027D00040B2002807DB044A4109012300F01F0032
:1027E000834042F82130704700E100E040B2002809
:1027F0000CDB4309064900F01F0020330122824010
:1028000041F82320BFF34F8FBFF36F8F704700BF96
:1028100000E100E0054B420900F01F0053F82220C0
:10282000012303FA00F01040704700BF00E100E010
:1028300040B20028A8BF00F1604001F10101B8BF1B
:10284000064B4FEA4111ACBF00F5614000F00F00AC
:10285000C9B2B4BF195480F80013704714ED00E0FA
:10286000044B054A23F07F039360BFF34F8FBFF300
:102870006F8F70470000000000ED00E008B5FFF723
:10288000EFFF074AD2F8883023F47003C2F888308B
:10289000FFF73EFCFFF748FC00F05EF80CF09EFDF1
:1028A00000ED00E042F8203C009B42F81C3C0A4945
:1028B000019B42F8183C029B42F8143C21F00101B4
:1028C0004FF0807342F8043C42F8081C0023203A81
:1028D0000265C0F8AC307047991E00000A4A0346F2
:1028E000906878B113F1160FD0F8980005D0A0F1D8
:1028F00040029A4205D8834203D2814228BF002079
:1029000070470020704700BFB875002008B5154615
:102910000C4A0D4B9060D0F8A8201A600E4600F0CB
:1029200045F82C4686F309880020044B984720463A
:10293000002100220023024C20470000D311010097
:10294000991E0000B8750020200B0020014B1022BA
:102950001A61704700ED00E0044800232021C218EE
:102960000133302B82F80013F9D1704700E100E009
:1029700008B5EFF30583064A103B02EBC30152F89A
:10298000330049688847BDE80840FFF73DBC00BFF9
:10299000F42A0100024B034A0348012100F078B8F1
:1029A0000000022000000020702D0100D0F89820C7
:1029B000054B403A1A60054A4021C3E90112184606
:1029C000012100F06FB800BF240B002000000B15A0
:1029D000084AC2F898000B6823F01F03034343F032
:1029E0001003C2F89C308B6843F00103C2F8A0309A
:1029F000704700BF00ED00E02DE9F043DFF8608094
:102A000085B00E461F4604464FF00009B14523DA53
:102A10006068D8B13FB1411E08421BD11F2819D9A7
:102A20002368194216D1236801930EF0F5FBA368C1
:102A300003430393D8F89050C5F30725D0B2013D66
:102A4000A84207D801A9FFF7C3FF421C09F10109F9
:102A50000C34DBE76FF01502104605B0BDE8F083DB
:102A600000ED00E0044B0522C3F89420BFF34F8F24
:102A7000BFF36F8F704700BF00ED00E0BFF35F8FC3
:102A8000024B0022C3F89420704700BF00ED00E025
:102A900010B5034C01232278FFF7AEFF207010BD64
:102AA000E382002008B50B4A00231278FFF7A4FF49
:102AB00010F1160F07D0084A0021D2F89030C3F366
:102AC0000723984200DB08BDC2F89800C2F8A010A6
:102AD0000130F2E7E382002000ED00E02DE9F04351
:102AE0005B4B5C4CD3F890302568C3F307239D42C1
:102AF00085B000F2A980FFF7C1FF00200C268542B7
:102B00001BD1554C554F25706846FFF7EDFADFF89D
:102B10004081DFF84C9106460025AE4214D123785F
:102B20004B490020D1F89020C2F307229342C0F213
:102B30008580FFF797FF002045E0616806FB0011E4
:102B4000FFF746FF0130DAE7009800EB05114FEA86
:102B5000051CCB683B40B3F5000F4DD00AD8B3F548
:102B6000001F33D0B3F5800F3BD0B3F5801F13D0D7
:102B70000135D2E7B3F1007F47D0B3F1805F4DD08C
:102B8000B3F1807FF4D150F80C3088684A680EF0B9
:102B900043FB40F0887009E050F80C3088684A68C0
:102BA0000EF03AFB40F0885040F43020CDE901238C
:102BB0000390D8F890302078C3F30723013B984264
:102BC00035D96FF0150005B0BDE8F08350F80C3032
:102BD00088684A680EF020FB40F0885040F40020DE
:102BE000E4E750F80C3088684A680EF015FB40F0B6
:102BF000C06040F40030D9E750F80C3088684A686B
:102C00000EF00AFB40F08270D0E750F80C30886874
:102C10004A680EF001FB40F48020C7E750F80C3002
:102C200088684A680EF0F8FA40EA0900BEE701A990
:102C3000FFF7CEFE23780133237099E7C1F898306F
:102C4000C1F8A00001336DE74FF0FF30BBE700BFD4
:102C500000ED00E07C2D0100E38200200000F0FF89
:102C60000000021108B5024B1B689847002008BD00
:102C7000300B0020034B044A1860937843F00203A2
:102C800093707047300B00202401002008B50649DE
:102C9000064821F00701C1F1005202F500320EF0A2
:102CA000BAF8002008BD00BFABB30020340B0020F1
:102CB00070B54169867A0B4D044659B1437ADB07FA
:102CC00006D42C2303FB06535B6A1B689B6898475A
:102CD000002363612C20214606FB0050BDE87040B4
:102CE0000FF0A3BBBC030020024B2C2202FB0030E0
:102CF000704700BFBC030020827A064B2C2101FBE9
:102D000002339A6A1B7F1B33801A23F00303B0FB44
:102D1000F3F07047BC03002038B5074B827A2C24AF
:102D200004FB02335B6AD3E901240C601568FFF7EA
:102D3000E3FF04FB005038BDBC0300202DE9F04345
:102D400085B005466846039190461C460FF0E6FCA8
:102D5000DDE90067EFF31189202383F31288BFF3C5
:102D60006F8F6B8B002B41D02A8B9A4225D9002282
:102D7000002328460CF072FC0446F0B189F3118858
:102D8000BFF36F8F039B002B41D032463B46684612
:102D90000FF0E9FCA27A264B2C2101FB02332046DE
:102DA0005B6A1B6803A91D68DDE90023A847606111
:102DB00070BB2046FFF77CFF24E0698B4B1E6B83C2
:102DC00089F31188BFF36F8F2B7F2A8BAC6A1B337B
:102DD00023F00303521A02FB0344154B154AEB1A66
:102DE0009B105343A3722B7FE372CBE789F31188C7
:102DF000BFF36F8F2346424628460CF02FFC044653
:102E00000028BFD10024204605B0BDE8F0836361EF
:102E1000012300252381039B6382E27A65602946B2
:102E200004F118000FF038FD63692582E360EAE7DA
:102E3000BC030020A38B2EBA70B50D4C2C2500B915
:102E400070BD037A4668002BFAD0013BDBB20372F7
:102E5000002BF5D1C3604360837A05FB03431B6AF3
:102E600013B198473046EAE7FFF722FFFAE700BFC1
:102E7000BC030020044A0123C2F840354FF08042D1
:102E80000020C2F87835704700E0014048B1054B9A
:102E9000054A1B68B3FBF2F35843044B43F00103AC
:102EA000184770475403002040420F00402D010096
:102EB00008B50448044A3C23C0E900230BF01AFF7C
:102EC000002008BD400B00203FC00F0010B50EF0E1
:102ED0007EFA0FF0FFFA0E4C30B1BFF35B8F236820
:102EE000BFF35B8F7BB910BD0CF0D8FFBFF35B8FD6
:102EF0002368BFF35B8F1BB9BDE810400CF0E2BF45
:102F00000A209847F8E7BDE810400A20184700BF9C
:102F1000480B002038B5044608480EF098F90546DD
:102F200048B1631EDBB21F2B96BF054A0021D15C5E
:102F30000C300EF0FAF9284638BD00BF140400200A
:102F4000ED3A01000E38012810B50AD809480EF0F4
:102F50007EF9044618B104210C300EF0E6F9204643
:102F600010BD09B10448F2E7BDE810400220FFF7A8
:102F7000D1BF00BF40040020BC03002010B586B0C4
:102F8000084B039303AB00240093074907484FF015
:102F9000FF334FF48062CDE904440CF0F9FC204685
:102FA00006B010BD0D3B010000840020700400201D
:102FB00008B501F023F9BFF35B8F084B1A68BFF324
:102FC0005B8F02F00B02BFF35B8F53E8001F43E8F7
:102FD00000200028F9D1BFF35B8F08BD88000020D6
:102FE00010B5012104460C300EF0C0F92146034A09
:102FF0000078BDE8104000230EF03ABA4C2E0100D4
:1030000010B5012104460C300EF0B0F92146034AF8
:103010000078BDE8104007230EF02ABA142E0100F4
:1030200010B5012104460C300EF0A0F92146034AE8
:103030000078BDE8104000230EF01ABAFC2D010004
:103040002DE9F047884616468246002872D0BFF325
:103050005B8FDFF8E490002359E8004F49E8003225
:10306000002AF9D1BFF35B8F002C63D02046FFF715
:1030700043FE324D0C2303FB005027464388534543
:1030800011D0BFF35B8F59E8003F49E80072002A76
:10309000F9D1BFF35B8F002B4CD01F463846BDE8FB
:1030A000F047FFF7C9BEA64208D020460EF0CAF886
:1030B000328AF16804F10C000EF02EF92046FFF779
:1030C0001BFE0C2606FB00504368ABB1B8F1000FA5
:1030D00012D12046FFF710FE06FB00500121426886
:1030E000D2E90003127A03F01F06B1405B09DAB19E
:1030F00000EB83000EF0A9F92046FFF7FDFD0C263A
:1031000006FB00508368002BC8D02046FFF7F4FD73
:10311000704305F800802046FFF7EEFD06FB0055E2
:10312000A8680CF0CDFAB9E7C94300EB83000EF0B4
:10313000B6F9E1E7BDE8F087C00000204C0B0020A5
:103140002DE9F8430C460CF0A9FEE268218A1378B9
:10315000042B6DD1022908D82046FFF76DFE00240C
:103160000CF0B0FE2046BDE8F88353783E2B08D122
:103170000329F1D0D378012B01D00A2B49D10327A1
:1031800005E0052BFBD00E3B012B42D8012704F1B3
:103190000C0630460EF0FAF8012105463046B4F828
:1031A00010900EF0DBF8022130460EF0DFF80378C5
:1031B0003E2B804607D1E3681B78012B01D00A2BF8
:1031C00006D1032614E0052BFBD00E3B012B29D999
:1031D0001A4A1B491B4841F27B130DF068FE00237D
:1031E00083F31188BFF36F8F0323184602DF022693
:1031F000154A98F80000032321460EF039F9B2076A
:1032000012D56369A4F8109013FA85F5E560BB0741
:10321000A5D521460D480EF01EF80D490D480FF0BA
:1032200043F99CE70126E3E72046FFF705FEEEE7BA
:103230002046FFF701FE6FF0150491E71D3B0100EA
:10324000513B01006A3B0100E42D0100C400002055
:10325000C80100204805002038B51C480EF010F8C1
:10326000044688B300F10C0528460EF087F80428C0
:103270001DD1284602210EF079F803780E3B012B70
:1032800005460ED8124A1349134840F6B2430DF0D2
:103290000EFE002383F31188BFF36F8F03231846BC
:1032A00002DF0E4A2878032321460EF0E1F820467B
:1032B000FFF7C2FD0A4BD3F8C4302BB1BDE838404C
:1032C000084909480FF0F0B838BD00BFC40000201D
:1032D0001D3B0100873B01006A3B0100FC2D010002
:1032E00000000020C80100204805002010B5C1E9F9
:1032F00000239DF808300B720C46FFF7FDFC034BD2
:103300000C2202FB00335C6010BD00BF4C0B0020A0
:10331000F8B502460B4610480DF099FF0446C0B1BF
:1033200004210C300DF0EEFF2046FFF7E5FC0B4DBD
:103330000C2707FB0050002646802046FFF7DCFCE8
:1033400007FB005086602046FFF7D6FC07FB0055C0
:103350006E602046F8BD00BFE80300204C0B002043
:103360000138C0B202289ABF014B185C0020704798
:10337000133C010002289ABF014B185600207047E9
:10338000103C0100034B0146D3F8E40082689268C8
:10339000104700BF0000002008B5044804210EF0CB
:1033A00054F8BDE8084000F029BF00BF88000020A5
:1033B000014902480FF078B8B801002070040020DD
:1033C00070B505460C4659B94FF0FF304FF0FF314C
:1033D000FFF79EFF044618B96FF06805284670BDD8
:1033E0002046FFF789FC164B0C2202FB0033A6187F
:1033F00030465D800DF0CAFF03280BD9032130460B
:103400000DF09BFF0580238A033B8370012130462A
:103410000DF09BFF40F635439D4208D12046FFF753
:10342000B1FF054648B12046FFF706FDD6E705483F
:1034300021460EF0EFFFFFF7BBFF0025CEE700BFF0
:103440004C0B0020CC0000202DE9F043064687B04D
:1034500017460C4669B94FF0FF304FF0FF31FFF7C8
:1034600057FF044658B96FF06805284607B0BDE815
:10347000F083887AFFF738FC304B834258D1012221
:10348000002168460EF0DBFF2046FFF735FCDFF831
:10349000B0900C2303FB0090C0F808D020460DF03C
:1034A00005FF01463046FFF78BFF054618B1204661
:1034B000FFF7C2FCD9E74FF4A022002368460CF0C6
:1034C00039F9804690B14FF4FD731E4A1E491F48DA
:1034D0000DF0EDFC1E48424631460DF0E8FC85F348
:1034E0001188BFF36F8F0323184602DF2046FFF7D2
:1034F00003FC0C23584319F80060AEB12046093E86
:10350000FFF79AFC092E0CD8DFE806F0150B0B0824
:10351000050B0B0B0B126FF00B05A6E76FF00C05FC
:10352000A3E76FF00405A0E7002FC0D03C609CE744
:103530006FF0150599E76FF06E0596E7E803002038
:103540004C0B00201D3B0100B53B01006A3B010014
:10355000BE3B0100F7B50022114640F60340FFF7DD
:1035600073FF0446002850D1FFF722FD214601AA2F
:1035700041F20300FFF768FF0446002845D1019A95
:103580009D4DD168D1F80100D1F8051005F12C034B
:1035900003C31046FFF750FC214601AA41F2010087
:1035A000FFF752FF044680BB0198C3685A7885F83C
:1035B00024205A88EA841A7985F82520B3F8072050
:1035C0002A85B3F805306B85FFF736FC214601AA42
:1035D00041F20200FFF738FF0446B0B9019FFA68D4
:1035E00005F13406531C413218685968344603C447
:1035F000083393422646F7D13846FFF71DFC95F86D
:1036000030305F0604D46FF01204204603B0F0BDE2
:1036100001AA002142F20300FFF716FF044600282A
:10362000F3D1019A754BD168D1F80100D1F805109A
:1036300003C31046FFF700FC95F830309E0619D4FE
:103640004FF0FF304FF0FF31FFF762FE06460028D3
:1036500000F0B88002210C300DF058FE01234470B8
:1036600003702246314640F66D40FFF7EDFE0446FA
:103670000028CAD195F85030180712D501AA0021A8
:1036800042F21C00FFF7E0FE04460028BDD101987D
:10369000C368D3F80120D3F80530C5E92623FFF726
:1036A000CBFB95F8923013F0180F01D1190604D511
:1036B00001F08AFA04460028A7D14FF0FF304FF0FE
:1036C000FF31FFF725FE044600287BD008210C308F
:1036D0000DF01CFEF0230022437002279723077091
:1036E0008370C270027142718271C271214642F2CE
:1036F0000100FFF7A9FE0446002886D14FF0FF30F5
:103700004FF0FF31FFF704FE064600285AD008218B
:103710000C300DF0FBFD8023437020230470847077
:10372000047144718471C770C3712246314640F6FA
:103730000140FFF789FE044600287FF466AF01468A
:1037400001AA4FF60140FFF77FFE044620BB019817
:10375000FFF772FB214601AA4FF60240FFF774FE05
:103760000446C8B90198C368B3F80130A5F87530AC
:10377000FFF762FB95F875305A070DD501AA21466F
:103780004FF60340FFF760FE30B90198C3685B78DD
:1037900085F87430FFF750FBEB7923B903B0BDE82F
:1037A000F04000F0C3BA2E78002EF7D195F87530AE
:1037B0009B061ED54FF0FF304FF0FF31FFF7A8FDFD
:1037C000044610B96FF068041FE706210C300DF0B5
:1037D0009DFDD5F801300360094B9B88838021460D
:1037E00032464FF60640FFF72FFE04460028D5D09C
:1037F0000BE76FF0850408E7000000209000002030
:103800000100002073B5264D0646D5F8E4000EF001
:10381000E4FC00283CD06FF0020105F188000DF0B7
:103820003EFE01210DF011FE10EA010433D11D4BC3
:103830001E600A4605F1A8000EF001FE05F1CC005D
:103840000EF0A9FD18480EF03FFE184916480094E6
:103850006FF007034FF496620CF09AF8144912487F
:103860000CF0D6F8D5F8E400124983681B68984735
:10387000044628B93EB9FFF76DFE78B9FFF78CFD15
:10388000204602B070BD05F178000CF07BF8F7E738
:103890006FF01204F4E76FF07704F1E70446EFE706
:1038A00000000020580B0020480500204088002020
:1038B000033C01004131000010B5FFF74BFE044608
:1038C00008B9FFF769FD044B1B681BB12046BDE832
:1038D0001040184710BD00BF580B002038B5032119
:1038E00004460C300DF042FDE3680578B0F80100A5
:1038F000197840F6354398420AD02246FFF7A0FBDC
:1039000035B104480BF0DCFEBDE83840FFF750BD90
:1039100038BD00BFA800002038B50CF0BFFA274D15
:10392000D5F8CC30002B44D00022002305F1A800AC
:103930000BF000FF00283CD10022002305F1CC0051
:103940000BF08CFE044668B91D4A1E491E4840F61D
:10395000C2430DF0ACFA84F31188BFF36F8F0323D9
:10396000184602DFD5F8C00020B1FFF765FA002342
:10397000C5F8C03020460DF099FCC5F8C0002046BF
:10398000FFF700FD98B111480BF09AFE2046FFF7B3
:10399000B3F90F4B0C2202FB00301F214088224656
:1039A000FFF74EFB2046FFF747FAFFF701FDFFF751
:1039B000FFFCBDE838400CF085BA00BF00000020D5
:1039C0001D3B01000C3C01006A3B0100A8000020E7
:1039D0004C0B002038B5042104460C300DF0C6FC19
:1039E0004578017840882246FFF72AFB35B1044824
:1039F0000BF066FEBDE83840FFF7DABC38BD00BF0B
:103A0000A800002070B54FF0FF320D464FF0FF3395
:103A100000210646FFF796FA044660B90A4A0B49A8
:103A20000B481A230DF043FA84F31188BFF36F8F0C
:103A30000323184602DF022104F10C000DF066FC9E
:103A400006704570204670BD163C01000C3C01001C
:103A50006A3B0100F8B50A4DEF7906460024E3B24F
:103A60009F4202D86FF0010007E0294630460DF072
:103A700046FD0735631C08B12046F8BD1C46EEE73D
:103A80000000002070B5144E0622314604460EF0A8
:103A90000BFFD8B14FF0FF304FF0FF31FFF738FC8C
:103AA0000546A8B1062221460C300DF035FC002257
:103AB000294642F20500FFF7C7FC40B933462268A9
:103AC00043F81D29A288B28001221A77002070BD18
:103AD0006FF06800FBE700BF1D00002037B504460B
:103AE0000D4689B1184928460DF009FD60B9174AFD
:103AF0002968C4EBC404A3181151AA889A80AA7932
:103B00009A71002003B030BD68460DF043FC0028D8
:103B1000F8D16846FFF79EFF0028F5DA0B4A0098B7
:103B20009DF80610C4EBC404A3181051BDF804009E
:103B300098809971002DE4D012592A609A88AA8041
:103B40009B79AB71DDE700BFDA3A0100000000208D
:103B500070B5044611B16FF0150070BDF0B1234986
:103B60000DF0CDFCD0B92046FFF774FF002837DAFE
:103B7000237863B91E4AD37993BB20681060A1797A
:103B8000A088917101219080D1711846E5E7012B41
:103B9000E1D1A37903F0C003C02BDCD1144DEB7944
:103BA000012B20D0BFF35B8FD5F88830BFF35B8F3C
:103BB000DB0707D4002CCED00C4920460DF09FFC2B
:103BC0000028C8D1EE792146731C3046EB71FFF70F
:103BD00085FF08B93046C0E7EB79013BEB71BCE7E4
:103BE0006FF07700B9E76FF00B00B6E7DA3A010043
:103BF000000000202DE9F3410446D8B101AA0021BC
:103C000041F20900FFF720FC054698B9019E1249D0
:103C1000D6F80C8008F10107062238460EF044FE63
:103C200028B10E49062238460EF03EFE30B9304625
:103C3000FFF702F9002002B0BDE8F081D8F80130AA
:103C4000C4F80130BB88A4F8053030462570FFF772
:103C5000F3F80120EFE700BFE73A0100E13A010085
:103C600007B56846FFF7C6FF044BD87118B169461F
:103C70000020FFF733FF03B05DF804FB00000020D5
:103C8000F0B5294DEE7989B0002E46D195F8763001
:103C9000DB0722D56A4631464FF60940FFF7D4FBD1
:103CA000D8B9DDF800C0DCF80C406378012B1E4663
:103CB00028BF012673B1A31C02AA123418685968E0
:103CC000174603C70833A3423A46F7D1186838604D
:103CD0009B88BB806046FFF7AFF8EE710024162684
:103CE0000127EB79E0B2834202D8B3B1002012E0A1
:103CF00008AB06FB0033694653F8182C33F8143C24
:103D0000CDF80120ADF805308DF80070FFF7E6FE24
:103D100001340028E5D009B0F0BD0021084609B003
:103D2000BDE8F040FFF714BF0000002010B50A4CBA
:103D3000E3790BB1002010BDFFF792FF0028FAD104
:103D4000E379002BF6D1FFF79BFF0028F3D1601C2D
:103D5000BDE81040FFF796BE00000020034B002294
:103D600099689A801960024B1A727047D801002036
:103D7000E4820020F0B5054687B00F464FF0FF30D3
:103D80004FF0FF311646FFF7C3FA0446C0B10621D3
:103D90000C300DF0BBFA46800026477005700671A6
:103DA0004671094A009503A920460523FFF79EFAAC
:103DB0003246214642F24200FFF746FB07B0F0BD13
:103DC0006FF06800FAE700BF8800002008B50246DF
:103DD000014607480DF0E5FB30B922B905480DF062
:103DE000DAFB40F3C01008BD6FF07700FBE700BFBF
:103DF0007C0B00208800002038B50546407A0C4630
:103E0000FFF7AEFA2073A87AFFF7AAFA607395F964
:103E10000C30A37195F90D306371EB7A2371EB8946
:103E200063812B88103BDBB20B2B96BF054A052321
:103E3000D35CE3712B8883F0100303F01F0323810D
:103E400038BD00BF4C3C010037B50546C379009032
:103E500014308DF804308DF805100DF0CEFB0C4BAE
:103E60001B689BB11C6804B1183C53F8143C13B197
:103E70006946284698474CB12346A4695B681CB143
:103E8000183C002BF4D1F7E7002BF1D103B030BD83
:103E90005C0B002008B5054B18460DF07CFB143B6D
:103EA00010F0040F14BF1846002008BD780B002046
:103EB0002DE9F04788B08A48002200230BF006FB6A
:103EC000002840F09B808748864D0DF064FB10F081
:103ED00001034ED02B1D93E8070008AB03E9070050
:103EE00081480DF058FBC0F340137E480DF053FBA2
:103EF0000246002873D073B17C490C2205A80EF04D
:103F0000D3FC002875D0002211461046FFF732FF7F
:103F1000044600286ED19DF81530190703F00405FA
:103F20006FD5002D40F0938028462E46BDF81A30FC
:103F300063B1BFF35B8F6C4B53E8001F41F040014E
:103F400043E80012002AF7D1BFF35B8F0DF10301A4
:103F50000DF0FAFA044600284CD14FF0FF304FF034
:103F6000FF31FFF7D5F9074600287BD16FF06804D1
:103F700040E05D485E4A0DF00EFB10F0800F0ED061
:103F80009089D1891269ADF816004FF48074ADF8AC
:103F90001440ADF81810ADF81A300792A0E7554C50
:103FA0002068616805AB03C3A068186092F891307F
:103FB0004C481E0744BF05238DF815300DF0EBFA71
:103FC000840706D53023ADF818306023ADF81630DD
:103FD00086E744480DF0DFFA4007F3D480E743B1A9
:103FE0000146FFF7C7FE044620B9404B2861C3E9EC
:103FF000010000243A480BF0E1FA204608B0BDE881
:10400000F087BDF816309DF81400ADF80530BDF806
:1040100018308DF80400ADF80730D5B101AEBDF809
:104020001C200AB9BDF81620BDF81E300BB9BDF82A
:1040300018309DF814108DF80C10ADF80D20ADF867
:104040000F305EB13078012808D103AD6EE700264D
:10405000E5E7421E5042504101AE67E74B1E584211
:104060005841F2E700F10C09032148460DF04EF9E2
:104070009DF815809DF803300370C8F34003824615
:104080008470437036B1012383700522314648465F
:104090000DF042F955B19AF8023043F004038AF862
:1040A00002300522294648460DF036F900223946ED
:1040B00042F24100FFF7C8F9044600289AD1BDF842
:1040C0001A2008F001010120FFF754FE04460028E1
:1040D00090D108AA12E90700044B83E8070088E79B
:1040E000980B00207C0B0020880000208C0B002007
:1040F00000000020282D01002DE9F3470546374830
:104100000DF049FA9946034634480DF044FA144636
:10411000DA070E4602D50B895B075CD428460DF002
:1041200052F9002846D0294668460DF041F92C4F37
:104130003B68A3B120460DF029F9B4F80480A4F837
:104140000490054623463F68F27996F905106846C3
:10415000B847A368A4F8048013FA85F52560214BBD
:10416000C6F800D01B68002B33D01D6805B1083D90
:1041700053F8082CAAB12F46A3F1080520460DF0EC
:1041800005F9B4F804A0A4F804902B6880462146F1
:1041900030469847A368A4F804A013FA88F3236074
:1041A0003D46B5B1AF682B688FB1083F002BE5D114
:1041B0003D46F7E72B78FF2B04D10B4968460DF0FD
:1041C000FCF9B4E729460DF0A2F90146F6E7002B09
:1041D000D4D10023336002B0BDE8F0877C0B00200F
:1041E000C80B0020C00B0020DA3A0100024B00226D
:1041F0001A60FFF7B3BD00BFC80B002010B5094C13
:104200004422002120460EF047FB04F11C000EF072
:1042100031F804F130000EF02DF8BDE81040FFF742
:10422000E5BF00BF7C0B0020032838B5054603D14D
:10423000BDE83840FFF73CBEFFF7C8FD044658B95B
:10424000064829460DF0E5F9FFF732FE044618B19D
:10425000024829460DF0C7F9204638BD7C0B0020E6
:10426000032808B5014602D003480DF0BCF9BDE8AB
:104270000840FFF71DBE00BF7C0B002010B50020DA
:10428000FFF7EEFF20B10BF059FE0020FFF7E8FF2B
:104290006FF0400111480DF097F910486FF48071EC
:1042A0000DF092F90E4B1B68B3B11C6804B1083CC9
:1042B00053F8043C03B1984774B1A268234642B155
:1042C0005B68A2F10804002BF5D1F6E7BDE81040C9
:1042D00018476368002BF9D110BD00BF880000208B
:1042E000C00B00202DE9F04F00F10C0989B0074602
:1042F00048460DF043F806464C484D4DDFF834A1D2
:104300000DF049F900F00103484802930DF043F91C
:10431000C0F38003019326B1029B2BB13B8A172B7C
:104320000AD809B0BDE8F08F2B7A0BB1FFF716FD64
:10433000019B002BF2D1F4E7182148460DF016F846
:104340003A8A90F817B003885A45C3F341180446D7
:1043500003F010030AD2384601930CF073FF019B5F
:10436000002BDED1324B02221A72DAE77BB104A9AC
:10437000FFF742FDE37D4A4604A9A01CFFF7BCFEFF
:10438000E17D48460CF0EAFF013EF6B2C3E72B7A26
:104390002BB9B8F1000F19D104A92046E8E7C17A7A
:1043A000EA7991420DD1811C0722284603930EF031
:1043B0007BFA039B28B9B8F1020F12D1FFF7CEFCAC
:1043C000DEE7B8F1000FE7D0012BD9D0B8F1020F2A
:1043D000F4D0A11C2846E27A0DF0EFF80123EA712F
:1043E0002B72BAF80430BAF806205B44934205DD1C
:1043F00002232B72B8F1010FC2D0DFE72B7A022B18
:10440000F8D0F9685A4650460CF086FFB8F1010F13
:10441000BAD004A92046FFF7EFFCBAF804305246A0
:1044200004A9A01CFFF768FEC8E700BF7C0B0020B2
:10443000E4820020D801002008B5074B1A89824287
:1044400005D103F114000DF0A6F8820701D4002075
:1044500008BD1846FCE700BF640B00202DE9F047BB
:10446000164B1B6880460D4691462BB31C6804B161
:10447000183C53F8102CA2B12646A3F11804284684
:104480000CF084FFA368B5F804A007462A46494605
:1044900040469847AB68A5F804A013FA87F72F6049
:1044A00034464CB1A669A36826B1183E002BE6D16C
:1044B0003446F7E7002BE2D1BDE8F0875C0B002023
:1044C000F0B587B0C568FFF7E5FC044620B92B7846
:1044D000442B13D107B0F0BD00F114060221304681
:1044E0000DF081F80120FFF7BBFE2B78442B05D19E
:1044F000304607B0BDE8F0400DF07FB82E1D3046C5
:104500000CF061FF314640B168460CF051FF5CB9D8
:10451000B5F801000DF025F8DCE70CF0F8FF0146D6
:1045200068460DF04AF8F2E704F11406032130461C
:104530000DF037F8F8B9E279EB789A4214D0B5F873
:1045400001000DF00EF81F27032130460DF029F869
:1045500028B1694620460DF030F8EB78E371394612
:104560002046FFF771FCB5E70722694620460EF0AA
:104570009BF90028E3D12F78002FE5D101213046A7
:1045800027740DF046F8B5F801302381AB896381BB
:10459000AB7BA381E87AFEF7E3FE3946A0731022D5
:1045A00002A80EF079F96389ADF80E300321A37BE0
:1045B0008DF8103030460CF0F4FF48B1EB78E37121
:1045C00020460CF000FF6946D0B120460CF0F0FE0A
:1045D000E3798DF80C300421304602940CF0E1FFB1
:1045E000124B1B6880F001008DF81100002B3FF486
:1045F00071AF1D6805B1183D53F8183C3BB909E08F
:1046000020460CF0DAFFE3E7002B3FF463AF02A98A
:1046100020469847002D3FF45DAF2B46AD691B68DF
:10462000002DF1D0183D002BF1D1F6E75C0B0020F6
:1046300010B586B001AA02A90DF04AF8B0B90C4B2A
:104640001B689BB11C6804B1183C53F8043C13B1BF
:10465000019802A998474CB12346A4695B691CB133
:10466000183C002BF4D1F7E7002BF1D106B010BDB8
:104670005C0B00202DE9F04F00F10C0785B00646D9
:1046800038460CF07BFE05462548DFF898B00CF064
:1046900082FF00F0010922480CF07DFF4FF0010A73
:1046A000C0F3800815B905B0BDE8F08FB9F1000F6F
:1046B00002D1B8F1000FF6D0338A082BF3D90921C3
:1046C00038460CF053FE037A328A01339A4204468C
:1046D000E9D3ADF80CA07F238DF80630037A0344AC
:1046E00069465B7A8DF80530FF238DF8043000238E
:1046F000ADF80A3002788DF80720042A98BF1BF81D
:104700000230ADF80830037A3A460130FFF7F4FC86
:10471000217A38460131013D0CF020FEEDB2C1E7AF
:104720007C0B0020583C0100F8B5054622480CF0EF
:1047300032FF43070F463CD52A78012A03D96FF090
:1047400015042046F8BD6B780F2BF8D86888031F36
:104750009BB243F6FC74A342F1D8A9880B1F9BB20D
:10476000A342ECD88842EAD37AB914480022002345
:104770000AF0ACFE04460028E3D1FFF727FB04460D
:1047800040B10E480AF01AFFDBE70CF0DBFE002810
:10479000EBD1D4E728686968094E0A4B03C6A868BC
:1047A000306020461F60FFF73FFD044606F12400FD
:1047B000E8E76FF00A04C4E788000020AC0B002093
:1047C000800B0020C80B002008B5FFF70FFD0A4B37
:1047D0000A4800226FF040011A600CF0F5FE430613
:1047E00004D506486FF480710CF0EEFEBDE8084079
:1047F0000020FFF735BD00BFC80B00208800002057
:104800000A4B196800F1080231B98160596839B959
:10481000C3E90022002070478A4204D00968F3E708
:104820000A605A60F6E76FF010007047C00B002076
:10483000034BC01A034BC0105843C0B2704700BFAF
:10484000640B0020ABAAAAAA38B5224B93F891308A
:104850009B06054638D500F11402012110460CF0E4
:10486000A0FE80B1012110460CF09BFE78B3288990
:104870000CF077FE044620B916212846FFF7E4FA2B
:104880000024204638BDFFF705FBA8420246F7D1B9
:10489000FFF700FB82421AD10120FFF7E1FC04463A
:1048A0000028EED14FF0FF314FF0FF30FEF730FD22
:1048B000014630B1224642F24500BDE83840FEF7DD
:1048C000C3BD6FF06804DCE76FF08504D9E76FF0D3
:1048D0001504D6E7000000202DE9F843634A92F85A
:1048E00091309C0605460F4604D46FF0850420469F
:1048F000BDE8F883FFF7CEFA002840F0B180EB79ED
:104900000F2B00F2B080AB89B3F5FA7F80F0AB805B
:10491000EB890A3B9BB243F6F6718B4200F2A3800F
:10492000AB68580703D592F89430D906DDD55048C6
:104930000CF031FE10F0010602D06FF00B04D6E748
:10494000182231464B48DFF82C810DF0A5FF48486E
:1049500031460CF05EFE4FF0FF304FF0FF31FEF7B6
:10496000D7FC814630B908F114000CF046FE6FF018
:104970006804BCE70E210C300CF0C8FC0E22314656
:1049800004460DF089FFAB68DA0748D5032108F12A
:1049900014000CF03EFE237843F001032370AB6853
:1049A0009B0707D52378324843F002032370042184
:1049B0000CF02FFEAB685E0742BF237843F0040380
:1049C0002370AB68180742BF637B43F00103637336
:1049D000AB68D90642BF637B43F002036373AB68E5
:1049E0009A0642BF637B43F004036373AB685B06C4
:1049F00042BF637B43F010036373AB89A4F80930B3
:104A0000EB89A4F80B300022494642F24400FEF73D
:104A10001BFD044650B116480CF0EFFD67E7294630
:104A2000A01C0CF0CAFDEB796370B8E710480221B6
:104A30000CF0EFFD0120FFF7F7FB044630B1012039
:104A4000FFF70EFC0B48FFF7FFFE50E70948C7F8D9
:104A5000008029460CF0B1FDEB7988F8073046E775
:104A60006FF00F0443E76FF0150440E700000020EB
:104A7000780B0020640B00200A4B196800F1180223
:104A800031B98161596839B9C3E900220020704702
:104A90008A4204D00968F3E70A605A60F6E76FF0CB
:104AA000100070475C0B00202DE9F04F074687B0DF
:104AB00015460E4619B39378102B1DD81378DA07D4
:104AC0006ED55C0718D03D4B5A78012A14D93C4A60
:104AD00092F8922050060FD56A78022A04D0012A53
:104AE0000AD11A78510707D5EA78012A04D99B78A8
:104AF000934201D36B682BB96FF0150455E013781E
:104B0000DA074DD595F803904FF0FF304FF0FF31A5
:104B1000FEF7FEFB8046002845D000F10C0B062175
:104B200058460CF0F3FB0023036083803B8903802D
:104B300004468670BEB1AB7803712B78DB0743BFA8
:104B40006B78C370D5F804A0DFF878A080F80590E2
:104B50005CBF0223C370494658460CF0D7FB62790C
:104B600051460DF08BFE052307F1140203A94046C0
:104B70000096FEF7BBFB02AA414642F25300FEF745
:104B800063FC044688B902983A89C368B3F80130D7
:104B90009A4210D16EB12B78FB73FEF74DF904E009
:104BA0004FF00209B0E76FF06804204607B0BDE897
:104BB000F08F2346F0E76FF00404EEE7D283002085
:104BC000000000205D3C01002DE9F341002101AA15
:104BD00042F25800FEF738FC044670B90198C368E9
:104BE0005F789D7893F803801E79FEF725F9054BD1
:104BF00083F802801F70DE705D70204602B0BDE851
:104C0000F08100BFD283002008B50A46034610B9E0
:104C10006FF0150008BD0029FAD0094991F89210EB
:104C2000C9060AD5012114300CF049FD0028EFD047
:104C30001846BDE80840FFF737BF6FF08500E9E789
:104C40000000002000F1070C2CF0030C10B4541EDF
:104C50001860A4B2ACF80020023A93B201FB04F24F
:104C60004FF0000C40F802C074B103FB011403FBC9
:104C700001F22044121B4FF6FF7C013B9BB26345BF
:104C80008050A0EB0100F8D110BC704703460068CB
:104C900010B102680AB91A60704700F1070C2CF0D5
:104CA000030CD11DBCF800C021F003010CF1FF3C46
:104CB000A1F800C0EFE700BF0B687BB1073323F01A
:104CC00003031A88013292B20346D1F800C043F8B8
:104CD00007CB23F003031A80086070470122F3E733
:104CE000401A90FBF2F080B2704700BF531E11448F
:104CF0009BB242B1DB430138CA1811F8013D00F8FC
:104D0000013F9142F9D17047014402E010F8013BA4
:104D10001BB98842FAD1002070470120704700BFBC
:104D200010600860704700BFD2F800C0CCF80000E7
:104D3000D2F800C0CCF8041010607047884203D04D
:104D40001AB1436813607047002070470B688342B4
:104D500009D02AB1586810601A680A60184670476E
:104D6000002BF9D1FAE70023F8E700BF2DE9F04165
:104D7000DFF830800C4E0C2706F130044546221D2A
:104D8000214628460C3CFFF7CBFFA642A5F10805BB
:104D9000F5D1043F3B1DA8F12008A6F13006EBD168
:104DA000BDE8F081480C0020D40C002010B403466C
:104DB0008C469AB101EB4101144803EB430409010D
:104DC00001EB84010144487A0C7AA04204BF01300F
:104DD000087210BC6146184608F0CABC01EB4102DB
:104DE0000A4C120100EB400302EB830323449C7A3C
:104DF000DA7AA24201D010BC704701329A72044B99
:104E000001225A5410BC08F0E3BC00BF500C002033
:104E1000CC0B0020F8B506461C460D4602B322789E
:104E20006378D21A12F003023AD1274F71004FEA89
:104E3000450C3144AC44890001EB0C1101330431C1
:104E4000DBB27A18606823702146FFF76DFF1F4BB5
:104E50000122294630465A5508F0BAFC0020F8BD18
:104E600008F0A0FC0028DAD02946304608F08CFC77
:104E70000028D4D005EB450206EB4601124F6378BB
:104E8000120102EB81023A447100907AD27A904288
:104E90004FEA450C0CD02078C01A10F00302C8D09D
:104EA000012A03D00133DBB22370D0E71046F8BDEE
:104EB0002278D21A920702D00233DBB22370D4E9EF
:104EC00002039847CAE700BF500C0020CC0B00201B
:104ED0002DE9F04FDFF8649119F8003089B0002B0C
:104EE0005AD0DFF85CA13C2204234FF0000B00EB0A
:104EF000400712FB00330324CDE904BB09F800B0DE
:104F00000AEB0717039302948346B8460023B96A55
:104F100058F8240F079307AAFFF710FF044607AAC3
:104F2000B4B1079D2E786978761A06F00306012E33
:104F300035D02B78591A01F003010129DBB23DD19C
:104F4000D7E90901FFF7FAFE044607AA002CE8D1C9
:104F500097F82E3097F82F209A4203D087F82F30F9
:104F60000123049397F82C3097F82D209A4203D010
:104F700087F82D3001230593029B5D1EEBB2FF2BBA
:104F80000293A7F10C07C0D1049AD846DDF814B0FB
:104F900012B1BBF1000F45D009B0BDE8F08F013967
:104FA0006970079BD3E902039847079D2A786978BF
:104FB000D3B2521A02F00302012A21D0B86A019337
:104FC00000224146FFF7C2FE6C60019B6A786B705D
:104FD0002B789B1A03F00303012B08D0D7E90901B2
:104FE00007AAFFF7ABFE012E044698D10EE0039B03
:104FF0006A70294620460AEB0302FFF795FEEDE7AB
:10500000D7E9090107AAFFF799FE0446029B8BB175
:1050100001235946584609F80B3008F0D9FB09B06E
:10502000BDE8F08F5A464146404609B0BDE8F04F12
:1050300008F09EBB002C8BD0EAE700BFCC0B002011
:10504000500C00204B1EDBB271B1411E00EB030C73
:10505000002011F8013F23B15A1E01301340C0B2A5
:10506000FAD16145F5D170470846704732B370B543
:105070004FF0000E04460E46F44670464FF0FF35E2
:10508000C6F108035FFA8EF19342A8BF1346615C34
:10509000DBB2314105FA03F621EA060101FA0CF10F
:1050A0009C44D31A13F0FF0240EA01005FFA8CFC23
:1050B0000EF1010E4FF00006E2D170BD10467047B0
:1050C00030B5027E0568FF2A18D002EB820302EB9E
:1050D00043038A4205EB83032BD04FF0000C01E021
:1050E00091420DD096461A789C6802EB820302EB3F
:1050F0004303FF2AA44405EB8303F1D1002030BD14
:10510000714519D00FFA8EFE98681B780EEB8E024F
:105110000EEB420EFF2B05F82E3008D003EB830276
:1051200003EB420305EB83039A6802449A606044F0
:1051300030BD96464FF0000C1A780276E2E700BFC9
:10514000A2EB010C1CF4000F10B4836844690AD16F
:105150002CF07F4C6344A3420DD8E41A0023446131
:10516000836010BC7047891A21F07F418B4208D9B7
:105170005B1AA342F1D91B1B00244461836010BC5D
:1051800070470C44E41AE9E72DE9F04F87B0427A02
:10519000036844680293002A00F0F380531EDBB2D8
:1051A00004EBC3038B46039305948246039B5A6822
:1051B0005E780492BBF1FF0F69D00BEB8B030BEB16
:1051C0004303029ACDF804B012F823B04FEA8308E3
:1051D00002EB830400254FF0FF0C84F800C0DAF8DE
:1051E00000709AF8183007EB08096345D9F80810E1
:1051F0000FD1C0E0091A06D1B9F81E80BEF81EE032
:10520000F04500F2AC8017F82220FF2A9C46134696
:1052100009D003EB830203EB420207EB820EDEF8B8
:1052200008008842E6D9BCF1FF0FC9F8081089F8D8
:10523000003000F090800FFA8CFC0CEB8C020CEB31
:10524000420C019A07F82C20FF2B08D003EB8302B5
:1052500003EB420307EB8307BB685B1ABB60A378D1
:1052600001336370002DA5D06B6A4FF000022A70E5
:10527000AA7013B1A96A002098476368002B99D1DE
:105280006B6A2362AB6A6362BBF1FF0F95D1039B2C
:10529000049F9A7806EB860306EB4303711CB24227
:1052A00007EB8305CEB25CD00399087817F823107A
:1052B000B04208BF00260429ECD16A78029902EBBB
:1052C000820802EB480801EB8804012094F801C031
:1052D000A1788C454FEA88080BD04FF0000207F800
:1052E00023206B6AA8700BB1A96A9847039B9A7830
:1052F000D0E7AB8A01924FF6FE729342DAF81410AF
:1053000007D04FF6FF729B1AB3FA83F35B0984F858
:105310002830EB6863602B69236200226262AB8AEB
:105320004FF6FD70834288BF1346A383AB69A36128
:10533000EB69E3602B6A2361AB68A36062616A6812
:105340002046FFF7FDFE4FF00003E383E37843F0D0
:105350000103E3703FE7019A8AF8182074E70146D9
:1053600061E7039B05995A701A469142A3F108031D
:1053700007D003931AE707F80830019B8AF8183022
:105380006DE707B0BDE8F08F2DE9F04F467E0123B1
:105390008BB08376002E40F0BB80037EFF2B8346CC
:1053A00000F0B58007F0D8FDDBF81430DBF81C20E6
:1053B000DBF80080C01A20F07F4A9BF81830524575
:1053C00094BF00220122FF2B039200F046811FB2FE
:1053D000B14635463B4634E0039B23B9DBF81C302D
:1053E0004B4540F29B80E78BE3786FF30003013776
:1053F000E37094F82830BFB20EF1FF3EE7835FFA06
:105400008EFE002B00F08780A38BBB4280F0838050
:10541000E76884F802E087B16069DBF81430626AFB
:10542000A9EB00001844236901930023009320F0A6
:105430007F404FF6FF730021B847029BFF2B44D0FB
:105440001BB203EB830203EB420308EB8304A26865
:1054500052453AD818F8233094F802E00293637862
:10546000A3EB0E03DBB2012BAAEB020A9144E4D1B9
:10547000A669002EB0D1E7680EF1FF3E84F802E085
:10548000002FDAD0E18B626A60690B4621690191D5
:10549000E17801F001010091DBF81410A9EB0000A4
:1054A000084420F07F400021B847002E4FF0000351
:1054B000E383039B18BF01230393E378002262F385
:1054C0000003E370029BFF2BBAD12E469BF80B30F2
:1054D0009BF80A209A4208D10132D2B2022A1ABF9E
:1054E0001646334600238BF80B600BEB8303002238
:1054F000C3F80C90DBF824408BF81A205B4601229D
:1055000004210320A4460BB0BDE8F04F6047867627
:105510000BB0BDE8F08F84F802E08EE7029BFF2B12
:1055200079D0DDF808C0A38BE18B606805900CEBA7
:105530008C0299420CEB420228BFCB1A08EB820284
:105540002CBF9BB20B4603FB00039068049386427A
:105550000FFA8CF356D3CDE9065E8446DDF814E0ED
:1055600009910593089116E0002D3FD1E178D37899
:1055700001F0010103F00103994233D31378FF2BAB
:105580003CD003EB830203EB420208EB82029068FB
:105590008444664532D39369002BEFD0D38B918B33
:1055A00055688B42E0D2002DE8D0BEF1000FE5D067
:1055B0001F468B42E2D3049B07FB05573F1ABB42B1
:1055C0002CBF00270127E378D17803F001054B4079
:1055D00001F00101A94203F0010303D8002BCDD152
:1055E000002FCBD0DDE9065E099FFDE6BEF1000F7E
:1055F00002D05F1ABFB2DCE77746E4E7DDE9065E7A
:10560000059B0899E7680EF1FF3E84F802E0002F41
:105610003FF417AF37E72E46E5680EF1FF3E84F8FA
:1056200002E0002D3FF452AF2169E38B6069626AAA
:105630000191E178039F01F001010091DBF8141062
:10564000A9EB0000084420F07F403946A847E378E2
:10565000E78367F30003E37038E7B14636E700BF3E
:10566000837E002B40F0CE822DE9F04F467E8FB036
:105670008246002E7AD1837AC27A012141769A42FB
:105680004169099100F0BF820133DBB2022B12BFE6
:105690001A463246334600EB82028372D268099B77
:1056A0000592134423F07F43436101279AF8183091
:1056B0000B9307F051FC9AF80920DAF800300193B7
:1056C000531EDAF804500390DBB2002A00F0E182A6
:1056D000CDE90C6705EBC309FF2304930695CDF8CC
:1056E00008A0D9F804B04FF0000A99F8032099F8FF
:1056F00002800FFA88F101EB810008F1010301EB50
:1057000040044245DBB20BEB84055FD099F80010F2
:10571000994208BF002389F802301BF824006978F9
:10572000042839D901EB810301EB4307019B03EB0B
:10573000870608287278B37822D8D21A12F0FF02AE
:105740002CD106281CD1029BDB7E8B424FD00BF85C
:1057500024A06B6A85F802A0002BC6D0A96A00209D
:10576000984799F8032099F80280C2E7446A042117
:10577000034601220420A4460FB0BDE8F04F604765
:105780000BF824A04FF00103AB706B6A002BACD078
:10579000A96A01209847A8E79846AAE705281DD1DD
:1057A0006B684BB9AB683BB9EB682BB92B691BB97C
:1057B0006B6933F07F43E3D0012A1AD0029B0421A6
:1057C0005C6A01220846A04789F80280069A914542
:1057D000A9F1080300F0DB80994682E7012A00F076
:1057E00098800628EAD1029BDB7E8B42AFD16968A4
:1057F000AFE0DDF808804046FFF762FCB060D8F803
:1058000014C0039B059AA3EB0C0323F07F431344BE
:10581000984240F2B680C01A7368002B53D0AB8A0E
:10582000002B50D0013B9AB2AA827168F38B884258
:1058300024D9CDE907B401F101081BE0726ADFF851
:10584000BCB2AF4C9344A34584BF02F1E87202F5A9
:10585000D432C646346A94BF8E4602F5A572013B27
:10586000A0EB0E00121B9BB288427262F38340F2DF
:105870004981AA8A9A42E1D3DDE907B4934221D251
:105880004A1CCDE9072BD6F820E00A94726ADFF8AB
:105890006CB29B4C72449344A345884607D8A2F14E
:1058A000E872A2F5D432DDF81C80A2F5A5720133AE
:1058B0009BB27262F383AA8A9A424044E6D8DDF82A
:1058C00020B00A9CB2836B680344B360AA68736912
:1058D00013447361039A61463046FFF731FCEA686E
:1058E000B3691344B3612A6993428CBF9B1A0023A6
:1058F000B361AB7D1BB1F27863F30002F270019BE0
:10590000049A03F8272073786A780492013373703D
:105910001DE706283FF417AF029F3846FFF7D0FB7C
:10592000B378B0607370FA7E6B789A427FF40FAFF1
:105930001BF82430062B3FF45AAF029AFF23D3768C
:105940001BF82430062B3FF452AF082B3FF44FAF27
:105950000399029B5A698B1A1E0209D4059A23F0F7
:105960007F4313440299CA699A4288BFCB61EEE62D
:10597000059B521A22F07F4293428CBF9B1A002350
:10598000F0E7726913441B1A7361002044E7DDE9F4
:105990000C67DDF808A09AF81850002F00F0BA80C4
:1059A000039B099ADAF800809B1AFF2D23F07F49A8
:1059B00000F086810027CDE90665AB46059E01977C
:1059C00007E0A37863709AF818B0BBF1FF0F00F0FE
:1059D00092800BEB8B050BEB450508EB8504A36868
:1059E000B34200F2AB80019AA178E08B1A44019295
:1059F0006278521ADAF81C108B42A6EB0306A9EB68
:105A0000030931BFC91A4FF0FF3300218AF81B3058
:105A1000CAF81C10A369D2B20BB1022A14D0002319
:105A2000A36018F825308AF818306168C1B9002AD7
:105A3000C7D0012A01D00028C3D0236A002BC0D0D0
:105A4000616A01209847BCE7002800F0A38000238A
:105A5000A36018F825308AF8183061680029ECD066
:105A6000B4F81EC0BCF1000F50D1B4F81CC06046A1
:105A7000D4E90873CDE90284002201F1010E04E0AB
:105A800001388846441C424411D0DFF870801C4C19
:105A90003B449844A045F3D8A3F1E8730138A3F53B
:105AA000D433F046441CA3F5A5734244EDD1DDE99F
:105AB000028494F828006362002800F0A780099B04
:105AC000A260019AA4F81EC09A18DAF8141022F005
:105AD0007F422046FFF734FB049B08F825306378AB
:105AE000CDF810B00133DBB263709AF818B0BBF197
:105AF000FF0F7FF46EAFDDE9066526E05A2B17FF36
:105B0000592B177FDDE907B4AA8AB7E6A37863703B
:105B10000020ADE704995046FFF736FB9AF818309D
:105B20000B9A93421AD1954218D100238AF8193062
:105B30009AF81A3043BB0FB0BDE8F08F32469B1A7B
:105B4000A360079D069E9AF818B00B9B04995B45CD
:105B50005046E1D0FFF718FB9AF81830FF2B00F001
:105B60009B800B9AFF2A00F08780DAF8002003EB75
:105B7000830103EB410302EB8302D2F80880B8F102
:105B8000000F15D18AF81980DAF824405346012213
:105B90000321EFE5CAF81C308AF81BB0A06018F8A2
:105BA00025308AF81830616800293FF40AAF57E7BA
:105BB00007F0D2F90A270446DAF81430E21A22F084
:105BC0007F42904507F1FF3702F103014AD9414571
:105BD0002CBF5B18434423F07F452846DAF8283071
:105BE000984707F0B9F9031B2D1B23F07F430333BC
:105BF00025F07F45AB4236D90FB10446DCE700DE25
:105C00000446D9E77047374605964FE591457FF63C
:105C100056AF0390481C0290DFF8A8E00398CDF837
:105C2000148005E0884642440130914580B212D983
:105C3000DFF894803B449844F045F3D8DDF80880C1
:105C4000A3F1E8734244A3F5D43301309145A3F5A1
:105C5000A57380B2ECD86044DDF8148063621FFA4B
:105C600080FC2CE7012600238AF819309AF81A30B4
:105C700033433FF460AF87E707F06EF9044607F05F
:105C800047F99AF8183000287FF46FAFCAF814402B
:105C90006BE7FF2304937EE607F04AF904460028E9
:105CA0007FF443AFCAF81C0007F056F98AF8194090
:105CB000CAF814009AF81A30002B3FF43CAF63E79F
:105CC000AB4642E7592B177F5A2B17FFF8B5069FB3
:105CD0009DF81C50089CC8B9154E32605A1E31728E
:105CE00073727760D2B283B107EBC2025460104680
:105CF00012F8083903EB830103EB41018742A5EB5E
:105D0000030304EB8104DDB2F0D10DB10120F8BD35
:105D1000099B33620A9B7362FF240B9BB362347648
:105D200007F01AF975817061F476F5612846F8BDBF
:105D3000100D002040B9064B1A7EFF2A01D11872BF
:105D400070476FF00F0070476FF01500704700BF8D
:105D5000100D002010B40A4B2C2202FB0032546AB2
:105D60005CB100EB800200EB420003EB8003A44631
:105D7000012210BC03210220604710BC704700BF05
:105D8000100D00202DE9F843274E04462C2505FB75
:105D9000046504EB840704EB470406EB84066C6897
:105DA000084604EBC00714F83080FC7897F801E04F
:105DB000BDF8301004F1010C5FFA8CFCE04598BF8F
:105DC0004FF0000CE6452CD0D7F8049004EB840E7D
:105DD00004EB4E0E09EB8E044FF0040809F82E80F8
:105DE0006360089BA3600A9BE3600B9B23610D9B90
:105DF000A3610E9BE3610F9B2362109B6362119B67
:105E0000A36202236270A182A37087F803C0D5E960
:105E100008359847334641460022A847A078BDE898
:105E2000F8830120BDE8F883100D002010B58AB07A
:105E30000C9C00940D9C0294002401940E9C0394ED
:105E4000BDF83C400494109C0594119C0694129C4F
:105E50000794139C0894149C0994FFF793FF0AB0CD
:105E600010BD00BF2DE9F047264DBDF82C709DF800
:105E70003090044608462C2101FB045104EB8406B3
:105E800004EB460405EB84054C6804EBC00614F8EB
:105E90003080F47896F801E004F1010C5FFA8CFC94
:105EA000E04598BF4FF0000CE64528D0D6F80480B6
:105EB00004EB840E04EB4E0E08EB8E044FF0050A43
:105EC00008F82EA06360089BA360099BE3600A9B0F
:105ED00023610D9B63620E9BA36202236270A78203
:105EE00084F81690A37086F803C0D1E90836984765
:105EF0002B4600220421B047A078BDE8F08701209E
:105F0000BDE8F087100D00202DE9F04106461F4D39
:105F100006EB8604084606EB44042C2105EB8407B7
:105F200001FB0654666806EBC00516F8306095F86C
:105F300003E069780EF1010C5FFA8CFC664598BFAE
:105F40004FF0000C61451ED069680EEB8E060EEB1B
:105F5000460E01EB8E064FF0060801F82E807360A6
:105F6000069B7362079BB36202237270B37085F85D
:105F700003C0D4E9083598473B4600220421A847CE
:105F8000B078BDE8F0810120BDE8F081100D00205F
:105F90002DE9F04106461E4D06EB8604084606EB49
:105FA00044042C2105EB840701FB0654666806EBCC
:105FB000C00516F8306095F803E069780EF1010C21
:105FC0005FFA8CFC664598BF4FF0000C61451CD011
:105FD00069680EEB8E060EEB460E01EB8E064FF057
:105FE000070801F82E807362069BB3620223727069
:105FF000B37085F803C0D4E9083598473B460022C2
:106000000421A847B078BDE8F0810120BDE8F08107
:10601000100D002006F0A0BF401A20F07F4070470E
:1060200001481021704700BF8070D000002303702A
:106030000B70704738B5054600200C4603F08CF90C
:1060400010F0060F0ED13DB9074B44B1206818601F
:10605000A2889A80002038BD044B002CF6D11C6029
:106060009C80F7E70C2038BD440D00203C0D00203B
:106070000128034605D8044A0448002B08BF1046EF
:1060800070470020704700BF440D00203C0D0020E9
:1060900001280AD8064A074B002818BF134618687B
:1060A00008609A888A80184670470023184670470F
:1060B0003C0D0020440D002010B5044604F082FD84
:1060C00050B905F09FF960B906F0FEFD70B92046A1
:1060D000BDE8104009F0F4BA00DE05F093F900289D
:1060E000F2D000DE06F0F0FD0028F0D000DE204601
:1060F000BDE8104009F0E4BA0860014809F0E0BAD0
:10610000D83C002009F0DCBA2DE9F0471C4F3B8851
:1061100098422CD913F0FF0527D0DFF868A0DFF8EC
:1061200068809AF89540DFF864909AF894300134CA
:10613000E4B2252C08BF0024A342404615D0FEF748
:10614000A5FD0646484686B1FEF7A0FD88B106606B
:106150009AF895304AF823003B888AF89540013D2B
:10616000013B15F0FF053B80DFD1BDE8F087054618
:10617000D3E730460449BDE8F047FEF79DBD00BFB8
:10618000800D0020003A0020840D0020C80F002060
:106190002DE9F84F324B334FDFF8CC90DFF8C0B029
:1061A000181D062220214FF00008A7F81C80FEF7DA
:1061B00049FD2D4B06220821181DFEF743FD97F8D7
:1061C0001CA07C7F06260134E4B2072C08BF002403
:1061D000A245484613D0FEF759FD0546584675B10D
:1061E000FEF754FD002836D0C5F8048005607B7F9B
:1061F00047F82300013E16F0FF067C77E3D11B4BE6
:106200002522181D4FF49271FEF71CFD184B4822F1
:10621000181D0821FEF716FD1548FEF737FDB0B131
:10622000144A111FFEF77CFD1148FEF72FFD80B1C7
:10623000114A111FFEF774FD104B2422FF201A8013
:10624000FFF762FF04F0CAF80020BDE8F88F00DE17
:10625000E6E700DEECE704492846FEF72DFDCEE731
:10626000CC3A0020903B0020983A0020C80F002034
:10627000840D00207C0D0020740D0020800D002076
:10628000F0B5584E83B0D6E9000101AAFEF756FDDD
:10629000044648B3019D002D00F092802B79013B0C
:1062A0002C2B18D8DFE803F02255171722311731AD
:1062B0003141174B311717171717171717171717DC
:1062C0001717171717171717171717171717222248
:1062D00022172217220000DED6E9000101AAFEF7EC
:1062E0002DFD04460028D5D103B0F0BD3D497068AE
:1062F0000022FEF72BFD3C4A29462046FEF714FDFE
:106300003A4B186809F0DCF9BDE73649706800229D
:10631000FEF71CFD95F8203003F00F03072BEAD1A0
:1063200029462046FAF784F9ADE770682D49002226
:10633000FEF70CFD2946204603F08AF9A3E77068B2
:1063400028490022FEF702FD2946204603F092FD6F
:1063500099E7244970680022FEF7F8FCAF6837B16E
:106360003B78002B39D03B78013BDBB23B702B7B79
:10637000032B34D8DFE803F005272B02284603F06F
:10638000C5FD1B4A00232B73537F117F0133DBB202
:10639000072B08BF002399421DD02C60517F42F883
:1063A00021505377002F3FF46EAF3B78002B7FF4E2
:1063B0006AAFBB68002B3FF466AFF868984762E7A6
:1063C00000DE019D6AE7284602F048FFD9E728462B
:1063D00003F0E0F8D5E700DEE4E700DEC3E700DE27
:1063E000CFE700BF780D0020740D0020D43C0020C2
:1063F000903B002030B5274B274C186087B006F043
:1064000079FD2378002B3ED0244C254D254ACDE93B
:106410000445254C0394254C0294022004230521B5
:106420000D24CDE900241074107613701172002031
:106430001F4AFFF74BFC58BB012200211D480BF0FF
:10644000FEFF04F06FFB08B107B030BDFFF7A0FE00
:106450000028F9D104F0D4FF0028F5D102F0C8FDDE
:106460000028F1D106F076FB0028EDD103F02AFCDC
:106470000028E9D103F088FF0028E5D107B0BDE886
:10648000304006F01BBCFEF771FC01232370BBE714
:1064900000DED1E7D43C0020D68300201DD80000C8
:1064A000BDD800002C3F0020FDD70000F03C0020AC
:1064B0004C3F0020D83C002010B586B003F016FCFD
:1064C00058BB02F0BBFE68BB1C4A1D4B0024A2F85F
:1064D0002041A3F894400122214668460BF0AFFF0B
:1064E000184B224621460320C3F808D0FEF792FC41
:1064F000D0B94FF0FF324FF0FF33684609F01AF978
:10650000FFF746FE90B903F025FFA0B90021012056
:1065100006B0BDE81040FFF78DBD00DE02F08EFE34
:106520000028D1D000DECFE700DEE2E700DE03F096
:1065300011FF0028EAD000DEE8E700BFB03B0020F2
:10654000003A00201402002008B5FFF7B5FF04F060
:106550001FFB00B108BDBDE80840FFF7EBBB00BF63
:106560002DE9F043DFF88C80234D83B00746A8F176
:10657000040900263E606968286801AAFEF7DEFB70
:1065800032462946044668B301980379012B12D09C
:106590002B2B26D16868FEF7D9FB41462046FEF733
:1065A0008BFB012003F08CFE019803F083FE012099
:1065B00003F094FEDDE76868FEF7C8FB414620461D
:1065C000FEF77AFBB9F80030232B0FD801980B495E
:1065D0000133A9F80030FEF76FFB0120FFF794FDAF
:1065E000C7E73860002003B0BDE8F08300DEB9F8EB
:1065F0000030EBE7840D0020700D0020C80F002054
:1066000070B5224982B000234868019301AAFEF7C1
:106610009DFB002835D01E49FEF74EFB01990B79F2
:106620000E2B0FD801229A4045F2210002422AD1B6
:1066300012F4075F0DD10B2B08D1887902F044FECC
:1066400002B070BD272BFBD02D2BF9D000DE02B09D
:1066500070BD91F8203003F00F03072BF0D1CD6807
:10666000002DEDD00A4E25242868ED68013C314606
:10667000E4B2FEF721FB002DE2D0002CF4D100DEC5
:10668000F2E700DEC7E7002BDAD1DFE7700D00206C
:10669000840D00202DE9F843046806461CB3424FE0
:1066A000DFF80881254624682B792D2B18D8DFE8E0
:1066B00003F021171717172121212117174A3B2112
:1066C000441717171717171717171717171717172D
:1066D0001717171717171717172F2F2F17171721F8
:1066E00000DE002CDED100233360BDE8F843FF203C
:1066F000FFF70ABD002B4DD03B88232B4ED801332A
:10670000414628463B80FEF7D7FA002CCAD1EAE77B
:10671000012003F0D5FD284603F0CCFD012003F055
:10672000DDFD002CBED1DEE795F8203033B31A2B07
:1067300010D03E2B0ED0442B33D1A86803F026FB9B
:10674000002CAFD1CFE741462846FEF7B5FA002C22
:10675000A8D1C8E7D5F8089014492846FEF7ACFA46
:10676000484603F07FFBD9F88C001149FEF7A4FAE4
:10677000484603F00BFB002C94D1B4E7D5F8089001
:106780000A492846FEF798FA484603F06BFB002CAE
:1067900088D1A8E700DE3B88232BB0D900DE3B88F8
:1067A000ADE700DEC9E700BF800D0020C80F002064
:1067B000840D00200148FEF769BA00BF840D002057
:1067C0000149FEF779BA00BF840D00200148FEF7A9
:1067D0005DBA00BFC80F00200149FEF76DBA00BFC7
:1067E000C80F0020014AFEF79FBA00BF740D0020B9
:1067F000014B186808F064BFD43C002008B5044A77
:10680000FEF792FA034B1868BDE8084008F058BF3D
:10681000740D0020D43C0020022810B50C4602D094
:106820000B68022B07D004484FF0FF324FF0FF33C4
:1068300008F080FF206810BDD83C0020014B18688C
:10684000704700BF6C0D002030B505682B7887B00D
:10685000EBB104460122002168460BF0F0FD0D4B20
:10686000C5F80CD0AB602B788BB10B4B00221146D6
:1068700003209C60FEF7CEFA38B94FF400420023A3
:10688000684608F057FF07B030BD00DEF5E76FF04F
:106890007700F8E70561000004020020F0B5254EFE
:1068A000336885B00C461746002B36D0994215D177
:1068B0000223039303AB0246009303211E4B0020E7
:1068C000FFF766FB022805460CD0039B022B09D17B
:1068D00095B133680BB19C4221D014B36FF02D00F9
:1068E00005B0F0BD15484FF0FF324FF0FF3308F010
:1068F00021FF039D002DECD13846FFF7A5FF33683B
:106900000BB19C4211D0002CE8D10028E8D010F146
:10691000780F08BF002005B0F0BD3160C8E7002344
:1069200033606FF0770005B0F0BD35600028D7D038
:10693000EDE700BF6C0D0020F9600000D83C00209E
:106940000C4991F8942091F895309A420AD8A3EB1B
:10695000020C5FFA8CFC604509D89A4207D051F8C6
:106960002200704725339B1ADBB29842F7D90020EA
:10697000704700BF003A0020094A92F8941092F83C
:1069800095308B4209D04B1CDBB2252B08BF00236E
:1069900052F8210082F8943070470020704700BF01
:1069A000003A0020014AFEF7BFB900BF7C0D00206D
:1069B0000122024B11460020FEF72CBAF401002000
:1069C00010B5054AFEF7B0F90122BDE81040034BAF
:1069D00011460020FEF71EBA7C0D0020F4010020B5
:1069E0002DE9F0431A4D9DF81C8095F821C10CF15A
:1069F000010E5FFA8EFEBEF1090F994695F820311F
:106A000008BF4FF0000E73451DD0144605EB4C1C1B
:106A1000E36807460E4610685168926864460FC4E2
:106A20009CF81C30CCF8186008F0010823F0030330
:106A300043EA0803CCE904978CF81C3085F821E17F
:106A40006046BDE8F0834FF0000C6046BDE8F0837F
:106A5000B03B0020054890F8203190F821219A425F
:106A600014BF00EB43100020704700BFB03B002074
:106A700001460B480A7890F82131082A84BF90F823
:106A800020210A70934208D0531CDBB2092B08BFA7
:106A9000002300EB42100B7070470020704700BFCE
:106AA000B03B00202DE9F04F3D4E96F8201196F8AE
:106AB000213187B08B42039047D04FF0000906EB9D
:106AC00041110B24CDF81090CA46CB46CDF8089062
:106AD000CDF814900D7FD1F80080CF68C5F3400247
:106AE00005F00105002C4FD0013CE4B282B396F8CA
:106AF000211196F82031994227D00133DBB2092BBE
:106B000008BF0023994286F820311ED006EB4311BE
:106B10005B01C868002ADDD135BBBBF1000F37D05F
:106B2000BAF1000F029A08BF4246029208BFBA4665
:106B30000A7F9507CED4D2071DD48345F3582BD0B6
:106B40008245C7D1029A9A42C4D107B0BDE8F08FFE
:106B5000144B0398996011460192FEF75BF9019A74
:106B60000028C4D000DEC2E7049A7AB1B9F1000F60
:106B700008BFB946DCE7BAF1000FABD1049B8342F2
:106B8000E3D04845A6D1E0E700DEADE70497CFE7C4
:106B9000BB46CDF81480CBE7059A9A42D0D1D4E712
:106BA000B03B0020E4010020054B1A7F597F914241
:106BB00004D053F8220010B10C3070470020704709
:106BC000903B0020074A117F92F81DC08C45034678
:106BD00006D052F821201AB102F10C00137370474D
:106BE00000207047903B002070B5114A117F537F01
:106BF0008B421BD04B1CDBB252F82140072B08BF45
:106C00000023137794B10223054600262068094A21
:106C1000237121462660A560FEF786F80122064B07
:106C200011463046FEF7F6F8204670BD0024FBE71B
:106C3000903B00207C0D0020F401002010B582B0B4
:106C4000049B9C7A6FF341049C720024CDE90044BC
:106C500004F0BEF802B010BD10B50346007F1A69FB
:106C60009969012482B02040CDE90004586904F0FC
:106C7000AFF808B902B010BD7730FBD000DEF9E7FD
:106C80000B8A002B33D030B5054683B001F10C00E0
:106C90000C460AF073FB012826D1002301A92046E7
:106CA000019301F05FF80146C0B1C36828691A7802
:106CB000042A05D003682846984720B103B030BDA8
:106CC0005B78052BF6D1019D45B1284602F08CF882
:106CD0000346019907486B710BF09CFB2046FCF7BB
:106CE000ABF8002003B030BD6FF01500E6E76FF0A1
:106CF000150070472C40002010B50469FFF724FCF4
:106D000040B90548FBF70AFD0448FBF707FD0020E2
:106D1000206010BD00DEF4E720060020D806002029
:106D20002DE9F0432E4FD0F8108083B006464FF087
:106D300000094FF0FF324FF0FF33384608F08EFC69
:106D40000028F6D090F9053001905A1E032A2FD85A
:106D5000022B35D04FF0FF324FF0FF330220FCF70B
:106D6000D9F804460198002C34D0214601F064FB88
:106D7000019B01A8C3F80090FFF78CFC20460AF0A5
:106D800095FA0546214600200AF0B0FA2B8A012B1D
:106D900004462946304607D9D8F80030984709F00C
:106DA000CDF8002CEAD1C4E72846FCF745F8F6E711
:106DB00000DE019B01A8C3F80090FFF76BFCB8E769
:106DC0000022002301210020FCF7BCF804460198B2
:106DD000002CCAD1046001A8FFF75CFCA9E700BF42
:106DE0002C40002070B5114E114D82B00DF1020102
:106DF00001A8FFF7B5FB0028F8D1019B6BB1FFF7A5
:106E0000FFFB019C204601F0EFFF019960712846CD
:106E10000BF000FB019B002BE8D14FF0FF324FF04D
:106E2000FF33304608F086FCE0E700BF4440002016
:106E30002C400020F0B50546076989B00E461F4872
:106E40000BF0A9FA4FF0FF3200211D480BF0F7FAC2
:106E50001B48FFF7CFFA044660BB3E6001F0E4FF39
:106E6000002600276FF00903CDE90334CDE906675A
:106E7000CDE90144134B144900954FF4E0721348D7
:106E800008F04CFE1249114808F0C2FD6FF00702ED
:106E9000CDE90324CDE90667CDE901440D4B0E4948
:106EA00000954FF460720D4808F038FE0C490B480D
:106EB00008F0AEFD204609B0F0BD00BF2C40002018
:106EC00044400020E56D0000408D00202006002099
:106ED000602E0100216D0000408F0020D8060020A8
:106EE000702E010010B508F0D9FF054C20460BF0BC
:106EF0005EFA20460BF04FFABDE8104008F0E2BF02
:106F00002C400020038800B5C3F3441303EB430C6B
:106F10008444B2FA82F29CF802E05209013362F32F
:106F2000000E03EB43038CF802E0F1B10A88C25271
:106F30000278D30612D1531C03F01F0363F304023B
:106F40000270028863F3491202F47873202B0280E6
:106F500004BF6FF3491202805DF804FB0388C3F39A
:106F60004413013303F01F03EBE7C152E0E700BF16
:106F70002DE9F04FDFF8B09183B0D9F800609DF8AB
:106F800034400194002E5CDB07460D4614469846BB
:106F90005FD0DFF898A14FF0000B05E00BF1010B7B
:106FA0005E450AF1260A54D05146062220460BF0CF
:106FB0007BFC0028F2D11AF8013CAB42EED15C4CCC
:106FC000262303FB0BF3E518E97921FA07F2D6072C
:106FD00078D5072F39D108EB480203EB420222444F
:106FE0004FEA4807117AC90602F1080600F08380CB
:106FF0000C9951B34978157B4FEA111CBCEB151F56
:1070000040F088802D020B0205F470610C9D92F80F
:107010000BC02D7803F470632B4341EA0C019942B5
:107020005ED1B378DB0710D4019B53B926234744C4
:1070300003FB0BF303EB470323449A7A42F001026C
:107040009A72002003B0BDE8F08F012003B0BDE8C4
:10705000F08FDFF8E0B03648DBF800A0D4F800C0CD
:10706000019A262303FB0AF3591C40F801C001448E
:10707000A4888C80C4180121C554B9400833E1713B
:10708000C15A2D4C2140C1520625191815FB083351
:107090001844CB882340CB808B8923408B814B8A3B
:1070A00023404B820C99FFF72DFF0F2ED6BF731C88
:1070B0000AF10103C9F80030102B08BF0023CBF8F8
:1070C0000030BEE7062000FB08300123BB4008303B
:1070D0000B43019A0C99EB712044FFF713FFB0E7C3
:1070E0000C9BD5725B781373019B73B9B37843F033
:1070F0000103B370A5E7062000FB08300830019AB1
:107100000C992044FFF7FEFE9BE7B37860F3000381
:10711000B37096E7062202FB08330833019A0C99F4
:10712000E018FFF7EFFE8CE760400020654000208C
:10713000644000205C40002000FCFFFF2DE9F04F80
:1071400087B09146199E9DF844200492129A0592A8
:107150000C369DF94C20039304469DF95030029261
:107160003046189A01930D46022100929DF85C70FA
:10717000DDF84080BDF854B0DDF858A00AF0C6F83C
:107180003E21017007F11A014170012130460AF0D9
:10719000BDF8014630460D260E7007F11901C9B23F
:1071A0000AF0B4F80121DDE90132A0F801400170D4
:1071B000B8F1000F35D00399C170D8F800104160C4
:1071C000B8F80410018195FAA5F5B5FA85F50135F1
:1071D00080F80B908572BAF1000F29D09AF801104F
:1071E000090914F00404837301734273A0F80FB00B
:1071F00000F1120310D0049A059942740A68C0F88D
:1072000012208A889A80009907763A46193007B08A
:10721000BDE8F04F0BF032BB4474C0F812409C80C4
:10722000F1E780F80380C0F80480A0F80880CAE77E
:10723000FF21D6E72DE9F04F4D4D04460B4695E86A
:10724000030085B00290ADF80C10080C49498DF888
:107250000E004968880077D547490968C90473D585
:107260001E7E464B1B7876421546A71C76B2002B35
:107270005CD1237803F00F03012B71D094F801A0A7
:10728000AAF106080AF1140B5FFA88F80AF1130A4A
:107290005FFA8BFB5FFA8AFAC1460C350221284659
:1072A0000AF034F83E23037080F801B0012128462B
:1072B0000AF02CF803460D221A70514628460AF0AF
:1072C00025F8034601201870217801F00F0101F123
:1072D00010020DEB020111F8082CA3F8012022780E
:1072E000C2F38012DA70D4F802205A60FF21BA8803
:1072F00019737F211A8159730022214658819E7388
:10730000DA731A7411F8080B00F00F05012D1ED066
:107310005A74C3F81220DA824A4603F1190083F83E
:10732000188005B0BDE8F04F0BF0A8BA0022CDE9F7
:10733000002220781346C0F380113A4600F00F0077
:10734000FFF716FE002894D005B0BDE8F08FC0F31B
:10735000C0105874A268C3F812208A88DA82DBE76A
:107360004FF000094FF0190A4FF01A0BC84694E786
:10737000902E0100F0000020E8000020D7830020BC
:107380002DE9F04F93B09046119341F02003259DD5
:107390000B939DF878300C939DF984300D939DF8F4
:1073A0007090BDF88830BDF890B0269E289F95F863
:1073B00000C00E930246119B10921B780F93209BE6
:1073C0006446E52C93F900A028BFE524239B06938F
:1073D0000E9B05930D9B0794CDE903A31F9B02937E
:1073E0000C9B01931D9B00933B68099333680F9A94
:1073F0000B98089341464B46FFF7A0FE33682344A1
:1074000033602B781B1B2B7002204FF4A02200232B
:10741000FBF780FDABEB040B1FFA8BFB01463860DA
:10742000002858D0279809F050FF95F800C0BCF10B
:10743000E50FCBD8109AD2686146002A45D0E345C3
:1074400046D9BCF1000F64D1209B7F21197092F8BE
:1074500022108C0659D092F82310C8074CBF02F1B5
:107460002A0002F124008B0748BF06300C0748BFF2
:107470000230CB0607D58178119B4909013119707B
:1074800092F8231003308C0648BF12304B0603D508
:10749000209B10F9011B197092F82210C1F305010D
:1074A0000131CCB202F12201411AC9B2A14203D288
:1074B000611A50FA81F0214692F821408C420DD891
:1074C0004FF0000300212B708C468B453FF673AFC5
:1074D00013B0BDE8F08F00DE3968A3E7306092F8A2
:1074E00021C0ACEB010C5FFA8CFCDC45614684BF2B
:1074F00059465FFA8BFC594585F800C0FFF45BAF35
:10750000BCF1E50F3FF657AFE2E702F1230001219E
:10751000D2E7119B109293F800A0209BCDF83CA0DD
:1075200093F90040A2466446239B06930E9B059365
:107530000D9B0794CDE903A31F9B02930C9B019322
:107540001D9B00933B68099333680F9A0B9808932F
:1075500041464B46FFF7F2FD3368234433602B78F6
:107560001B1B2B7002204FF4A0220023FBF7D2FC40
:10757000ABEB040B1FFA8BFB0146386038B1279840
:1075800009F0A3FE2B78E52BCED8109A5CE700DE3D
:107590003968F4E72DE9F04F9A46B3B07B4B2A9255
:1075A0005A68CE684FF000097F239200CDE92E99EA
:1075B000CDE922998DF8B4908DF8B5908DF8B690FC
:1075C0008DF8B7908DF8B2308DF8B330CDF880904B
:1075D000CDF8849040F175826D4B1B68DB0440F15F
:1075E0007082CDE9139935468C46CDF86090CDF880
:1075F0009090CDF87090CDF89C90CDF8A490CDF8F7
:107600006C90CDF87C90CDF84890CDF87490CB4636
:10761000CDF85490CDF87890CDF89890CDF8A09012
:107620001A96CDF894908846CDF8ACA082789CF854
:1076300018309CF819E0199312F03F044FEA9213A6
:107640000EF00101169300F07C8190F803A01AF06F
:10765000010400F1040300F07E81E04500F0E781C1
:107660001A9CA44500F0E381002310931C461AF0F5
:10767000020600F10A0300F07381E04500F0CC81BE
:107680001A9EB44500F0C881002111910E460633C0
:107690001AF0040F18BF01331AF0080116BF179330
:1076A000179102331AF010010F910FD01A998C45DF
:1076B00000F0C281E04500F0C98199785F294FEA66
:1076C000511700F2C681791C0F9103331AF0200F75
:1076D00002D059881D9112331AF0400F18BF13F9C8
:1076E00001ABC2F3050200F1020102F10102A3EBBA
:1076F0000101D2B2C9B208BF4FF07F0A914205D84A
:10770000571A17F0FF071CBFDB1911464278914248
:1077100040D2521A1498D2B2114601441F2940DCBB
:10772000E04500F01F811EF0080F0DD01B990F9847
:10773000CDF894A0002818BF01462191012118938B
:107740002092CDF8A0C02491BBF1000F129908BF80
:1077500021461291109908BF8B46B9F1000F139979
:1077600008BF31461391119908BF8946189900291D
:1077700000F04A81159B13449BB21593002D00F035
:107780000C8105F12000AC46ED684FE7F0000020C9
:10779000E800002000231498194601441F291A46C6
:1077A000BEDD249B1A9EDDF8ACA04746D846CB46EA
:1077B000DDF894904BB1189B2E93209B8DF8B4303C
:1077C000219B8DF8B2908DF8B530279B3BB1239B60
:1077D0008DF8B3301C9B2F93229B8DF8B630299BDC
:1077E00013B11B9B8DF8B7302E9B002B00F0D0817E
:1077F0004FF00209B8F1000F00F0D0810024924B45
:107800001B78002B40F099816401E5B2BBF1000FB9
:1078100003D01F9B43F004031F93199B149A5C42EF
:107820002A9B30939DF8B630934264B2C0F06081D9
:10783000E52B00F25D812A9A07931E9B06931D9B00
:107840001F990992CDE90443139B9DF8B720CDF809
:1078500008B0CDE9008329432F9B08930D469DF97D
:10786000B33003935146129B2846FFF767FC2E9EC8
:10787000002E00F07E8102204FF4A0220023FBF7AF
:1078800049FB05F09F0545F00805064630900028A5
:1078900000F094812A98314609F017FD9DF8B43024
:1078A000159A934201D3E52B22D92A9B0B93159B62
:1078B00008931E9B07931D9B2898CDF80CB0CDE92B
:1078C0000543139BCDE90183129B009330AB0C93CE
:1078D0002EAB0A932DAB09930DF1B20304935246DC
:1078E0000DF1B5032946FFF74BFD9DF8B430309EEE
:1078F00007931E9B06931D9B2E9A0892CDE9044385
:10790000139B9DF9B2200392CDE900839DF8B52029
:10791000129B0996CDF808B045EA49105146FFF789
:107920000DFCFC6854B131AD002631942346E46867
:107930001E602846FEF7AEFE002CF6D133B0BDE83F
:10794000F08FCDE91044C31C0F94264601211794F3
:107950004FF07F0ADAE61AF0020610947FF48DAE3B
:10796000119695E6169B1F93179B0F991E93012264
:107970000023CDE91433DDF840B0DDF84490CDF8B4
:107980008CA0129413961C9327921B91CDF898808B
:1079900022932992002D7FF4F4AE249B0F9A1A9E15
:1079A000DDF8ACA04746D846CB46DDF89490002BD6
:1079B00000F09880209B8DF8B430219B8DF8B53075
:1079C000189B2E93279B8DF8B2903BB1239B8DF88B
:1079D000B3301C9B2F93229B8DF8B630299B13B19B
:1079E0001B9B8DF8B730131E18BF01234FEA4309C4
:1079F000189B002B7FF4FEAEB8F1000F00F0D08092
:107A00004C464FF00009FAE61C9900294DD0149B12
:107A100013449BB21493B1E600294FD1D8F8081053
:107A20001193096891F83A60C6F381062FE604784D
:107A30001093C4F380141AE6910900293FF43AAE7A
:107A400000210F9141E600BFD7830020002D7FF475
:107A500034AEDDE924391A9E4BB1189B2E93209B3E
:107A60008DF8B430219B8DF8B2908DF8B530279BFE
:107A70003BB1239B8DF8B3301C9B2F93229B8DF839
:107A8000B630299B13B11B9B8DF8B730002E3FF405
:107A900055AF31AD002431963346F6681C60284658
:107AA000FEF7F8FD002EF6D148E71C930123CDE93F
:107AB000222ACDF898C0149227935FE61193FE26F0
:107AC000E5E5002E3FF43AAF31AD00243196334660
:107AD000F6681C602846FEF7DDFD002EF6D133B0B7
:107AE000BDE8F08F279B002B7DD0249B18936DE77A
:107AF000149B08932A9B0B931E9B07931D9B269810
:107B00001F99CDF80CB0CDE90543139BCDE9018356
:107B1000129B009330AB0C932FAB0A930DF1B6037D
:107B200009930DF1B303049352460DF1B703FFF728
:107B300027FC9DF8B630309A7EE61E9B0093129982
:107B40001F9B019442460720FFF712FA00283FF4DA
:107B50005BAEFC68002C3FF4F1AE31AD00263194F1
:107B60002346E4681E602846FEF794FD002CF6D1FB
:107B7000E4E6FC68002C3FF4E1AE31AD31942346DD
:107B8000E4681E602846FEF785FD002CF6D1D5E698
:107B9000B8F1000F07D09946022430E6454635E695
:107BA000B9F1000F2AD01E9B73B19DF9B3307F2B22
:107BB00007D04FF000094025C84627E600DE309E7A
:107BC00068E62F9B002BF4D1002E3FF4B7AE31AD09
:107BD000002431963346F6681C602846FEF75AFDAD
:107BE000002EF6D1AAE6299B13B11B9B8DF8B73066
:107BF000131E18BF01234FEA4309FDE64D4605E673
:107C0000F0B5013887B01446092806D8DFE800F03F
:107C100009283E050550056281946FF0150007B0F4
:107C2000F0BD4E4B0D21188809F045FC0D21206058
:107C30000C3009F06BFB4FF4806200234FF002140C
:107C40000321A0F8052063220370C0F80140C17130
:107C5000037242728372C3720373002007B0F0BDD7
:107C60003E4B4121188809F026FC412120600C3050
:107C700009F04CFB002104463E2200F8031B0AF0E9
:107C80000BFE40F2A733A4F80130E6E7334B09219D
:107C9000188809F010FC092120600C3009F036FB2F
:107CA0000346002203F8012BC0F801205A60D4E7F4
:107CB000C9680020FEF7BEF9284B0121188809F099
:107CC000FAFB012105460C3009F020FB002303706C
:107CD0002560C2E7224E214F0FCE01AD0FC533689C
:107CE00038882B80132109F0E6FB132120600C302B
:107CF00009F00CFB0446002301AE04F8013B844666
:107D00000FCE2D88CCF801006160A260E36025826F
:107D1000A3E7124B1821188809F0CDFB1821206029
:107D20000C3009F0F3FA00230446012100F8023B6D
:107D300005F066F8607090E7084B2121188809F07B
:107D4000BAFB212120600C3009F0E0FA0146002343
:107D500001F8113B013005F0A3F87EE7F075002033
:107D6000982E01002DE9F041038A8AB00027022BEA
:107D700005973AD904460E460C30032109F0F6FA6D
:107D8000228A83789A4230D30288DFF85883C2F37C
:107D90008523082B90B2A8F80020C2F3090540D033
:107DA00011D8032B26D0042B19D16A1E082A16D805
:107DB000DFE812F030011101FF0015001500150079
:107DC00015001500F0003F2B09D105AA21462846D1
:107DD000FFF716FF163040F0CA82B8F80000012104
:107DE0000AB0BDE8F04109F078BB002420460AB093
:107DF000BDE8F081032D00F09882632D07D0012D9E
:107E0000EDD1E268B84B1168526819605A600121DF
:107E100009F051FB012104460C3009F077FA077094
:107E2000E4E76A1E582ADAD801A353F822F000BF0B
:107E30003982000019820000D1810000DF7D00003E
:107E4000C7810000DF7D0000DF7D0000DF7D0000D6
:107E5000DF7D0000DF7D00003D8000003D800000F0
:107E6000DF7D0000DF7D0000DF7D0000DF7D0000A2
:107E7000DF7D0000DF7D0000DF7D0000DF7D000092
:107E8000DF7D0000DF7D00008B8100006D81000040
:107E9000DF7D0000DF7D0000DF7D00000F8300003C
:107EA000DF7D0000DF7D0000DF7D0000DF7D000062
:107EB000DF7D0000DF7D0000DF7D0000DF7D000052
:107EC000DF7D0000DF7D0000DF7D0000DF7D000042
:107ED000DF7D0000DF7D0000DF7D0000DF7D000032
:107EE000DF7D0000DF7D0000DF7D0000DF7D000022
:107EF000DF7D0000DF7D0000DF7D0000DF7D000012
:107F0000DF7D0000DF7D0000DF7D0000DF7D000001
:107F1000DF7D0000DF7D0000DF7D0000DF7D0000F1
:107F2000DF7D0000DF7D0000DF7D0000DF7D0000E1
:107F3000EB820000A7820000DF7D0000818200004C
:107F4000798200006F820000658200005B82000081
:107F5000C7800000A980000089800000DF7D00004C
:107F6000DF7D0000DF7D0000DF7D0000DF7D0000A1
:107F7000DF7D0000DF7D000053800000DF7D00001A
:107F8000DF7D0000DF7D0000DF7D0000F980000064
:107F90003D810000072109F08EFA072104460C30CC
:107FA00009F0B4F90146002001F8010BFEF770F862
:107FB0001CE7092109F07FFA092104460C3009F079
:107FC000A5F90346002203F8012B6021C0F8012027
:107FD0005A6041710AE7412109F06DFA41210446D6
:107FE0000C3009F093F900210546402200F8011BEE
:107FF0000AF052FC04233D493D4AEB72C020EB7568
:108000004FF40A73A871C5F81A10C5F82620A5F810
:108010000F30EBE6092109F04EFA092104460C3035
:1080200009F074F94FF450610023324A01800D21A8
:108030008370C3700171C0F80520D7E6012109F0F3
:108040003AFA012104460C3009F060F90C23037060
:10805000CCE6E068841D06880379C27881780194B3
:1080600040790090B0B202F05DF803210546B8F8FF
:10807000000009F020FA032104460C3009F046F90B
:108080000570A0F80160B1E6032109F014FA03219C
:1080900004460C3009F03AF90146002301F8023B8E
:1080A0000130FDF7C3FFA1E6022109F004FA022125
:1080B00004460C3009F02AF900230370054602F04B
:1080C00049FA687092E602F047FA0546B8F80000EF
:1080D000012109F0F0F9012104460C3009F016F9EC
:1080E000057083E6F0750020F0000020170CC00832
:1080F00060FF80305900FFFF0DF113030DF11102F5
:1081000006A90DF1120002F059F90521B8F8000096
:1081100009F0D1F9052104460C3009F0F7F89DF873
:1081200012209DF813309DF811100371C170427038
:108130009DF8182082700023037057E6E468A17848
:10814000208801F0A9FD05460028BFD1A278B24BD6
:1081500092071B7840F13281B04A13B113680133A2
:10816000B4D1AF49002313600B60AFE7092109F0D8
:10817000A2F9092104460C3009F0C8F8002300F8E0
:10818000013B082102F014FD30E6E068002306AA56
:1081900000F1100105F0E4FB1121B8F8000009F02E
:1081A0008AF9112104460C3009F0B0F80646002384
:1081B00006F8013B06AD07460FCDC7F80100716018
:1081C000B260F36012E6E1680120FDF733FF7CE75F
:1081D000092109F070F9092104460C3009F096F8DC
:1081E0000346002503F8015BC0F801505D600646B8
:1081F000FDF716FF2B4661F30703C1F3072262F375
:108200000F23090C61F31743090A61F31F63C6F8D2
:108210000100C6F80530E9E5042109F04CF9042114
:1082200004460C3009F072F800231B21032203706E
:1082300041708370C270D9E5E2687A4B11681960A9
:1082400052685A60012109F036F9012104460C30C8
:1082500009F05CF800230370C8E5E068C17902F01A
:10826000EDF932E7E068C17902F0A6F92DE7E3689D
:10827000188801F005FD28E7304601F09FFC24E74F
:10828000E368654A197812784C0779D5002A40F0DE
:108290008F80624A624D002414602C605C7B1F2C2E
:1082A00075D90C219CE5E1680878002861D04B78ED
:1082B000002B5ED0594B1A68551C00F08780564D34
:1082C0002C78002C00F08A8000221A60544B1A602F
:1082D0008A88498800F0F8FE0C2805464FF0010115
:1082E000B8F8000008BF0025F3E6E468A278237818
:1082F000657812F0010240D0E078A188E28800F0B1
:10830000010040F002000095F8F7B6F8DDE609211B
:1083100009F0D1F8092104460C3008F0F7FF0023DA
:10832000414A02604360037260E53C493F4B3A4A70
:108330004FF0FF3008604FF0FF3041F6FF71C3E9A6
:108340000001384B17701F200021C3E90001FEF720
:10835000B3F8B8F80000012109F0ADF80121044696
:108360000C3008F0D3FF0770FEF7BCFD3EE5059C1E
:108370003CE5294B00221A70AAE702201146C2E709
:10838000002A8BD1254A4FF0FF34146086E79A7893
:10839000084659780294B3F80B400194B3F80940A9
:1083A0000094033301F048FB0146B8F8000017E5DC
:1083B0001A4A146801347FF471AF6BE7002B7FF425
:1083C00085AE164B4FF0FF321A607FE60022124C4A
:1083D000134D1A6001232A60237079E70123002AD4
:1083E0002B707FF775AF124B262000FB0235114A28
:1083F000188803F8014C10401880D8881040D880A5
:10840000988910409881588A1040588226339D429E
:10841000EED108785CE700BFD783002060400020E1
:108420005C400020E800002000303300F000002015
:108430006C40002000FCFFFF0379032B00D1704744
:108440002DE9F04F053B8DB004460D4600F12006A6
:10845000222B24D8DFE813F027009600E902A900B8
:1084600023002300BC00DB007201CA0223002300AA
:1084700023002300230023002300230023002300E4
:1084800023002300230023002300230023002300D4
:10849000230023002300230023002300FC0200DE2E
:1084A0000DB0BDE8F08F9E4B9E4A93E803005368E1
:1084B000ADF82C100A0C217E8DF82E2003F000520E
:1084C0004B425EB2637E0A9013F0010340F0978343
:1084D000002AE5D0944A12689707E1D5934A1278AA
:1084E00004F12208002A40F01B8494F8203003F0A5
:1084F0000F03012B00F0248494F82130A3F1060926
:1085000003F1060B5FFA89F905335FFA8BFB5FFA1B
:1085100083FA4F460C350221284608F0F7FE3E2329
:10852000037080F801B00121284608F0EFFE0346F1
:1085300002221A705146284608F0E8FE0123037013
:1085400094F8203003F00F0330336B4404F128011A
:1085500013F8083C437094F82030C3F38013837001
:10856000D4F82230C0F80330B8F80430A0F807304F
:1085700000F10A0380F809903A4618460AF07EF99D
:10858000C6558DE790F8203003F00F03072B04D178
:1085900090F82130002B40F096832A462146304641
:1085A0000DB0BDE8F04FFEF745BE90F8203003F067
:1085B0000F03072BF1D190F82130002BEDD00423CD
:1085C0002A46214630460DB0BDE8F04FFEF7E2BF27
:1085D000544B5B6898007FF563AF534B1B68D9031E
:1085E0007FF55EAF0C350221284608F08FFE4FF470
:1085F0009F7303800121284608F088FE1123037031
:10860000002128460DB0BDE8F04F08F07FBE454B75
:108610005B689A007FF544AF434B1B689B047FF572
:108620003FAF0C350221284608F070FE41F23E03B0
:1086300003800121284608F069FE0E2303700F21F4
:10864000284608F063FEF707054600F1B18394F869
:1086500020302B70442B3FF423AF354BA768D3F861
:1086600000B097F88A9097F88B10BBF1000F07F1D4
:10867000840A09F0010925DD2E4E03914FF0000810
:108680003146062250460AF00FF9002840F0898250
:1086900016F8013C4B4540F08482274A0399034673
:1086A000262000FB082202F1200092F82060F60646
:1086B00008D092F82420B1EB121F03D1827863F323
:1086C00000028270E388A5F8013097F88A30C3F37E
:1086D00000022A7197F88A2003F00103910744BF32
:1086E00002332B71D7F88430C5F80530BAF804305E
:1086F000A5F8093097F88B30EB7094F8212092FAA6
:10870000A2F3002AB3FA83F308BF4FF0FF3301331B
:10871000EB72638CAB8194F82430AB73C0E600BF7E
:10872000202D0100F0000020E8000020D783002069
:10873000604000206540002064400020C24B5B6820
:108740009A007FF5ADAEDFF804A3DAE9003803F450
:1087500080465B0440F12D8283681A68B2F87C3051
:108760009BB2002B3FF49CAE837E818B04919F07CC
:1087700000F1B882049B1F2B00F2B48294F82210FF
:10878000237E059311F03F0700F08B8294F823308D
:10879000D8074CBF04F12A0904F124099F0748BFF8
:1087A00009F1060958074ABF19F8010BFF20800993
:1087B000039013F008001CBF484609F1020913F0AA
:1087C000100B07D099F802705F2F3FF669AECB46C9
:1087D00009F103099F0648BF09F112095F064CBF62
:1087E00019F9013B7F230693C1F3050304F122012C
:1087F0000133A9EB0101DBB2C9B2994200F2A882B0
:108800005F1A17F0FF07099700F0C482CDF81C909B
:108810001946B94494F821308B4200F251824FF04E
:1088200000094F4692F88A1001F00403002800F076
:108830009D82002B00F0B381637E5B0640F1AF8127
:108840000B0700F19C81002E00F0A981059B069A80
:108850000499CDF818B05B428F4238BF7F225BB2DB
:1088600005932946934601F10C063046022108F093
:108870004DFDF72FB8464FF03E0328BF4FF0F708E5
:10888000037008F1080343700121304608F03EFDF3
:1088900003460F2208F107011A703046C9B208F0EA
:1088A00035FDE3880380059BC370039B80F802B00D
:1088B000037180F806800646494642460730A7EB1A
:1088C000080709F0DBFF17F0FF0740F08281DDF8B1
:1088D00018B0BBF1000F00F0F88194F91930DAF804
:1088E0000480002BC0F2F681022373714FF0000B5D
:1088F00018F0020F3FF4D4AD079B002B3FF4D0AD2E
:10890000099A222A7FF6CCAD1A465B782C2B7FF48D
:10891000C7AD537F16783F2B3FF6C2ADBBF1000FBA
:1089200000F052820BF10C0B0221584608F0EEFCCD
:1089300041F23E4303800121584608F0E7FC03461C
:1089400022221A701321584608F0E0FC079FE388A2
:108950000380052205460321B818FCF787FBBC1DE0
:10896000A870052200212046FCF780FB0C22E8704D
:108970000721F81CFCF77AFB0322A880052120467A
:10898000FCF774FB04221146A87107F10900FCF7FB
:108990006DFB04221146E87107F10C00FCF766FB41
:1089A00028727B7BA5F809301422002107F11300FF
:1089B000FCF75CFB030CC0F30722E8722A736B73AD
:1089C0000C22042107F11500FCF750FBE8817B7FA6
:1089D0005B0901332B7497F822303A2E4FEAD313F8
:1089E0006B740CBF01230023AB7459E5164B5B6815
:1089F00098007FF555AD154B1B6819047FF550ADF8
:108A00000C350221284608F081FC40F23E330380F9
:108A10000121284608F07AFC102303700221284621
:108A200008F074FCE38803803AE590F8203003F006
:108A30000F03072B7FF4B1AD90F82130002B3FF4EA
:108A4000ACAD0223BCE500BFF0000020E800002030
:108A5000CD4B5B689A007FF523ADCC4B1B68DB02E6
:108A60007FF51EAD806850F8407B01F0E3FB0646C1
:108A700000287FF415ADB7F87C309BB2002B3FF493
:108A80000FAD384601F074F994F82330E78CFF2BD2
:108A9000814600F0828194F82060012E38BF0126C3
:108AA00006F106084FEA48085FFA88F808F1010A5B
:108AB0005FFA8AFA0C350221284608F027FC3E238B
:108AC000037080F801A00121284608F01FFC03462E
:108AD00015221A704146284608F018FC237EA0F89B
:108AE0000090C3EB4331C3EB81035B00A0F803307C
:108AF00094F82430437194F82130C3F381118171CB
:108B000094F8251081709B090246A0F8097040F086
:108B1000368194F82230D37194F823301372FF2BEE
:108B20002BD094F82030002B00F03C812EB311465E
:108B300004EB8605B4F9283013F5004F00F04181AD
:108B40009B1003F1800080B2FF2800F23A815BB2F3
:108B50000B73B4F92A3013F5004F00F02F819B10EE
:108B600003F1800080B2FF2800F228815BB2043458
:108B7000A5424B7301F10201DCD1D67290E4BBF146
:108B8000000318BF012300900193843201F001011A
:108B900004230720FEF7ECF900283FF454AEAB465F
:108BA000A6E608F10108C34506F126067FF468AD84
:108BB00088E508F0020333433FF472AC83681A6817
:108BC000B2F87C309BB2002B3FF46AAC838B0493E9
:108BD000D4E502204FF4A0220023FAF79BF90146C6
:108BE000002800F0E7802846089108F06EFB4FF05F
:108BF000010308997371C1444FF07F0B33E6002ADB
:108C00003FF44EAC614B1B685B057FF549AC94F8B3
:108C1000203003F00F03012B40F0CE805C4B1B781B
:108C200004F1220773B194F820000023C0F38011EF
:108C3000CDE900333A4600F00F00FEF799F900281D
:108C40007FF42EAC0C350221284608F05FFB41F280
:108C50003E2303800121284608F058FB03460B22DF
:108C60001A702846112108F051FB40F201130380CD
:108C700094F82030C3F380138370D4F82230C0F806
:108C80000330BB88A0F8073094F82030C3F3C0133A
:108C90004372A36AC0F80A30A38DC3810674FFF73C
:108CA000FFBB94F82130012B56D97F20CDE9060770
:108CB000FF200390099704F12309BB4638460121A0
:108CC0005B1ADFB2AEE501237AE4DAF8048086F8B5
:108CD00005B00DE6049B1E2B3FF606AE0123BB46F6
:108CE000737105E60C350221284608F00FFB40F6AB
:108CF0003E0303800121284608F008FB0F23037080
:108D00000721284608F002FBE488048047F67F71BB
:108D100040F2FF220023418082808371FFF7C0BBB5
:108D2000CDE9003394F820004246C0F3801100F0F2
:108D30000F00FEF71DF900283FF4D7ABFFF7B0BBDB
:108D400000274FF00B0A4FF00C0BB946FFF7E2BBC0
:108D50000023079309935DE57F23CDE9063792F859
:108D60008A100997FF23B9460393BB464A077FF54C
:108D700016AF637E5B063FF566ADAB46B8E5012BEB
:108D800018BF0223C7E600BFF0000020E800002063
:108D9000D7830020099B07933CE54FF00C084FF068
:108DA0000D0A87E648F280039381D672FFF778BBFD
:108DB00000DE4CE400DE16E700DE2FE76FF07F03F5
:108DC000D5E66FF07F03C3E64FF4A0220023022014
:108DD000FAF7A0F8834620B12846594608F075FAFC
:108DE000A0E500DEF8E700BF0379032B16D0053BB2
:108DF000222B13D8DFE803F01614141412121414E3
:108E0000141412121212121212121212121212123E
:108E100012121212121212121212140000207047B3
:108E200001207047022070470C490D4A0D4B4FF04E
:108E3000FF3010B408600C4C4FF0FF3041F6FF716A
:108E4000C2E900014FF0000C1F200021C3E900011E
:108E500084F800C010BCFEF745B800BF6040002099
:108E6000F0000020E8000020D783002070B588B013
:108E70001C460D9D9DF830C02E4616F8103B013360
:108E8000DBB22B70002B62D03649374B0C81C1E925
:108E900000028A7ACE606CF300028A720022996026
:108EA00001201146FBF7B6FF002852D1EB8B3BB1F6
:108EB0000134A4B2A34226D91B1BEB8308B070BDBA
:108EC000A88B0028FAD0002CF8D0284B284AEB1A9F
:108ED000A2FB032313F47F6FC3F307123DD10023DA
:108EE00001210232E883D2B2CDE90533CDE9031185
:108EF000CDE9013300931846FCF7B4FF10F0FD0FE5
:108F0000DCD000DEDAE7298FE9B1184A1944AB1A40
:108F1000174AA2FB0323091B13F47F6F89B2C3F323
:108F200007121DD100230232CDE90313CDE9053329
:108F3000CDE901330093D2B201211846FCF792FF2C
:108F400010F0FD0F07D10023EB8308B070BD00DEE9
:108F50009AE700DEAAE700DEF5E700DEA88BBEE7B1
:108F600000DEDFE7DC420020440200209007002002
:108F7000398EE3380368596B11B10868FDF73EBCC0
:108F8000704700BF00B17047064B10B502460C4653
:108F9000022001219C60FBF73DFF00B910BD00DEFF
:108FA00010BD00BF3402002003788BB110B50E4B0A
:108FB00000F11001996082689AB90C4C0A4B0022AA
:108FC000C0E9024111460120FBF724FF38B910BD6A
:108FD0000369596B11B10868FDF710BC704700DEDA
:108FE00010BD00DE9968E8E724020020758F0000BC
:108FF00000F0B4BA70B591F83A3043F001030C4672
:10900000064681F83A30023001F11002C0B2FDF795
:1090100045FCA8B900F0EEFAC569064615B12B6803
:109020009C4201D0002070BD00F09CFB08B178305C
:109030001ED1F369002BF5D09D42F3D100DEF1E79C
:1090400010F1780F054613D040F29123094A0A49DE
:109050000A4807F02CFF0A482A46314607F027FF46
:10906000002383F31188BFF36F8F0323184602DFB9
:109070000C2070BDAC2E0100EC2E0100042F01006D
:10908000242F010070B50F4D95F83A309B0716D587
:1090900029460020FFF7AEFF044670B995F83A3034
:1090A0006E6B60F3410385F83A3036B1686330681F
:1090B000FDF786FB3046FDF78FFB204670BD0C2484
:1090C000204670BD9007002000283CD070B5574D59
:1090D00095F83A300C4699078AB0164643D45B0798
:1090E0000CD50120FCF7C4FF0621FBF70DFE00287C
:1090F0007ED074B9AC832C87204631E04CB9AC8368
:109100002C876C634948EC830AB0BDE87040F7F7E0
:10911000FFB94749288D42F2107304FB03F3A1FB0A
:1091200003235B0AB3FBF0F39BB2AB836EB92E87CC
:10913000FDF740FB044600285FD0FDF747FB002801
:1091400058D004600CE0FFF79DBF3A4A06FB02F2DC
:10915000A1FB0212520AB2FBF0F2D31A2B870020B5
:10916000AC8B6863CEE7002C3FD0002A3DD0AA8BA1
:10917000002A3AD02A8F002A37D05A073FD501203B
:10918000FCF776FF0621FBF7BFFD88B342F21072B1
:10919000274B284802FB04F1A3FB012106FB00F04A
:1091A0002A8D490AA3FB0030B1FBF2F189B2400AD3
:1091B000B0FBF2F0401A80B20023CDE901330093F6
:1091C000A9831D49288709ACCDE905140121CDE902
:1091D0000311022203216B63EB8318460992FCF70B
:1091E00041FE2146FDF718FB00B10C200AB070BD0E
:1091F0001220FBE72046FDF7E3FA0720F6E70C4ACA
:10920000288D42F2107304FB03F3A2FB03135B0AE5
:10921000B3FBF0F399B2074B06FB03F3A2FB032366
:109220005B0AB3FBF0F35B1A98B2C5E79007002026
:109230005917B7D100881300F960000008B5FFF78F
:1092400021FF054B93F820206FF3020283F82020C2
:10925000BDE8084000F090B99007002081680B8FAE
:1092600003B170478B8B002BFBD0CB8B002BF8D13D
:1092700000B5124A12488B838A1AA0FB020212F42C
:109280007F6F83B0C2F3071013D14B6B821C4FF07A
:109290000B0CD88083F804C0D2B20091094B012195
:1092A0000020FCF775FE10F0FD0F04D103B05DF84F
:1092B00004FB00DEE9E700DEF8E700BF90070020CE
:1092C000398EE338858F000038B9084B93F83A207F
:1092D00060F3410283F83A20704700DE002292F8E2
:1092E0003A3062F3410382F83A30FFDE9007002003
:1092F000024B00280CBF1846002070479007002042
:10930000034A044B801AA3FB0030C0F307107047D8
:1093100090070020398EE338044A0068044B801A15
:10932000A3FB0030C0F30710704700BF9007002078
:10933000398EE338024B834218BF0020704700BFCC
:10934000900700200068034B984214BF00201030A3
:10935000704700BF90070020B8B90D4A92F83A3024
:1093600099070CD5117D126CC3F34000C1F3401373
:109370009840131E18BF012340EAC3007047106CC9
:10938000003818BF0120C000704700231B6CFFDEAF
:1093900090070020016A0023036231B14B7E086808
:1093A00043F080034B76FDF729BA00DEF6E700BFF5
:1093B00038B5CB690C460546C3B1186800F0C6FC49
:1093C0005DB948B10B490C4B0022D9600220012144
:1093D0009C60FBF71FFD38B938BD08B10749F2E7BB
:1093E000E3692BB10649EEE700DE38BD00DEE4E7B5
:1093F00000DEF7E79593000074020020B9940000A6
:109400002D95000010B5039C9DF808C0227801320C
:10941000D2B22270A2B10B490860887A0B810A4B44
:1094200000226CF30000103488724A60CC609960AE
:1094300001201146FBF7EEFC00B910BD00DE10BDA7
:1094400000DEE8E7FC4200206402002038B5C36972
:1094500004465BB3216A29B3002323620868FDF741
:10946000C1F9E16A31B10023E362012308680B719D
:10947000FDF7B8F9FDF7BCF9E5692868FFF75AFF71
:1094800030B1AA6804F110039A4204BF0023AB6014
:10949000E3696BB10023E36120460649BDE838402B
:1094A000FBF70ABCE16A0029DDD1E5E700DED1E780
:1094B00000DEEFE714430020F8B5C36904463BB370
:1094C000236A33B12378EBB92046BDE8F840FFF7B3
:1094D000BDBFE66906B330680023A0F8B430E56A82
:1094E000C5B10D230027E7622B7100F041FCAB7E74
:1094F000E88043F00203AE60AB76EF60237825622C
:10950000002BE1D000DE2046BDE8F840FFF79EBF0B
:1095100000DED5E700DEE4E700DEDCE7C3690BB17F
:10952000FFF794BF00DEFFF791BF00BFC3696BB1C7
:10953000037803F0FF023BB1012A09D183684BB9DC
:10954000054BC0E902307047FFF780BF00DEEFE750
:1095500000DEF3E700DEF3E71D95000008B50448E0
:10956000044B01223021FBF76DFB002008BD00BF3A
:10957000184300201443002008B50448044B01227E
:109580003021FBF75FFB002008BD00BF184300201F
:109590001443002038B5164B84689C420FD1E36910
:1095A0000BB31D682846FFF7C5FED0B195F83A30D9
:1095B000DB0715D42046BDE83840FFF747BF2046FB
:1095C00000F0C4FB88B194F88A30DA0608D4E36C62
:1095D00033B1E36C1C68E369002BEBD100DEE9E7F3
:1095E00038BD00DEE2E700DEDBE700DEEBE700BFD0
:1095F00018430020024B00280CBF1846002070477B
:109600001843002008B5034900683022FBF768FBC7
:10961000C0B208BD1843002038B5056849B1EB69F0
:109620000C4643B11868FFF785FE003818BF0120CB
:109630002070E86938BD00DEF4E700BF0068034B26
:10964000984214BF00201030704700BF184300201C
:10965000F0B58B681F6883B0064638460C46FFF7A6
:1096600069FE002831D0E368A1680122227143B36A
:109670001D68EF69002F56D03868FFF75BFE0028A1
:109680002CD090F83A30DA0712D4EB69002B59D07D
:10969000EB69002B58D02B7803F0FF02002B2AD067
:1096A000012A55D1AB68002B54D12C4BC5E90235AA
:1096B00021463046FDF796F803B0BDE8F040FDF7CF
:1096C00097B88B68002BD3D1F2E7254B9F4216D178
:1096D000A36801222271002BCAD1E9E73B6893F805
:1096E0008A30DB06D1D526606B6A002B34D0DC6073
:1096F0006C6203B0F0BD2846FFF7A8FED8E7054628
:10970000384600F023FB08B3A7F8B450D4E902238D
:10971000019353B10D223846227100F029FB019BC1
:10972000E080E560A4E700DEA6E7D36B01930D229D
:109730003846227100F01CFB019BE080E560002BA5
:1097400096D1B5E700DEA3E700DEA4E700DEAFE7D1
:1097500000DEA7E700DEA8E72C62C9E71D95000040
:109760001843002038B5194930220446FBF7B8FAEF
:1097700004F1100503302A462146C0B2FDF78EF8E9
:1097800018B110F1780F12D038BDE369D3B1186861
:10979000FFF7D0FDA0B10E490E4B0022D960032087
:1097A00001219C60FBF736FB70B9002038BD2846CC
:1097B000FDF74AF80028EED010F1780FEBD038BD55
:1097C0000549E9E700DEE2E700DEEEE718430020A6
:1097D0004D94000054020020B994000000B9704775
:1097E00000DE704738B505999DF810E00C7891F8C7
:1097F0008AC00D7F0134CCF3800C6CF34105E4B2D8
:109800000D770C7001F11005B4B1D1F880400B490F
:10981000C1E900028A7A0B816EF30002084B8A725A
:109820000022CD60996001201146DC60FBF7F2FA5E
:1098300000B938BD00DE38BD00DEE6E76043002039
:10984000A402002010B50C4650B9064B002201219D
:1098500002209C60FBF7DEFA00B910BD00DE10BDEF
:1098600000DEF2E784020020D0F8B0104FF6FF735C
:109870000022CB80C0F8B0203E23086881F8203059
:10988000FCF7BCBF30B5B82283B00D460A49044688
:10989000FBF726FA021D00942B46D2B201210020CC
:1098A000FCF776FB10F0FD0F04D10023A4F87C3008
:1098B00003B030BD00DEF8E78C43002008600148AB
:1098C00005F0FEBE7043002000B9704700B583B0BC
:1098D0000191FCF7B3FF0199814202D103B05DF819
:1098E00004FB00DEFAE700BF10B50C4640B9074B99
:1098F0000246012102209C60FBF78CFA20B910BDC2
:10990000FCF79CFF8442FAD000DE10BD94020020D8
:1099100010B5154BD0F880209A4204460FD0D0F8ED
:10992000B0104FF6FF73CB8000223E23C0F8B0206A
:1099300081F82030BDE810400868FCF75FBF0B4994
:10994000B822FBF7CDF90E230246A4F8922084F842
:109950009030C4F89440D4F88C0004F18C01BDE838
:109960001040FCF74BBF00BF95CB00008C4300209C
:1099700070B52B4C94F88A3043F0100384F88A3089
:10998000042004F110022146FCF788FF50BBE36C71
:109990004BB11D682846FFF7E5FE08B1783025D1A8
:1099A000EB69002B3AD1D4F88C00FCF709FF256F46
:1099B0000026A4F87C6065B12868FCF701FF01204F
:1099C00000F07EFC284600F075FC012000F086FCCB
:1099D0002667002513491248A4F8B450FBF76CF928
:1099E000284670BD10F1780F054601D10C2070BDDE
:1099F00040F236230C490D480D4A07F058FA0D483D
:109A00002A46002107F053FA002383F31188BFF39D
:109A10006F8F0323184602DF0C20E8E700DEC2E761
:109A20008C43002088430020EC2E0100042F01000D
:109A30003C2F0100242F01002DE9F04F85B0044692
:109A40000020BDF838B0BDF83CA09DF840900092D1
:109A50000E461D46FFF74CFC28B1D0F84080074663
:109A6000B8F1000F03D00C2005B0BDE8F08FFCF773
:109A7000A1FE0190002800F09880FCF79BFE029068
:109A8000002800F08F80FCF7A1FE002800F08780FE
:109A900003904948FBF7FAF80399034600287BD066
:109AA00090F88A00019A68F3410083F88A000A60FE
:109AB000D3F8B000029AC3F88C20002879D1C3F8FB
:109AC000B01083F88B6084F002011E7F93F88A0047
:109AD000A3F878B0C1F3400161F341061E77DE7E42
:109AE000A3F87AA069F3C706DE768900C4F380067E
:109AF00020F01C0041EAC601014383F88A100021CE
:109B0000A3F87C10A3F87E10D964D9835984196412
:109B1000596403F15000019300F080FB019B196F21
:109B2000002944D10021C3E902111B611970796435
:109B300097F83C1004F0010421F00F012143CA07FB
:109B400087F83C100BD5CCB1197F97F83C4000202A
:109B500064F3000119773B6405B0BDE8F08F93F81A
:109B60008A10009A62F3000183F88A102968C3F80A
:109B70008410A988A3F88810002CE5D193F88A10E6
:109B8000009A62F3000183F88A102968C3F88410F0
:109B9000A988A3F88810D7E70846FCF71DFE0298AD
:109BA000FCF70EFE0198FCF70BFE07205CE700DED9
:109BB000B8E700DE83E700BF884300202DE9F041CD
:109BC00006460020FFF794FB002851D0036C002BC1
:109BD0004ED090F83C3043F0020380F83C30046CE7
:109BE000002C45D0D4F8B030002B41D094F88A3006
:109BF00043F0100384F88A30B4F87C309BB273B120
:109C00001E49B8222046FBF76BF8FF2833D80430F2
:109C100004F110022146C0B2FCF740FE30BB002028
:109C2000FFF766FB00250564D4F8B070D4F88C000B
:109C3000D7F80080FCF7C4FD4046FCF7C1FD38466C
:109C4000FCF7CAFD0C224FF6FF7384F89020A4F8AD
:109C50009230442204F18C03C4F8B05084F8AC2054
:109C6000C4F8944033602846BDE8F0817830D6D0FF
:109C70000C20BDE8F08100DEC9E700BF8C43002066
:109C800030B9044BB3F87C309BB20BB1FFF770BE18
:109C9000422070478C43002078B9094AB2F87C30E2
:109CA0009BB253B192F88A30890023F00C0301F083
:109CB0000C01194382F88A1070474220704700BF98
:109CC0008C43002008B50648064B0122B821FAF75C
:109CD000B9FF01220021044808F0B1FB002008BDB3
:109CE0008C430020884300207043002000B583B0DF
:109CF00001A8FFF763FF0B4BB3F87C309BB20BB1AD
:109D0000FFF736FE084B07480122B821FAF79AFF01
:109D100001220021054808F092FB002003B05DF805
:109D200004FB00BF8C4300208843002070430020C8
:109D300038B90548B0F87C309BB2002B08BF002032
:109D400070470020704700BF8C430020024B8342C5
:109D500018BF0020704700BF8C4300200068034BF1
:109D6000984214BF00201030704700BF8C43002081
:109D70000149B822FAF7B4BF8C43002002490068B9
:109D8000B822FAF7ADBF00BF8C43002038B5056F8D
:109D900004466DB12868FCF713FD012000F090FA2D
:109DA000284600F087FA012000F098FA0023236784
:109DB0000023A4F8B43020460249BDE83840FAF741
:109DC0007BBF00BF8843002070B5044615461E4681
:109DD00089B990F88A2002F00102AA4201D000203D
:109DE00070BD00F184010622184608F05DFDB0FA4E
:109DF00080F0400970BD1946104600F03DFC002877
:109E0000EDD094F88A3065F3000384F88A30336823
:109E1000C4F88430B388A4F8883070BD70B591F868
:109E20003C300C4603F00C01042901D0002070BD29
:109E3000D9070646154606D496F88B00401BB0FAA3
:109E400080F0400970BD90F88A0006F1840100F0AE
:109E5000010000F039FC0028E9D194F83C30DB0720
:109E6000E4D4E9E708B50020FFF742FA00230364D1
:109E700008BD00BF2DE9F8438B681E6896F88A304C
:109E800013F010083BD1B6F87C309BB2BBB34D7ECB
:109E9000C5F30115EB1C03F00303012B0C46074629
:109EA00018D91849D6F8B090B8223046FAF718FFFA
:109EB000A9F80600C6F8B080637ED9F8000003F068
:109EC0003003302B08BF4FF01A0889F8208049462C
:109ED000FCF794FC012D07D9012323712146384654
:109EE000BDE8F843FCF78ABC0D23074AC6F880207A
:109EF000237121463846BDE8F843F6F799BBBDE823
:109F0000F88300BF8C43002095CB0000F0B5846837
:109F100094F88A1011F010018BB03AD1B4F87C306B
:109F20009BB2002B35D0837C13F0040605465BD131
:109F3000028A678CCDE90866002A5BD1DB07228C98
:109F400029D50023A4F87E30237F658C6FF3C303EB
:109F5000BD42237742D0DDE9082301351343ADB27A
:109F600064D04049B8222046FAF7BAFE3E4BCDE90C
:109F70000534DDE90813021D00200091CDE90356E8
:109F8000CDE90100D2B20121FBF76CFF10F0FD0F0B
:109F90005CD10BB0F0BD94F88A10531C1F299BB202
:109FA0003AD9B3EB511F4FEA511255DAD21A62F384
:109FB0004711B4F87E2084F88A10002AC4D09A424F
:109FC0003FD9D21A92B20023062AA4F87E206384D5
:109FD0002FD97FBB237F67F3C3032377DDE90823F2
:109FE0001343D6D00025BCE720460BB0BDE8F040B7
:109FF000FFF748BC08AA09A9F6F7F6F9B4F87830D3
:10A00000638494F88A30228C66F3471384F88A308C
:10A01000AB7CDB07BFD594E7B4F87E20002ACED115
:10A02000B4F87C2092B2A4F87E20C6E7002DB0D010
:10A0300097E70123227F012663F3C3022277354687
:10A040008FE70A492046FFF71DFCA2E7FCF7F6FB65
:10A0500084429ED000DE9CE705492046FFF712FCB3
:10A0600097E700BF8C430020C9980000E9980000E2
:10A0700045980000F8B500284DD1294E96F835C016
:10A0800096F8343063450C46054640D1237819468E
:10A0900043B9012A3BD96378013A0134D2B2194657
:10A0A000002BF6D06078282809D001339BB29A4261
:10A0B0002DD9521A013A12F0FF021C44E6D1082BA6
:10A0C00025D10CF10107FFB2022F21D00620282351
:10A0D00010FB07303D46D4F8023033503044A379AA
:10A0E0000371052107EB4707FAF7ACFF06EB4707BB
:10A0F00000F03F0097F82D30012860F3050387F842
:10A100002D3004D9B4F80730F38686F83550F8BD01
:10A1100028200027DFE700DE002393F83530FFDE3C
:10A120008C4300202DE9F04782B00E469DF8289020
:10A1300090461F46FFF7FCFD002864D0C37E03F065
:10A140000703042B04465AD010F8505F0DF10701A5
:10A1500002F0BEFDEDB28246CEB9C5EB0515254431
:10A1600095F85230DB070ED5037866F300030370D1
:10A170009DF807303146A02284F851302046F7F789
:10A18000FBF8002845D1002002B0BDE8F08708F1B7
:10A19000FF33012B2FD8A9F102030A2B2BD80B9BDD
:10A1A0004BB319464A46033008F068FB9AF8003072
:10A1B00068F342038AF800309AF80230102F69F3EE
:10A1C00006038AF8023016D89AF80030FF0003F030
:10A1D000060347F00107C5EB05151F4325448AF820
:10A1E000007095F852209DF8073012F001020ED051
:10A1F00084F85130C7E7112002B0BDE8F0870C2089
:10A2000002B0BDE8F087422002B0BDE8F087A0218F
:10A21000B2E70230B7D000DEB5E700BF10B51E22AE
:10A2200004460021023008F037FB002323706370DE
:10A2300010BD00BF027843789A4208BF03780F220E
:10A2400002FB030002300078C04300F001007047B9
:10A250000C4991F8842091F885309A420AD8A3EBF2
:10A26000020C5FFA8CFC604509D89A4207D051F87D
:10A270002200704721339B1ADBB29842F7D90020A5
:10A28000704700BF44440020094A92F8841092F8B5
:10A2900085308B4209D04B1CDBB2212B08BF002339
:10A2A00052F8210082F8843070470020704700BFC8
:10A2B000444400200149FAF7FFBC00BFCC44002011
:10A2C000054A0028137802DC0344137070471F2BE3
:10A2D000FAD900DE1378F7E7D88300202DE9F84398
:10A2E000194F3B78984228BF184630B3DFF85C908E
:10A2F000DFF85C8099F88540451EEDB20134E4B288
:10A30000212C99F8843008BF0024A34215D0FCF713
:10A3100051FA0646404686B1FAF7B8FC78B10660B5
:10A3200099F8853049F823003B7889F88540013D4C
:10A33000EDB2013BFF2D3B70E0D1BDE8F883304624
:10A34000BDE8F843FCF73CBAD88300204444002021
:10A35000CC44002010B5094B09490024181DA1F870
:10A36000844020224FF4B871FAF76CFC054B202290
:10A37000FF201A70FFF7B2FF204610BDCC4400202A
:10A3800044440020D883002010B5094B094900241B
:10A39000181DA1F8844020224FF4B871FAF752FC3E
:10A3A000054B2022FF201A70FFF798FF204610BDB2
:10A3B000CC44002044440020D883002038B54FF01E
:10A3C000060C1C460C2380F800C013700D4602F0EA
:10A3D0007DFC14232870237038BD00BF054B064A4E
:10A3E00010B41F204FF0FF3425211C60187111702C
:10A3F00010BC7047D0720020D983002042880088AA
:10A4000050407047F0B5344D344C48404FF0030C89
:10A41000060A5FFA80FE0EEB8E2E06EB862004EA1B
:10A42000401705EA400605EA4E0004EA4E1E3E4388
:10A4300040EA0E0000EB002706EB062E06EB0E2688
:10A4400000EB0720360CC0F3074040EA062000EB83
:10A4500000100CF1FF3C08441CF0FF0C80B2D7D177
:10A4600041401F48A0FB01400C1A00EB540040097A
:10A4700000EBC00400EB8400081AC0F3C40400F031
:10A480000705145D2C41E407C0B21CD401FB03F3A3
:10A49000561EC3F307430432604600F1080516F860
:10A4A00001CFEDB201461CF0010F01F101044FEAAA
:10A4B0005C0C02D043B1013BDBB2E1B2A942F2D164
:10A4C00008469642E9D1F0BD0730401AC0B20728CD
:10A4D0000846F6D8F0BD00BF1021020040840800F5
:10A4E0004D91CFBA2DE9F047884691461E460BB1F3
:10A4F000FF233370164F00F0010A3D46002406E0AA
:10A50000534519D00134082C05F1080511D007EB8B
:10A51000C4008079C207C0F34003F1D4002EF1D00B
:10A520003378FF2B08BF34700134082C05F108057F
:10A53000EDD1FF20BDE8F08706222846414608F00D
:10A54000B3F90028DED1EB794B45DBD1E0B2F1E77E
:10A55000D872002008207047164B9A7B93F806C0EB
:10A56000997D6FF300029A739A7F6FF300029A77D6
:10A5700093F82E206FF3000C6FF300016FF30002CD
:10A5800083F806C0997593F826C093F8361083F8BF
:10A590002E2093F83E206FF3000C6FF300016FF351
:10A5A0000002002083F826C083F8361083F83E208E
:10A5B000704700BFD8720020F0B50678FF2E83B038
:10A5C0002DD0471C0A4604460D460DF107033946B7
:10A5D0003046FFF787FF072829D99DF80720072A6B
:10A5E00021D8154901EBC20C00239CF8060066F344
:10A5F00041008CF80600D4F8010041F83200B4F8AC
:10A600000520ACF804209CF806208CF8075042F096
:10A6100001021846E6468CF8062003B0F0BD002380
:10A62000184603B0F0BD0723184603B0F0BD12234F
:10A63000184603B0F0BD00BFD872002084460078F1
:10A64000FF2814D008B50A4600230CF10101FFF7DA
:10A6500049FF0728034601D9422008BD054A02EBFD
:10A66000C30300209A796FF300029A7108BD00209D
:10A67000704700BFD87200202DE9F843114F88467B
:10A680003E46002500F0010903E0082D06F108060A
:10A6900014D007EBC5030135987910F00104C0F31D
:10A6A0004003F2D04B45F0D106224146304608F037
:10A6B000FBF80028E9D12046BDE8F88300242046B5
:10A6C000BDE8F883D87200202DE9F047134F884683
:10A6D00091463E4600F0010A002503E0082D06F1F0
:10A6E000080617D007EBC5030135987910F001046F
:10A6F000C0F34003F2D05345F0D106223046414624
:10A7000008F0D2F80028E9D1F3794B45E6D120468C
:10A71000BDE8F08700242046BDE8F087D87200200D
:10A7200000F046BA684620F007018D4601B502F0F8
:10A7300021FCF7F769FDBDE801408546704700BF81
:10A7400008B50A4BD3F840213AB90120FAF7C0FB0B
:10A75000BDE808400220FAF7BBBB0020C3F8400167
:10A76000D3F84031FBF7F6FAEFE700BF00B0004046
:10A770000020FAF7ADBB00BF90B90E4B0E4A197816
:10A7800010788842CBB20DD10C480D4990F800C02A
:10A79000013313700B78634507D003780B70704753
:10A7A00000DEEAE700DE1378EEE700DE03780B70E8
:10A7B000704700BFDA830020DB830020DF830020A6
:10A7C000DE8300200B4A0C4B117893F800C08C45B7
:10A7D0000DD012781A70094A094B18B911781878F7
:10A7E000884202D012781A70704700DEFAE700DE65
:10A7F000EFE700BFDD830020DC830020DA83002048
:10A80000DB83002002F0E6BC08B50B480B4B027856
:10A8100019788A420CD00A4B017000220399996082
:10A8200001201146FAF7F6FA00B908BD00DE08BDAE
:10A8300000DE1978EFE700BFDA830020DB83002019
:10A84000B40200202DE9F041304A314D12782B78C6
:10A850009A428AB00E4605D12E4B2F4A1B781278A9
:10A860009A424BD03768DFF8B48007F12D0424F00A
:10A870007F44D8F800102046FBF7CEFB10F4000010
:10A8800002D10AB0BDE8F081254A264B11781A782A
:10A8900091421CD03046244BC168C8F800400022C9
:10A8A000CDE90732214BCDE90322CDE90531CDE9D0
:10A8B00001222D2300932C780134E4B23B4611464B
:10A8C00010462C70FBF7B2FA0AB0BDE8F081114ACD
:10A8D0001149127809789142DCD01A780132D2B24B
:10A8E0001A700022124B009211461046FBF750FBE3
:10A8F00010F0FD0FCED000DE00DECBE70768DFF8FA
:10A900001C8007F12D0424F07F44C4E7DE8300207F
:10A91000DF830020DA830020DB8300202073002007
:10A92000DC830020DD83002079A7000009A8000057
:10A93000C5A700007A4A9368002B00F096802DE9A5
:10A94000F04F136889B08146002B46D04FF0FF339B
:10A950008DF80A300DF10A00FCF78AF80446002849
:10A960003BD0037F9907F5D1857A15F00205F1D127
:10A97000C3684B4555D00668A8462F460DF10A001E
:10A98000FCF776F88346F0B1027F9207F6D1827A1F
:10A990009307F3D4C268B8F1000F21D04A4558D0CC
:10A9A000DBF800A031465046FBF736FB00F4000010
:10A9B00000280DF10A001CBF5F465646FCF758F808
:10A9C00083460028E0D1002F08BF27463946384685
:10A9D000FFF738FF30F0020339D109B0BDE8F08F3E
:10A9E0004A458046DCD1237FE16843F002032377A8
:10A9F0002046A3699847FF238DF80A300DF10A001D
:10AA0000FCF736F804460028E7D0037F9F07F5D10E
:10AA1000837A9E07F2D4C3684B4502D000DED4F897
:10AA20000C903F4A4846D2E9001303AA98470646CD
:10AA3000002843D010F1100F59D0394A00209368F4
:10AA40001168984716F10B0F10D08C36C5D000DE78
:10AA5000C3E7227FE16842F0020222772046A26922
:10AA60009047D8457FF472AFC5E770472C4A002362
:10AA7000D2F80890D2E9004802261360FF278DF82B
:10AA80000B700DF10B00FBF7F3FF90B1037F9A07FA
:10AA9000F7D40DB9DB07F4D4C368A342F1D1037F27
:10AAA000826943F002030377214690478DF80B70CB
:10AAB000E7E70125AE420AD02E46E0E7237FA269F0
:10AAC000E16843F0020323772046904785E70022A0
:10AAD000CDE904220692039B00964946404604AA0B
:10AAE0000794FBF77DFF00287FF477AFAFE7A37AE9
:10AAF00043F00203A3720DF10A00FBF7B9FF014610
:10AB000000283FF46AAF037F9D07F4D1837A9C0746
:10AB1000F1D4FFF797FE30F002033FF45EAF96E703
:10AB20002473002010B5174807F057FB30B3164BBD
:10AB300000249C6000F0FEF900281EDB2146012065
:10AB40002246F7F775FE22460B200121F7F770FE2B
:10AB5000214622461820F7F76BFE0C4B1022C3F853
:10AB600004230120F7F734FE0B20F7F731FE1820FD
:10AB7000F7F72EFE02F018FA204610BD6FF0120013
:10AB800010BD00BFA02A0100247300200010004067
:10AB900008B500F0DFF9002809DB0120F7F726FEF1
:10ABA0000B20F7F723FE1820F7F720FE002008BD42
:10ABB000034603488AB2194683681B68184700BFDA
:10ABC000A02A01000020704730B5044683B078B356
:10ABD0001D4B1A68824225D0FF250DF107008DF824
:10ABE0000750FBF745FF38B91AE0A1420AD00DF132
:10ABF0000700FBF73DFF98B1037F9B07F7D4C168BF
:10AC0000002CF2D1037F826943F00203037790475F
:10AC10000DF107008DF80750FBF72AFF0028EBD154
:10AC200003B030BD9B686BB1014600209847D3E765
:10AC3000054A9368002BCFD011680029CCD00020A2
:10AC40009847C9E700DEC7E724730020002070475B
:10AC500010B50446FBF7FEFE8CB90D4B9A68AAB1FD
:10AC60001C6800229A601A6004B124680020FBF777
:10AC700019FF2046FBF7B8FF28B1002010BD0028BF
:10AC8000F3D100DEF1E700DE002010BD00DEE7E7D3
:10AC900024730020054A136892681B1A18BF012309
:10ACA000B2FA82F00B704009704700BF2473002095
:10ACB0002D20704710B51446FBF7ACF92146FBF781
:10ACC000ABF9034610F4000004D103330E2B88BF08
:10ACD000184610BD002010BD262810B504461DD012
:10ACE000272813D0252809D00A281FD9272822D998
:10ACF00000DE2046BDE8104002F0D4B9022002F088
:10AD0000CBF92046BDE8104002F0CCB9502002F04B
:10AD1000C3F92046BDE8104002F0C4B91A2002F081
:10AD2000BBF92046BDE8104002F0BCB9023040003B
:10AD300002F0B2F9E5E70330400002F0ADF9E0E7D8
:10AD400002F01ABA08B502F045FABDE8084002F070
:10AD5000A1BB00BF08B502F03DFA02F09BFBBDE8C5
:10AD6000084002F05FBB00BF08B502F033FA02F002
:10AD700091FB02F075FBBDE8084002F053BB00BF39
:10AD800008B50146114802F005F902F059FA60B120
:10AD900002F06CFC02F040F900F004F900280EDB30
:10ADA000BDE808400020FFF753BF02F0F3F902F0BE
:10ADB0005DFC02F031F900F0F5F80028F0DA00DE71
:10ADC0000020BDE80840FFF743BF00BF05A8000012
:10ADD0002DE9F04F89B01F469DF848B0FF2380460B
:10ADE000894692468DF81F300DF11F00FBF740FE9B
:10ADF000002866D0037F9D07F6D1837A9C07F3D4A1
:10AE000005683E689DF81F30059304462946304684
:10AE1000FBF702F9BBF1000F4CD0BC4208BF002485
:10AE200026460DF11F00FBF723FED0B1027F9107EC
:10AE3000F7D1827A9207F4D402680490294610462A
:10AE40000392FBF7E9F8039A049B00F40000002842
:10AE50000DF11F001CBF15461E46FBF709FE00281A
:10AE6000E4D1059B8DF81F30314B9A687ABB76BBD5
:10AE700024B1BBF1000F48D1BC4244D1FA681A603A
:10AE8000C3E901893846D04704460DF11F00FBF79E
:10AE9000EFFD014650B1037F9A07F6D1837A9B07F5
:10AEA000F3D4FFF7CFFC30F002033FD1204609B0C6
:10AEB000BDE8F08F0002B0D5FF23354605935C4610
:10AEC000AEE71B4B9A680446002AD7D0264649466F
:10AED000CDF800B0534640463A46FBF781FD0146A7
:10AEE00078B1BBF1000F09D1BB7A980706D4C6B17F
:10AEF0003046FFF7A7FC30F0020310D16FF0760464
:10AF0000D4E700DEEDE700DEB8E7CDF800B0534649
:10AF10003A4649464046FBF763FD0028EED100DE85
:10AF2000ECE7002C14BF26460E46E1E700DEBDE745
:10AF30002473002010B5012002F026FF04490023ED
:10AF400001244B608C60CB60BDE8104006F067B810
:10AF50003473002010B5012002F016FF04490446A6
:10AF600006F0D8F82046BDE8104006F0AFB800BFA4
:10AF70003473002008B50A4BBFF35B8F53E8002FF2
:10AF8000511C43E800100028F8D1BFF35B8F002A62
:10AF900001DD002008BD02F0FFFE002008BD00BF5B
:10AFA0003073002008B50E4BBFF35B8F1A68BFF3F8
:10AFB0005B8F002A11DDBFF35B8F53E8002F511E1A
:10AFC00043E800100028F8D1BFF35B8F012A01DDB0
:10AFD000002008BD02F0F6FEFAE76FF0770008BD2A
:10AFE0003073002032207047014B33F81000704757
:10AFF0007C2F010000B9704700DE7047814208B520
:10B000008B8909D09BB1CB898BB9134801F0C2FF62
:10B0100002F0C0F8002008BDCBB90B79DA07F9D4EB
:10B020000B7CDB06F6D40D4801F0B4FFF0E7CB69EA
:10B0300013B16FF08B0008BD094B1360FFF79AFF47
:10B04000002802DB6FF00A0008BD00DEFAE7CB89BA
:10B05000002BE2D1D9E700BF9DB1000095B20000FE
:10B0600069B200000021F6F7EFB900BF08B5064B42
:10B0700003989860002211460120F9F7CBFE00B931
:10B0800008BD00DE08BD00BFD402002010B5044694
:10B09000FFF76AFE2379227C6FF3000322F0180287
:10B0A00023719B06227417D5962002F003FA002321
:10B0B00018461A46194602F031F90120FBF740FC08
:10B0C00088B1203002F04AF802F09CF92146074886
:10B0D000BDE8104001F05EBF02F082F90120FBF7ED
:10B0E0002FFC0028EDD100DEEBE700BF11B500001A
:10B0F00010B50446FFF738FE02F0A8F90120FBF76F
:10B1000061FD20B12046BDE81040FFF739BE00DEEA
:10B110002046BDE81040FFF733BE00BF08B5FFF77B
:10B12000B5FF02F031F8BDE8084002F0FFBA00BFF9
:10B1300070B50546FFF706FE02F052F90120FBF755
:10B14000FFFBF0B1203002F009F802F065F800BB17
:10B1500002F0FAFA00210446084602F00FF8002136
:10B160000646084602F006F83444CB34201A02F0B2
:10B1700089FA02F047F929460748BDE8704001F016
:10B1800009BF00DE203001F0E9FF02F045F8002899
:10B19000DED000DEDCE700BF11B5000030B50446AC
:10B1A00085B0FFF7E1FD0DF10F012046FFF772FDBD
:10B1B00008B105B030BD054602F048F92279009586
:10B1C000C2F34103013303F00303032B08BF002341
:10B1D00063F3420222712B46012229462846FAF7E0
:10B1E000D7FE9DF80F3073B1A389002B30D1237C9B
:10B1F000DA060FD494F90430002B1EDB2046FFF74B
:10B20000BFFD05B030BD0120FBF7DCFC0028EBD111
:10B2100000DEE9E76FF304132374FBF7ADFB01468F
:10B22000F0B10A230B718C60A368CB600868FBF750
:10B23000C7FB94F90430002BE0DA0A4B002101220D
:10B2400008469C60F9F7E6FD0028D7D000DED5E778
:10B25000E389002BCBD1237943F080032371C6E728
:10B2600000DEDEE7C402002070B5C36804461E6835
:10B27000FAF7D0FE05463046FFF71AFD00232D1AD7
:10B28000C4E90053238120460121BDE87040F6F750
:10B29000DBB800BF10B50446FFF7F8FE237922792A
:10B2A000C3F34103013303F00303032B08BF00235F
:10B2B00063F34202227114BF03F125002520FFF73A
:10B2C0000BFDFAF7A7FEC11C002002F073F9BDE8E0
:10B2D000104002F02BBA00BF10B548B10C46FFF782
:10B2E00061FE00280BDB2046BDE81040FFF7B0BC34
:10B2F000044801F04FFEBDE8104001F04BBF00DEF6
:10B30000F1E700BF9DB100002DE9F043054683B091
:10B3100003200F4690461E46FBF712FB00286AD01A
:10B320000446FBF729FB4FF6FF73E3802B7C58079D
:10B3300049D003F00703012B57D0042B58D000DE6F
:10B3400094F8202002F00F03042B45D0072B3CD1AA
:10B350000023AB60A56002F083F9206102F0EEF9F2
:10B360008146287C414600F0070001F007FF637E1C
:10B37000A9EB000068F34103606163760095297CC6
:10B380001E4B424601F0070104F1200000F0BAFB19
:10B39000A37E60F30003A376DB0716D52B7C43F076
:10B3A00010032B746FF00F0597B97F20637E207612
:10B3B00066F30003206863762146FBF701FB28460D
:10B3C00003B0BDE8F083052323710025002FECD0E6
:10B3D00002F022F8C0B2E9E72B7C1907F5D5052366
:10B3E00063F3030284F82020EFE706232371A7E725
:10B3F00008232371A4E76FF06805E0E735B9000082
:10B40000002070470020704710B582B00446FFF757
:10B41000B1FD002809DB084A0849094800940023C7
:10B42000FBF70CFC18B902B010BD00DEF3E7773073
:10B43000F9D000DEF7E700BF65B00000D9B2000028
:10B44000FDAF000070B50B4C0546FFF78DFCE560C5
:10B450002E68FAF7DFFD05463046FFF729FC00238A
:10B460002D1AC4E90053238120460121BDE8704014
:10B47000F5F7EABF4473002003791B0703D5101EBC
:10B4800018BF012070470120704700BF70B51D46EE
:10B4900011B1DB78DC072ED56B78072B28D9E9783A
:10B4A00089071ED50D2B23D906790AB133071FD57D
:10B4B0002B78C6F38012B2EBD31F4FEAD3141DD002
:10B4C000C6F3C106012E13D99CB1EB7B03F0C00378
:10B4D000402B0DD1059B13B1059A01231370012454
:10B4E00007E0002AFBD00179C1F3C004204670BDFB
:10B4F0000024204670BD0C46204670BD0622113047
:10B5000005F10A0107F0D0F90028E8D0D8E700BF1C
:10B510002DE9F04385B0044601F088FE10F0FF03EA
:10B5200013D1FF228DF80D308DF80B308DF80E20E1
:10B530008DF80C20FFF718FCA148214601F02AFDE8
:10B5400001F028FE05B0BDE8F08301F08FFE05464E
:10B5500001F090FF8DF80B0001F096FF0022FF2311
:10B560008DF80D208DF80E308DF80C0001F064FF81
:10B57000064601F045FFEDB20746FFF7F5FB002D4B
:10B58000DAD00120FBF7DCF90546002800F0D9806D
:10B5900095F8203003F00F03072B05F1200800F089
:10B5A0009C8023799DF80B201B0738D495F8202028
:10B5B000002312F00F01F6B28DF80F3032D00629B9
:10B5C00030D04520C840C00700F1BD80012900F0FF
:10B5D0009580072940F0D080237C5A07ACD022798F
:10B5E00012F00102A8D10DF10F010191FF2100918C
:10B5F000434601212046FFF749FF00289CD095F8DB
:10B600002130002B98D09DF80F303A463146204625
:10B61000FFF77AFE00288FD010308DD192E7002AF4
:10B62000C4D189E795F82130052B85D9252B83D8FE
:10B63000237903F02103202B18BF0023E5D19620A6
:10B6400001F038FF002001F01FFE00233A4631468A
:10B650002046FFF759FE00287FF46EAF01F010FE80
:10B660000278032161F30302027095F8202001782B
:10B67000C2F3801262F3C7110C220170427022796A
:10B68000C9B2C2F3801262F38611024602F8021BAD
:10B69000D4F81110C0F80210B4F815109180D5F844
:10B6A00022208260EA8C828101F05EFD01F0B4FD0F
:10B6B00000285FD102F03AF8237943F001032371A7
:10B6C00095F820301D0703D1237C43F00803237431
:10B6D0003C48214601F05EFC34E70DF10E03019376
:10B6E0000DF10D0300930DF10B0203AB4146204613
:10B6F00000F0E4FC00287FF454AF57E795F82130C0
:10B700000C2B7FF419AF94F80480C8F38013B3EBCB
:10B71000D21F4FEAD21922D0C8F3C108B8F1010FE5
:10B720007FF60AAFB9F1000F3FF406AF95F82D3060
:10B7300003F0C003402B7FF4FFAE01238DF80F30E0
:10B7400061E700DE24E795F82120052A7FF6F4AEB4
:10B75000252A7FF65AAF07293FF43EAFECE60622D2
:10B7600005F1280104F1110007F09EF800283FF4CC
:10B770004AAFD1E700DE9DE704297FF4DDAE95F8FE
:10B780002130052B7FF6D8AE252B3FF6D5AE237999
:10B79000DB077FF5D1AE01F073FD95F8203002781C
:10B7A000C3F38013B3EBD21F7FF4C6AE083006227A
:10B7B00005F1220107F078F800287FF4BDAE1EE7FE
:10B7C0001DB1000031B1000030B5044683B0FFF771
:10B7D000CBFABCB10DF107012046FDF71DFF9DF826
:10B7E000073005466BB1234B1B88002B38D01DB1A9
:10B7F00095F90430002B25DB2046FFF7C1FA03B092
:10B8000030BD50B91B4B1B88002BF5D10220FBF734
:10B81000D9F90028F0D100DEEEE7FBF7ADF80146DC
:10B8200028B38B7E8D600A220A71EA6B0868CA60B1
:10B8300043F002038B76FBF7C3F82046FFF7A0FA2C
:10B8400003B030BD0C4B0021012208469D60F9F782
:10B85000E1FA0028DFD12046FFF792FA03B030BDAD
:10B860000220FBF7AFF90028C1D100DEBFE700DE00
:10B87000D7E700BFF2750020E4020020F8B50746C4
:10B880000D461646FFF75EFA0120FBF759F890B314
:10B89000203001F063FC01F0A3FD01F0BDFC40BBD2
:10B8A00001F052FF7B790446012103F0070001F00B
:10B8B00065FC7B79044403F00700022804F1A3042B
:10B8C00015D004280CBF4FF4BC73282301211C445D
:10B8D00001F050FC201A01F0D5FE01F027FF01F025
:10B8E00091FD31462846BDE8F84001F053BB1823CE
:10B8F000ECE700DED4E700DECAE700BF8368024958
:10B9000002469868FFF7BABFA5C000000149024689
:10B91000FFF7B4BF89C00000884208B507D0FDF723
:10B9200011FD00280CBF6FF08B00002008BD00DE69
:10B93000F5E700BF2DE9F84F8146FFF715FAD9F872
:10B940000CA0D9F808009AF8027001257F09BD40C3
:10B95000EDB289F80C50FDF7F5FC002800F0858069
:10B960004FF0000B9AF900309AF80240002B4FEA92
:10B9700004249AF8013004F4F85444EA03049AF8D1
:10B980000030B5BF4FF496721E224FF49E784FF0F0
:10B990002E0813F0400F14BF32264FF4FA76374BBF
:10B9A00002FB04F404FB06F6A3FB0636344B00222C
:10B9B000012128461A8001F031FBAA0002F0FC02A6
:10B9C000FF21082001F096FB9AF8000000F03F00EC
:10B9D000FFF782F909F12000B60C01F0BFFBBBF1C3
:10B9E000000F3DD02748594601F0D4FA962001F0C7
:10B9F00061FD2A4601230021284601F08FFCD9F879
:10BA00001430012128461C44FFF79AF9A41B241A7C
:10BA1000A4F11001002001F0FBFD0F3C844281469F
:10BA20002AD101212846FFF78BF946440346B14449
:10BA300001212846994401F0A1FB012F81440DD03A
:10BA4000022F0CBF4FF4BC702820484401F028FEA0
:10BA500001F06CFEBDE8F84F01F0D4BC1820F4E70B
:10BA60000948494601F096FAC0E7D9F808B00146FE
:10BA70005846FDF7D1FD75E700DED2E783DE1B43B4
:10BA8000F275002089C00000A5C0000010B568B1A3
:10BA90000C46FFF787FA00280FDB0220FBF792F82D
:10BAA00068B12046BDE81040FFF7D2B8054801F064
:10BAB00071FABDE8104001F06DBB00DEEDE700DE7D
:10BAC000EFE700BFC9B7000010B582B00446FFF72A
:10BAD00051FA002809DB084A084909480094002364
:10BAE000FBF7ACF818B902B010BD00DEF3E7773011
:10BAF000F9D000DEF7E700BFF11500008DBA0000B5
:10BB000019B900002DE9F04F0446007883B000F029
:10BB10000F00072889469046019340F0928066788E
:10BB2000002E00F08880A3789D0600F08480E378E2
:10BB3000D8074CBF0A340434990748BF063413F0C1
:10BB4000040B1CBFA34601341A0748BF0234DB06AE
:10BB500071D5A2786378170207F4F8571F436AD0AB
:10BB60005F2A4FEA521366D8227802F03F01242957
:10BB700061D809F003010E4412F0800F06F10906A6
:10BB800014BF4FF496711E21C9F34000F60001FB6B
:10BB900007F7C640394406F5967081424BD312F040
:10BBA000400F18BF3225294A08BF4FF4FA7507FB2A
:10BBB00005F54FF0010AA2FB05250AFA03FAAD0CC0
:10BBC0005FFA8AFABBF1000F39D001F0B7FFB0B3CA
:10BBD0009BF800B00BF01F0B06EBCB0B4146484621
:10BBE00001F0CCFA01210346504605F28D459A46F4
:10BBF000FFF7A6F85D4455440544AF421BD8012029
:10BC0000FAF79EFE0546F0B10C9BAB60EC6001F0CC
:10BC100095FD41460446484601F0B0FAA41B241A9B
:10BC2000294601986C6101F0B5F901F0B3FA0120E1
:10BC300003B0BDE8F08F002003B0BDE8F08FB3463D
:10BC4000CCE700DE6BE700DEDEE700BF83DE1B43F0
:10BC50002DE9F04F85B006460D46914601F0E6FA13
:10BC6000C0B268B9FFF776F8002D00F0D780AF4872
:10BC7000294601F08FF905B0BDE8F04F01F08ABA0E
:10BC800001F0F4FA044601F0F5FB824601F0FCFBFA
:10BC900001F0D2FB074601F0B3FBE4B28046FFF7A8
:10BCA00059F8002C00F0B7800320FAF749FE04464B
:10BCB000002800F0B08090F8203003F00F03072B2D
:10BCC00040F0A98090F82130002B00F0A48090F87B
:10BCD0002310C94311F0010108D15FFA8AF2FF2352
:10BCE0003046FFF7C9FB002800F095800023FFB223
:10BCF0008DF80F3004F1200A002E00F0B88033795F
:10BD0000980640F1B480002D00F072812B7913F079
:10BD1000400240F0588194F822107F2940F2AA8016
:10BD20000DF10F030193FF23009311465346304654
:10BD3000FFF7ACFB002800F09C800420FAF700FE1F
:10BD4000002894D0962001F0B5FB484601F09CFAFB
:10BD500001F096FA0278032161F30302027094F86D
:10BD600020200178C2F3801262F3C7110C22017007
:10BD700042703279C9B2C2F3801262F38611024670
:10BD800002F8021BD6F81110C0F80210B6F8151010
:10BD90009180626A8260228D828101F0E5F901F072
:10BDA0003BFA002840F0678101F0C0FCFAF7E4FD9F
:10BDB00009232371002D00F047815D48A5602946C5
:10BDC00001F0E8F82B7943F040032B7101F048FCB7
:10BDD000206101F0B3FC41460546484601F0CEF92A
:10BDE0002D1A6561002F40F02B817F209DF80F30C8
:10BDF000627EA17E207643F0040322F00D0203F060
:10BE00000D0313436FF30001A1762068637621468A
:10BE1000FAF7D6FD87E0002D7FF429AF337CDF06EB
:10BE20001CD5FAF7A9FD0146002800F007810A2376
:10BE30000B718E60B3680868CB60FAF7C1FD337C84
:10BE4000DD060BD56FF304133A483374314601F025
:10BE5000A1F805B0BDE8F04F01F09CB9B1683348D6
:10BE600001F098F805B0BDE8F04F01F093B9002D4E
:10BE700064D02B79180611D4B16811B10879010684
:10BE80000CD40DF10F0300220193FF230093114600
:10BE900053463046FFF7FAFA0028BCD0A5602B794C
:10BEA000627EC3F3801363F3C30262762B7943F09F
:10BEB00080032B710023B360FAF75EFD01F0D0FB25
:10BEC000206101F03BFC41468346484601F056F9AB
:10BED000637EABEB000068F3410360616376002F83
:10BEE00052D17F20637E9DF80F20207623F005033A
:10BEF00002F0050213436376002D49D00E4B0095E6
:10BF0000424649465046FFF7FDFDA37E092260F3F5
:10BF10000003A376206822712146FAF751FDA37E23
:10BF2000DC0740F1A38005B0BDE8F08FC9B7000081
:10BF30000DB9000045B4000035B90000B36813B175
:10BF40001A79120610D40DF10F0300220193FF237A
:10BF50000093114653463046FFF798FA00283FF405
:10BF60005DAFB16800293ED0A660B368E3601B797D
:10BF7000627EC3F3801363F3C3026276B2681379FF
:10BF800043F08003137197E701F046FAC0B2A9E7C6
:10BF90003A4B0096424649465046FFF7B3FDA37E12
:10BFA000092260F30003A376206822712146FAF784
:10BFB00007FDA37ED80754D5337C43F010033374B8
:10BFC00005B0BDE8F08FB168002933D0087910F0D2
:10BFD00040022BD194F822007F283FF6A1AE1A062A
:10BFE0007FF54CAF5AE7337CDB063FF51AAF36E7F7
:10BFF000B368002BA7D01A795106A2D494F8222056
:10C000007F2A9DD90DF10F030193FF2300932A4648
:10C01000534629463046FFF739FA00288ED00420CF
:10C02000FAF78EFC00287FF48DAEF7E619067FF54F
:10C0300026AF33E71B067FF524AF2FE700DEF6E6D9
:10C0400001F0EAF9C0B2D1E6A660B368E3600C483B
:10C05000214600F09FFFB268137943F0400313714B
:10C06000B4E6084A138801331380E8E6054A1388CA
:10C0700001331380FBE500DE96E600BF35B9000012
:10C08000FDB80000F275002010B504460021FDF750
:10C09000C3FA6279214602F00702BDE81040FFF7BB
:10C0A000D7BD00BF034680681A7B037CDB0602D540
:10C0B0000021FFF7CDBD8168FFF7CABDC87800F049
:10C0C000010070472DE9F04F814685B0FEF74CFE28
:10C0D000D9F80CB0D9F808A09BF8027001257F09A7
:10C0E000BD40EDB289F80C509BF900309BF802403E
:10C0F000002B4FEA04249BF8013004F4F85444EA7E
:10C1000003049BF80030B5BF4FF496721E224FF423
:10C110009E784FF02E0813F0400F18BF32264C4B7C
:10C1200008BF4FF4FA7602FB04F40121284604FB11
:10C1300006F6A3FB063600F071FFAA0002F0FC022F
:10C14000FF21082000F0D6FF9BF8000000F03F0020
:10C15000FEF7C2FD09F1200001F000F83D4851460C
:10C1600000F018FF00210AF1400000F0D3FD017833
:10C1700011F001034FEA964602463DD1DAF860100D
:10C18000039339B12B2208680A71FAF70BFC039B61
:10C19000CAF8603001F024F9D9F81430012128469A
:10C1A0001C44FEF7CDFDA41B241AA4F110010020AD
:10C1B00001F02EFA0F3C8442814647D101212846E6
:10C1C000FEF7BEFDB0440346C14401212846994410
:10C1D00000F0D4FF012F81441FD0022F0CBF4FF479
:10C1E000BC702820484401F05BFA01F09FFA05B0CA
:10C1F000BDE8F04F01F006B94378C90803F01F030A
:10C2000001D09942C6D95046039200F0D7FD039A57
:10C2100028B101238AF86430BCE71820E2E79BF8D4
:10C2200002C0917892F800E09BF800304FEA5C1C65
:10C23000CDE9000C03F03F0301F07F010332CEF3A0
:10C24000410000F091FD0028A4D0E2E700DEB5E750
:10C2500083DE1B4341C800002DE9F04F90F8406099
:10C26000C6EB06130344904693F84220D40783B0EC
:10C2700069D540330F46DB7890F864105FFA86F991
:10C2800004463601D20803F01F0359BB0AB193429A
:10C2900059D2FDF7F9FF054600285ED0A6EB090349
:10C2A000234493F842A001F04FFC834601F07AFB4F
:10C2B00027222A71019001F041FCCAF3410A019B37
:10C2C00085F8200085F8238085F8243085F821B092
:10C2D00085F822A0A38AAC60013BEB84C7BB7F201A
:10C2E00028761AE06ABB256E6DB3272300272B71D1
:10C2F000FF2385F8207085F82330A38A013BEB8467
:10C3000001F050FB7F23C5E9024785F8240085F83A
:10C31000217085F822702B762766A6EB0906344437
:10C3200028682946FAF73EFB94F84330C3F3040229
:10C330000132002062F3040384F8433003B0BDE807
:10C34000F08F9342CFD36FF03C0003B0BDE8F08F85
:10C3500001F062F8C0B22876DFE700DE9EE700BF9A
:10C360002DE9F04F83B00E469DF830809DF8349053
:10C370009DF838A0002A63D0092905461F4669D0D8
:10C380000420FAF7DDFA044600285ED0FAF7F4FA42
:10C39000A37E2671A560EA6BE2606FF34103A3768A
:10C3A000B9F1000F67D17F20207601F059F92061A3
:10C3B00001F0C4F98346E87A394600F0070000F03E
:10C3C000DDFE7B00627E03F0020343EA0A1322F0E3
:10C3D000320203F032031343ABEB0000637660617B
:10C3E0002B7B627EC3F3400363F38612092E6276D1
:10C3F00004F1200A43D0FAF7BFFAE0600095E97A29
:10C400002A4B3A46504601F00701FFF77BFBA37E1B
:10C4100060F30003DA07A37640D52B7B43F00403D7
:10C420002B736FF00F0620682146FAF7BBFAB8F1BC
:10C43000000F35D1FAF7BCFA304603B0BDE8F08FF3
:10C44000B8F1000F01D009290DD10026304603B004
:10C45000BDE8F08F0320FAF773FA0446002895D15F
:10C460006FF00B06F2E701224946FFF7F5FE06469C
:10C470000028EAD1DEE700F0CFFFC0B294E70095D4
:10C48000E97A0A4B3A46504601F00701FFF73AFBBA
:10C49000A37E60F30003A376DB07C2D40026C2E7C5
:10C4A000002249462846FFF7D7FEC3E7C5C0000073
:10C4B000F8B50023C36306460C461746FAF774FB2B
:10C4C000054678B3AB7904F0010444EA870423F00D
:10C4D000050304F005041C43134BAC711B78AB80BF
:10C4E00003222A70BBB1F37A03F00703022B17D0A3
:10C4F000042B0CBF4FF4BC7328232B6101F0FEF812
:10C50000044601F00DF9241AAC600023726BEA6056
:10C510007363B36373733046BDE8F840FEF730BC15
:10C520001823EAE700DECDE7E083002010B50446DB
:10C53000FEF71AFC237B5A070AD4104B1978002205
:10C54000891A204618BF0121BDE81040FFF7B0BF8F
:10C550006FF382032373FAF70FFA014660B18B7E03
:10C560008C600A220A71E26B0868CA6043F0020319
:10C570008B76FAF725FAE0E700DEF0E7E0830020AB
:10C580002DE9F04385B0054600F050FE10F0FF04A1
:10C5900009D1FEF7DFFB00222146284605B0BDE8A1
:10C5A000F043FFF785BF00F061FEC4B200F044FF26
:10C5B000064600F025FF114B4FF0010983F800906B
:10C5C000074601F0C9FA8046FEF7C4FB01F08AF87D
:10C5D00001F08EF8F6B201F097F801F09BF8CDE982
:10C5E0000086CDF808903B4622460D212846FFF7ED
:10C5F000B7FE1030CFD105B0BDE8F083E083002056
:10C6000038B538B30C460546FEF7CCFC002828DBCD
:10C61000EA682B89D189138201330B44D38128899D
:10C62000936A116B00FB03330B44D16A8B4228BF22
:10C630000B461363FAF7B8FAA8B18379032123F004
:10C64000050300220170828083712046BDE83840D6
:10C65000FEF7FEBA054800F09DFCBDE8384000F04A
:10C6600099BD00DED4E700DEE7E700BF2DC500007E
:10C67000884207D038B504460D46FCF763FE18B172
:10C68000002038BD002070472046FCF7D7FF002867
:10C69000F6D12046FDF762FB40B16A7B437B9A42AC
:10C6A0000AD3FF2BECD001334373E9E72B7B1B0745
:10C6B000E6D46FF08B0038BD01326A73F9E700BF32
:10C6C0002DE9F04184B0054600F0B0FD10F0FF0404
:10C6D0000CD1FEF73FFB2B6E002B7BD100222146B5
:10C6E000284604B0BDE8F041FFF7E2BE00F0BEFD11
:10C6F000C4B200F0A1FE064600F082FEEA7A3B4991
:10C7000095F80CC0D1F84C34D1F84C14D208074637
:10C710000CF001082AD0DB0626D0100707D4C1F39D
:10C72000811101295ED0022959D0002954D0304B03
:10C7300001221A7001F010FAFEF70CFB00F0D2FF94
:10C7400000F0D6FF00F0E0FF00F0E4FFB8F1000FCA
:10C7500014BF022003202AD001222146284604B01B
:10C76000BDE8F041FFF7A4BE0F2AE0D8204B01221C
:10C770001A7001F0F1F98046FEF7ECFA00F0B2FF12
:10C7800000F0B6FFF6B200F0BFFF00F0C3FF019665
:10C790000026CDF800803B4622460C210296284612
:10C7A000FFF7DEFD103099D104B0BDE8F081FAF753
:10C7B000C7F806460028CFD0FAF7DEF8737E306857
:10C7C000B5600C2243F03003327173763146FAF7CC
:10C7D000F7F8C1E700DE81E7D107C7D5A7E7530720
:10C7E000C4D5A4E79207C1D5A1E700BF001000405F
:10C7F000E08300200146808AB1F812C091F824201D
:10C8000091F8253060449A4280B208D0B1F826C031
:10C81000A0EB0C0C1CF4004F02D181F824301A4616
:10C8200002EB420301EB43034FF0060C5B7F0CFB72
:10C83000021203F03F03C98A1832FDF7E3BD00BFBF
:10C840002DE9F043C66B85B00446002E00F09A80B7
:10C8500000F0ECFCC0B2002864D1FEF77BFAFAF7D6
:10C860008BF8014600283BD10D4688460F4600DE76
:10C8700000210A228B7E8C600A71E26B0868CA6014
:10C8800043F002038B76FAF78DF8002D00F08F80CD
:10C8900094F84030C3EB0313234493F84230D90794
:10C8A0002AD5256E45B3272300272B71FF2385F852
:10C8B000207085F82330A38A013BEB8401F072F8E5
:10C8C0007F2385F8240085F8217085F82270AC60FC
:10C8D0002B76EF60276628682946FAF763F80BE0A5
:10C8E0008B7E8C600A220A71E26B0868CA6043F092
:10C8F00002038B76FAF756F8FAF75AF8237B5A07B1
:10C900000AD56FF38203002201212046237305B06C
:10C91000BDE8F043FFF7CCBD304605B0BDE8F043BD
:10C92000FEF72EBA00F0A2FCC5B200F069FD814608
:10C9300000F082FDC7B201F00FF98046FEF70AFA57
:10C9400001220292CDE900874B462A460921204662
:10C95000FFF706FD10F1100F32D0B5B10028CDD091
:10C96000FAF70AF80146002881D08B7E8C600A22F3
:10C970000A71E26B0868CA6043F002038B76FAF72B
:10C9800011F885E7FEF7F0F969E7F9F7F5FF0146D9
:10C9900000283FF46CAF8B7E8C600A220A71E26B38
:10C9A0000868CA6043F002038B76F9F7FBFFB8F121
:10C9B000000FA1D0012239462046FFF74DFC9BE72E
:10C9C00005B0BDE8F08300BF2DE9F041C4680389DC
:10C9D000E589A78A23821D44ADB2002382B00646B2
:10C9E0006582E3812046FFF705FF0137BFB23D4472
:10C9F00080460146A5823046F4F7D6FE18B10020E5
:10CA000002B0BDE8F0810146054604F1400000F0A7
:10CA100081F9037813F00107064618D084F86450B2
:10CA2000204600F0CBF9E0B1012384F8643073783C
:10CA30006FF30403737000F0D3FC00F0E3FC1248C2
:10CA4000214600F0A7FA002002B0BDE8F081216E77
:10CA50000029F0D02B2308680B71F9F7A3FF276694
:10CA6000E9E7E27AB178357802F00702CDE9000211
:10CA7000434601F07F01C5F34100F21C00F074F958
:10CA80000028D4D0D0E700BF81C500002DE9F041D7
:10CA9000C4680389E589A78A23821D44ADB20023B7
:10CAA00082B006466582E3812046FFF7A3FE013788
:10CAB000BFB23D4480460146A5823046F4F774FE7D
:10CAC00018B1002002B0BDE8F0810146054604F12E
:10CAD000400000F01FF9037813F00107064618D054
:10CAE00084F86450204600F069F9F0B1012384F81D
:10CAF000643073786FF30403737000F071FC00F01E
:10CB000081FC1348214600F045FA002002B0BDE840
:10CB1000F081216E29B12B2308680B71F9F742FFD0
:10CB20002766002000F016FEE7E7E27AB178357854
:10CB300002F00702CDE90002434601F07F01C5F390
:10CB40004100F21C00F010F90028D2D0CEE700BF5F
:10CB5000C1C600000020704710B582B00446FEF741
:10CB600009FA002809DB084A08490948009400230B
:10CB7000FAF764F818B902B010BD00DEF3E77730B9
:10CB8000F9D000DEF7E700BF8DCA000001C6000043
:10CB900071C6000010B582B00446FEF7EBF900281C
:10CBA00009DB084A0849094800940023FAF746F8C7
:10CBB00018B902B010BD00DEF3E77730F9D000DE1F
:10CBC000F7E700BFC9C9000001C6000071C6000038
:10CBD000F0B5384B0D4683B000221A70044600F0C1
:10CBE00005FA6879012100F0070000F017FA6A7968
:10CBF00092000820FF2102F01C0200F07BFA0120C5
:10CC0000F9F79EFE002852D0203000F0A7FA201D30
:10CC100000F05CFA2389A17A40F25B6043EA0141AB
:10CC200000F018FB287900F03F00FEF755F8224885
:10CC3000214600F0AFF9002104F1400000F06AF84D
:10CC4000037813F0010706460FD0204600F0B6F82F
:10CC5000C8B1012384F8643073786FF304037370F0
:10CC600003B0BDE8F04000F0BBBB216E0029F7D057
:10CC70002B2308680B71F9F795FE276603B0BDE812
:10CC8000F04000F0ADBB6A792B79B178357802F0CD
:10CC90000702CDE9000203F03F0301F07F01C5F375
:10CCA0004100F21C00F060F80028D5D0D1E700DE8A
:10CCB000AAE700BFE083002041C8000008B500F0EB
:10CCC000A7FE002008BD00BF0020704700F0DEBEB8
:10CCD000027843789A425FFA82FC11D080F801C052
:10CCE0000278944504D05A1C4370D3B2022B0BD067
:10CCF0004FF0020C0F2212FB03C20B70104470475E
:10CD00000133DBB2022BF3D1022200230B7010445B
:10CD1000704700BF00B5027890F801E096451BD03F
:10CD2000D3B25A1CD2B2022A13D04FF00F0C4FF0DC
:10CD3000020E1CFB02EC027009B101220A70C3EB67
:10CD40000313034460449A786FF300029A705DF80D
:10CD500004FB94460022EEE702234FF00F0C1CFB6D
:10CD60000E3C60445DF804FB70B58446BCF1010FD5
:10CD70000D469DF810009DF8141014461E4616D05E
:10CD800000F0A2FE00F026FE00F0BAFE2046294682
:10CD900000F00AFE0120FDF75BFA044650B1522173
:10CDA000283000F0C3FE84F82560002070BD00F03C
:10CDB0006FFEE7E76FF00B0070BD00BF70B5044673
:10CDC000006E10B10025284670BD94F86450002D07
:10CDD000F8D10220FDF73CFA064630B1FDF754FACF
:10CDE0000023266684F86430EDE70120FDF730FA71
:10CDF000064610B16FF00B05F0E76FF06805E2E74B
:10CE00004FF080530246D3F8A410013107D04FF001
:10CE10008051D1F8A00010F0010009D17047D3F87B
:10CE2000A8304FF6FF719BB28B42F0D100207047C3
:10CE3000D1F8A4301360D1F8A8301371C3F30723DD
:10CE400063F03F035371D1F8903001331CD0D1F817
:10CE50009430013318D0D1F89830013314D0D1F880
:10CE60009C30013310D0D1F89030C2F80630D1F8A0
:10CE70009430C2F80A30D1F89830C2F80E30D1F8A8
:10CE80009C30C2F8123008E00023C2F80630C2F825
:10CE90000A30C2F80E30C2F812300120704700BFCD
:10CEA00000234FF08052036043608360C360D2F878
:10CEB0008030013318D0D2F88430013314D0D2F846
:10CEC0008830013310D0D2F88C3001330CD0D2F836
:10CED00080300B60D2F884304B60D2F888308B60A1
:10CEE000D2F88C30CB60704700230B604B608B60B6
:10CEF000CB607047054B4FF480320021C3F8081512
:10CF0000C3F84423C3F80423704700BF00B00040B7
:10CF1000054B1878421C1A7018B9044B01221A608C
:10CF200070470120704700BFE183002000B000403F
:10CF3000074B187848B10138C0B2187018B9054BC2
:10CF400001225A6070470120704700DE1878F2E72E
:10CF5000E183002000B00040014BD3F80405704786
:10CF600000B00040024B00F5A87043F82010704755
:10CF700000B00040044BD3F8103123B1034A044BF6
:10CF800010681B6818477047001000407874002034
:10CF90007C740020024A034B11601860704700BF88
:10CFA000787400207C7400204FF080434FF0FF32F3
:10CFB0000021C3F8002EC3F8042EC3F8081EC3F8DE
:10CFC0000C2EC3F8101EC3F8142EC3F8182EC3F885
:10CFD0001C2EC3F8202EC3F8242EC3F8282EC3F825
:10CFE0002C2EC3F8302EC3F8342E704708B5084BEA
:10CFF0000022C3F8182500F08BFD064B4FF490512A
:10D000004FF41052C3F80018C3F8042808BD00BF3D
:10D010000010004000F00140704700BF054B02289F
:10D020000CBF0421032140F20122C3F81015C3F8FC
:10D030005026704700100040072819DC831EDBB221
:10D04000052B11D9002818DA031D1BDA10F1080F7F
:10D050001ADA10F10C0F19DA10F1100F18DA10F1BA
:10D06000150FCCBFEC20D8200A4BC3F80C05704735
:10D07000084B0820C3F80C057047064B0020C3F886
:10D080000C057047FC20EFE7F820EDE7F420EBE714
:10D09000F020E9E700100040014BC3F80805704795
:10D0A00000100040084B00F07F00C3F85405D3F88F
:10D0B000182522F00072C3F81825D3F8182542F07D
:10D0C0000072C3F81825704700100040084A00217C
:10D0D0000123C2F82C15C2F83035C378C2F82435C4
:10D0E0008178038843EA01431B02C2F81C3570476C
:10D0F00000100040C2F3820302F0030CA3F102030C
:10D10000B3FA83F30CF1FF3CBCF1020F4FEA531367
:10D1100098BFC2F340124FEA036396BFD2040022C5
:10D1200043F48013134300F00F000A4A184340F4FD
:10D130008070C2F81405D2F81805074B0340C2F8F6
:10D140001835D2F81835194341F44031C2F8181592
:10D15000704700BF001000400000F8FE014BC3F80C
:10D160000405704700100040014BC3F804057047E8
:10D1700000100040012070472920704702280CBF92
:10D1800005200A20704700BF014B01225A607047FA
:10D19000001000400B4B0C480C4910B44FF41064C5
:10D1A000C3F8084501224FF480245A60DA60C0F8C1
:10D1B0004843074CC3F808450020C1F800020A6143
:10D1C00010BC704700F0014000B00040001000406B
:10D1D000C001700C0F4B0022C3F80021D3F80011DE
:10D1E000C3F80421D3F80411C3F80C21D3F80C11AF
:10D1F000C3F86C21D3F86C11C3F87021D3F8701107
:10D20000C3F82821D3F82811C3F81021D3F810311E
:10D21000704700BF00100040034BD3F800010038F6
:10D2200018BF0120704700BF00100040034BD3F827
:10D230000C01003818BF0120704700BF00100040EB
:10D24000034BD3F85005B0FA80F04009704700BF97
:10D2500000100040044B40F20312C3F83425C3F819
:10D260003805C3F83C15704700100040034BD3F855
:10D270000004003818BF0120704700BF00100040B4
:10D280000048704774730020F0B41D4B1D4D1E4ABA
:10D29000C3F800222A781D4E1D4C1E4FC6F8687533
:10D2A00002F10C03DBB2D000DB00910003F18043FC
:10D2B00000F1804003F5F83300F5F83001F18041CA
:10D2C000C6F86C0501F5104104EB82041248C3F85E
:10D2D0001045C3F81405D1F840352D2B8ABFD1F87D
:10D2E000403501232D3BC1F840350132074B4FF447
:10D2F000106102F00102C3F804152A70F0BC7047F7
:10D3000000100040E28300200100100000F0014006
:10D31000409100406C110040041000402DE9F041A4
:10D32000284E294B294CC6F800322178284FDFF8C7
:10D33000A4E0DFF8A480CEF8688501F10C03DBB22D
:10D34000DB00CD0003F1804303F5F83305F18045A0
:10D3500007EB810705F5F835CEF86C554FEA810CDF
:10D36000C3F8107549F63465C3F814654AF2B8136A
:10D37000022A18BF1D460CF1804C42F2B84241F21D
:10D380008833022818BF13460CF5104C134A2B445F
:10D39000A2FB0323DCF84025B2EB931F85BF98095D
:10D3A000DCF8403501231B1ACCF840350131094B1C
:10D3B0004FF4106201F00101C3F804252170BDE8AB
:10D3C000F08100BF0010004001001000E283002047
:10D3D0004091004000F001406C110040D34D6210BC
:10D3E0000449054B0548C1F800024FF41062C3F828
:10D3F000082570470010004000F0014001001000B7
:10D4000000207047034AD2F8003243F48873C2F810
:10D410000032704700100040014BD3F848057047B8
:10D4200000100040034B0022C3F81C21D3F81C312C
:10D43000704700BF00100040034BD3F81C010038B8
:10D4400018BF0120704700BF00100040034AD2F807
:10D45000403623F0FF03C2F840367047001000400A
:10D46000034B0022C3F81421D3F81431704700BFD6
:10D4700000100040034BD3F81401003818BF0120FE
:10D48000704700BF00100040014BD3F810047047F4
:10D49000001000400449054B054A4FF48020C1F8B4
:10D4A0004803C3F80825704700B0004000F0014071
:10D4B000C001700C034B044A1B7803F5A87342F8B3
:10D4C00023007047E283002000900040F0B4A2F5F2
:10D4D00074232F4DA3F51073AB42044606D902F115
:10D4E000E87202F5D432013902F5A572294B2A48B7
:10D4F0002A4D2B4E0127DF600027C3F80475A0FBDF
:10D5000002020427C3F81075900C0227C3F80875AF
:10D51000244AC3F84005C5F848154FF48021C5F8E2
:10D5200044134021C2F84065C2F84435C2F80415DE
:10D530004CB34FF48013C2F804351B4A0121002478
:10D540000423D160C2F80445C2F81035154BC2F867
:10D55000084511601549C3F850150C32C3F854251D
:10D5600002F5AF32124CC3F8584502F5FC7201F5D2
:10D57000FF41C3F85C2558310832C3F86015C3F881
:10D580006425F0BC70474FF40013C2F80435D4E7AB
:10D59000BFBDF07F0080004083DE1B4300B0004031
:10D5A00048B1004000F00140009000406C11004084
:10D5B00040910040134A30B40123134C53604FF4A0
:10D5C0008025D360C2F84035104BC4F84815C4F824
:10D5D0004453402104F5A474C3F84045C3F84425DE
:10D5E000C3F8041530B14FF48012C3F804250120AC
:10D5F00030BC70474FF40012C3F80425012030BC42
:10D60000704700BF0080004000B0004000F00140C3
:10D6100070B4114BD8B14FF48012C3F804250F4BEE
:10D620000A460026012502E0D3F840416CB9C1EB5F
:10D630004201C3F84061481CD3F84021C3F84005BB
:10D64000DD64D3F84C259142EED370BC70474FF4A3
:10D650000012C3F80425E2E700F00140008000401A
:10D66000014BD3F84805704700B000400349044A15
:10D6700001234B600B6153601361704700800040D1
:10D68000009000400449054BC1F844054FF0886202
:10D69000C3F80425704700BF0080004000F001403F
:10D6A0000449054BC1F844054FF08862C3F80425CE
:10D6B000704700BF0080004000F00140054B064865
:10D6C0000649074AC3F84805C3F84C15C3F80425B2
:10D6D000704700BF00F00140001100404080004052
:10D6E00080000004014BD3F84405704700800040DF
:10D6F000014B1860704700BF70730020014B186821
:10D70000704700BF70730020014BD3F8400570478D
:10D7100000800040014B1860704700BF6C73002010
:10D72000014B1868704700BF6C730020024B4FF02C
:10D730000062C3F80425704700F00140014BD3F8A4
:10D740004805704700800040014BD3F848057047FA
:10D75000008000400449054A42F61103002818BF22
:10D760000B46C2F8043970471928202000100040E9
:10D770000139012905D80B200AB1F5F729B8F5F7C9
:10D7800035B800DE704700BF29B10139012905D83D
:10D790000B20F5F73FB81820F5F73CB800DE002065
:10D7A000704700BF88420FD0012807D002280DD152
:10D7B000A1F10100B0FA80F040097047A1F1020028
:10D7C000B0FA80F040097047012070470020704790
:10D7D000012904D0022902D039B100DE7047064B7E
:10D7E0004FF40062C3F800217047034B4FF0807282
:10D7F000C3F80021704700BF00E100E0032803D810
:10D80000054B185C28B1704700DE034B185C0028FC
:10D81000F9D100DE704700BFD8300100013810B4E4
:10D820001C46042806D8DFE800F008111A2303007C
:10D8300004292FD000DE10BC70470429FAD1194BFF
:10D840009C6010BC02210020F7F7E4BA0329F1D153
:10D85000154B01219C6010BC0846F7F7DBBA042980
:10D86000E8D1124B9C6010BC02210120F7F7D2BA1C
:10D87000032908D00429DDD10D4B02219C6010BC86
:10D880000846F7F7C7BA0B4B9C6010BC0121022079
:10D89000F7F7C0BA084B9C6010BC02210320F7F7D1
:10D8A000B9BA00BF44030020340300202403002041
:10D8B0000403002014030020F4020020014600208D
:10D8C000FFF750BB124B30B40121044600205960D1
:10D8D000C3F80445C3F80001C3F80401196005E06A
:10D8E000D3F8042132B9D3F804251AB1D3F80021B2
:10D8F000002AF5D05960D3F80421002AE7D1D3F8E3
:10D900000455002DE3D0C3F8042530BC704700BF98
:10D9100000E0004070B5114C0126D4F80455666053
:10D920000E20F4F763FFD4F8040140B10021C4F8DD
:10D930000411D5E90E323046BDE870401847D4F8DE
:10D94000003143B1C4F80001D5E90E3205F12001E0
:10D95000BDE87040184700DE70BD00BF00E0004029
:10D9600070B58CB00E4615460146102268461C461E
:10D97000F7F7BCF910220DEB02003146F7F7B6F9C4
:10D980006846FFF79FFF25B1102208A92846F7F740
:10D99000ADF92CB108AD0FCD20606160A260E360ED
:10D9A0000CB070BD0020704710B4094C0023C4F8BF
:10D9B000283939B10346014413F8012BC4F828294A
:10D9C0008B42F9D1024B0278C3F8282910BC70476A
:10D9D0000010004030B40C490C4C00234FF00045BF
:10D9E00011F8012FFF2A08BF03F5137203F5137016
:10D9F00003F1010314BF44F8202044F82250082BFF
:10DA0000EED130BC704700BFDC3001000010004098
:10DA10001B4A70B502F108001A4D1B4E4FF0010C65
:10DA200011E08C0004F1A0444FF0A04ED4F8003770
:10DA30002B4043F00303C4F800370CFA01F1CEF891
:10DA40000C15824215D012F8013FFF2BF9D003F0DC
:10DA50001F015B09E5D0012B0CD18B0003F1A04322
:10DA6000B646D3F8004A2C4044F00304C3F8004AF9
:10DA7000E3E770BD01F5E071002353F82130FFDECC
:10DA8000DC300100F0F8FCFF000300500C20704770
:10DA90000B4B0C4AC3F81029012909D00229084A66
:10DAA0000CBF4FF470230023C2F81439FFF752BEA5
:10DAB000034A4FF48033C2F81439FFF74BBE00BF5E
:10DAC00000100040803202000B4B0C4AC3F81029B2
:10DAD000012909D00229084A0CBF4FF4A0130023E2
:10DAE000C2F81439FFF736BE034A4FF4C023C2F818
:10DAF0001439FFF72FBE00BF001000408031010035
:10DB0000024B0122C3F82C29704700BF00100040CF
:10DB1000054B00204FF420510122C3F80009C3F83F
:10DB20000419C3F82C29704700100040024BC3F8B9
:10DB30005009C3F85419704700100040014BD3F846
:10DB40005809704700100040024BD3F84C04C0B293
:10DB5000704700BF00100040034BD3F8700100383D
:10DB600018BF0120704700BF00100040084B70B57F
:10DB7000C31A0D4607499B100446594306484022E4
:10DB800003F0E8FD2B4601462046BDE870401847EB
:10DB9000C4740020B76DDBB64C2A010073B50C4C81
:10DBA0000C4A4023041B00930D460B460A49A4105F
:10DBB00061430646094803F0F9FD011E05DA3046C7
:10DBC0002B4602B0BDE87040184702B070BD00BFE0
:10DBD000C474002017180100B76DDBB64C2A010091
:10DBE0000022F8B5012105461046F4F721FE104841
:10DBF00001F0A8F80446B8B901F0C4F82F690D493E
:10DC0000384603F0F9F9031E09DB01263E642D694D
:10DC1000084905F11C0003F0EFF9031E02DA1C4667
:10DC20002046F8BDEE64FBE76FF00404F8E700BFA0
:10DC30006DDD0000E83001007FB500220123CDE951
:10DC4000022304ABCDE90433094ACDF800D06B467A
:10DC5000CDF804D003F0D8FD002805DB4FF4804256
:10DC60000023684601F066FD07B05DF804FB00BFC5
:10DC70002918010010B5EFF31184202383F31288D3
:10DC8000BFF36F8F074A136823F00201DB071160AF
:10DC900002D4012003F071FF84F31188BFF36F8F6A
:10DCA00010BD00BF1475002030B4104B0C2202FBD5
:10DCB000003301460020D3E90E529863EFF3118040
:10DCC000202484F31288BFF36F8F1C6C04F0C0040F
:10DCD00044F002041C6480F31188BFF36F8F1DB100
:10DCE0002B46034830BC184730BC7047C474002032
:10DCF0004C2A010010B4EFF31182202383F3128821
:10DD0000BFF36F8F1748016841F002040460C80731
:10DD100007D482F31188BFF36F8F012010BC03F08A
:10DD200024BF4FF08041D1F80C04D1F80C14C9077E
:10DD3000EFD5EFF3118083F31288BFF36F8F0A4999
:10DD40000B6C03F0C00343F002030B6480F31188F3
:10DD5000BFF36F8F82F31188BFF36F8F002010BC69
:10DD6000FFF7A2BF14750020C474002010B1012871
:10DD700004D07047034B1B6C5B0701D1FFF794BFC6
:10DD8000704700BFC4740020024AC3B21C2003FBCA
:10DD900000207047C4740020094BBFF35B8F53E829
:10DDA000002F42F0010143E800100028F7D1BFF333
:10DDB0005B8F930702D4012003F0D7BE704700BFEA
:10DDC0001475002010B5EFF31184202383F312881B
:10DDD000BFF36F8F074A136823F001019B0711609F
:10DDE00002D4012003F0C9FE84F31188BFF36F8FC2
:10DDF00010BD00BF147500202DE9F0413849BFF374
:10DE00005B8F0746012251E8003F41E800200028CF
:10DE1000F9D1BFF35B8F33B9324933484B60CB60E4
:10DE20008A6003F0FCF87B1E012B2BD8012F07D151
:10DE30004FF08043D3F81C3403F00303012B21D0AF
:10DE400004F048FB0546F8B9284B1B78E3B14FF0C6
:10DE500080430222C3F808230646DFF894804FF07F
:10DE60008044D4F81824D4F81834D20315D503F01C
:10DE70000303012B01D0012F0FD155B386F3118875
:10DE8000BFF36F8FBDE8F081EFF31186202383F39A
:10DE90001288BFF36F8F0125DFE7ADB1304603F085
:10DEA000ACF9D4F81835002BDBD1D4F80421002AC2
:10DEB000D7D0C4F80431D4F804310123C4F818359C
:10DEC000C8F88031A360CCE70021212004F09FFB3B
:10DED000E7E74FF080430222C3F80423D2E700BFF4
:10DEE000C0740020B0740020E0740020E58300209E
:10DEF00000E100E008B5074804F06FF938B10648C2
:10DF0000F4F7B8FE0448F3F7A9FF002008BD6FF04E
:10DF10001200FBE7BC2A01001DDF00000A2838B50B
:10DF2000074D044604D1AB680D215B68284698472D
:10DF3000AB6803485B68E1B29847204638BD00BF34
:10DF4000BC2A0100EFF31182202383F31288BFF370
:10DF50006F8F0A4BD3F8001161B10021D3F8080587
:10DF6000C3F80011D3F80031C0B282F31188BFF3B7
:10DF70006F8F70476FF00A00F7E700BF00D00040D6
:10DF8000F0B5034610469C7893F803C0EFF3118276
:10DF9000202585F31288BFF36F8F1F7893F801E077
:10DFA000E41B04EA0C04A04288BFA0B23E180CEAAD
:10DFB00006063D461E7082F31188BFF36F8F0A1864
:10DFC0008A4216D177450CD1EFF31182202181F3DB
:10DFD0001288BFF36F8F1978597082F31188BFF3DD
:10DFE0006F8F1B79241AA34222BF064B01221A60AD
:10DFF000F0BD5E190135767901F8016B05EA0C0573
:10E00000DEE700BF00D00040DB432DE9F04713F00E
:10E0100001050E46144604D02248FFF7B1FFBDE8C3
:10E02000F0879AB3EFF31188202383F31288BFF3AC
:10E030006F8F0D20F4F7EEFB07460D20F4F7D6FBAB
:10E0400088F31188BFF36F8FDFF85CA0DFF85C8086
:10E05000CAF80051DAF800314FF400590123CAF828
:10E0600000302546C8F88091DAF8003183B1FFF717
:10E0700069FF031EC8F88091F6DB013DADB2735510
:10E08000002DF1D117B10D20F4F7A2FB2046C6E711
:10E09000EFF31180202383F31288BFF36F8F03F017
:10E0A000ACF8E1E74875002000D0004000E100E056
:10E0B0002DE9F041124F0D46144607F1450814B9F9
:10E0C0002046BDE8F0814FF0FF334FF0FF32384675
:10E0D00001F030FB224629464046FFF751FF064635
:10E0E000384601F0EDFA3EB94FF0FF324FF0FF3302
:10E0F000044801F01FFBE6E7A41BA4B23544DEE7A9
:10E10000187500203075002038B5194C01221146D1
:10E11000204604F094F90122002104F1180004F0D3
:10E120008EF940F20743A4F848304FF07063236340
:10E130000C2384F8343000250E4B84F84550A4F8A5
:10E140004650D3F8042542F00102C3F8042501210A
:10E15000C3F80051D3F80021C3F804132A4619600C
:10E160000D20F4F765FB0D20F4F732FB284638BD8F
:10E170001875002000D0004010B5FFF7E3FE00281E
:10E1800020DB174B93F8322093F8314093F833108B
:10E19000141B31EA0404C0B20DD193F8472093F860
:10E1A000464093F84810141B31EA04040BD10D4B80
:10E1B00001225A600EE09C180132114084F83500AB
:10E1C00083F8321010BD9C180132114084F84A00C7
:10E1D00083F847100448BDE8104001F071BA00BF51
:10E1E0001875002000D0004030750020F0B544685C
:10E1F0001646A068227C01F01F0587B045EA42154B
:10E2000000286DD0B6F5001F04D1294603F0C7FFE2
:10E21000002056E06268607CC2F8240501AA002054
:10E22000B6F5800F0190506037D1B3F1007F14BF75
:10E23000052304238DF804300023CDE90423039340
:10E24000E36823FA01F111F001010DF103073AD15E
:10E25000B6F1A07F37D105F01F036A0903F5E0731B
:10E2600026D0012A3FD1214A52F82330DB072AD495
:10E27000A0683A46294603F008FF16301BD00297E3
:10E28000A06803AA294603F0CCFD002819DBA0688A
:10E290000122294603F030FFBAE7B3F1C06F05D081
:10E2A000B3F1007F14BF01230223C3E70323C1E7B7
:10E2B0004FF0A042D8E7A068394600F0CFFE002812
:10E2C000DDDA07B0F0BDA0683A46294603F0DDFE6E
:10E2D0000028D5D19DF80310A06800F0B9FECFE763
:10E2E0006FF08500EDE751F82330FFDE00030050AA
:10E2F000420970B5034602D0012A17D070BD0D4EF9
:10E30000326951680029F9D003F01F0301250C6818
:10E310009D400029F2D08A682A4002D04B683046DE
:10E3200098472CB1236821461C46F2E7024EE7E7E6
:10E330002346F8E7842A0100682A010038B54568B9
:10E34000A86890B103F0D0FE014670B9A86803F048
:10E35000AFFE044658B902460649A86803F092FE8B
:10E36000224605210620F4F763FA002038BD6FF03D
:10E370000400FBE7F1E200002DE9F043476840F2BA
:10E380000636D0063B7C87B002EA060654BFC2F3CD
:10E39000401C4FF0030C01F01F05B6F5837F1446B7
:10E3A00045EA43158DF803C045D00DD8062E16D08A
:10E3B00005D8A6B1022E40D06FF0150038E0B6F5B2
:10E3C000807FF9D101260AE040F20222964236D03F
:10E3D000B6F5407F35D0B6F5007FEDD1022601239A
:10E3E000220303FA01F12ED57B68C3F80815B8683B
:10E3F00090BB05F01F036D092BD0012D75D13D4A4F
:10E4000002EB830284F48033D2F80017C3F3004395
:10E41000C4F3404444EA430421F4E16144EA8C0437
:10E4200021F0070144EA06230B43C2F8003700201D
:10E4300007B0BDE8F0830726D1E70426CFE705261D
:10E44000CDE70326CBE7630344BF7B68C3F80C1515
:10E45000CDE74FF0A042D3E70DF10202294603F0C9
:10E4600014FE14F4403F80460CD1B868294603F0EE
:10E4700041FEB8F1000FDAD19DF80210B86800F043
:10E48000E7FDD4E74FF0000901ABCDE90199CDE9F3
:10E490000439CDF80C90B86803AA294603F0C1FCF2
:10E4A0004845C4DB14F4003314D084F480349DF860
:10E4B00003308DF80E30C4F300448DF80C608DF8F5
:10E4C0000D40B8684B4603AA294603F062FD0028B8
:10E4D000CFDAACE7CDE904330DF103030393B86859
:10E4E00003AA294603F09DFCF1E703F5E07350F819
:10E4F0002330FFDE00030050036803F01F025B09B6
:10E50000026004D0012B034818BF002070474FF071
:10E51000A0407047000300502DE9F04FDFF88491D0
:10E52000DFF884A185B01546834600EB810140F2F7
:10E53000FF18594503D1002005B0BDE8F08FDBF886
:10E5400000305E04C3F3C322C3F3080400F1A380C8
:10E55000444519F802704FEA136312D0192B1ED9E3
:10E560004E2B40F09B80C5F8144503A80394FFF799
:10E57000C3FF039B012606FA03F3C0F808353246B1
:10E580004EE0192B09D94E2B40F088804FF0FF3315
:10E59000C5F814350BF1040BCBE74FF0FF34192B02
:10E5A0007CD8DFE803F00D1218311B21317B7B7B17
:10E5B0007B34617B7B7B7B7B7B7B7B7B646F72753E
:10E5C000C5F80C45601CD0D1E4E7C5F81445661CBD
:10E5D000E0D00026D3E7C5F80845F3E7621CC5F88C
:10E5E0000845D7D0002604E0631CC5F80C45D1D0FF
:10E5F000012603A80394FFF77FFF039B012202FA81
:10E6000003F3C0F80C350BE0C5F81045DFE7C5F89B
:10E610000845002FDBD1601CBCD0002632460627FF
:10E62000DBF80030019303F40040002818BF0022FB
:10E6300003A8009218BF01260394FFF75DFF039C17
:10E64000019B009A00EB8400C3F3412CD0F80047F3
:10E650003B0243EA8C03134304EA0A04234343EADC
:10E660004603C0F8003795E7C5F80C45D1E7C5F873
:10E670006045621CDBF800308CD0C3F30043002BF4
:10E68000B6D072E7C5F86445F3E7C5F86845F0E72A
:10E69000C5F86C45EDE76FF015004DE76FF08500AC
:10E6A0004AE700BF9A3C0100F0F8FCFF2DE9F04179
:10E6B000044647680D4603F00DFF88B14FF020086F
:10E6C000EFF31186314688F31288BFF36F8F6068CD
:10E6D00003F035F950BB86F31188BFF36F8FEFE776
:10E6E0001F4B1B78002BE9D04FF020086426606890
:10E6F00003F025F970B9012003F0E4F9013EF6D1E9
:10E700000021212003F083FFF0E786F31188BFF397
:10E710006F8FF5E7EFF31186314688F31288BFF368
:10E720006F8F606803F00BF90028EED0FB691D7055
:10E730006368FA691B680020C3F844250122C3F806
:10E740004825C3F82001D3F82041C3F85801D3F875
:10E7500058019A6081F31188BFF36F8FBDE8F08193
:10E76000E583002070B5012383400E4ABFF35B8F21
:10E77000DC4352E8001F01EA040542E80056002E7F
:10E78000F7D1BFF35B8F4FF4803282400648C0F868
:10E790000823BFF35F8FBFF36F8F0B4214BF0120BD
:10E7A000002070BD947500200010014070B40E4927
:10E7B000D1E90034D01AC31844F1000422F07F4696
:10E7C000C1E90034A6F50013B3F5400F09D2074B99
:10E7D0001B681A0A1B069C19054B42F10005C3E988
:10E7E000004570BC01F066BEE80700209875002067
:10E7F000F007002011B3BFF35B8F0123104A834061
:10E8000052E800CF4CEA030C42E800C10029F7D1DE
:10E81000BFF35B8F0B4A4FF480338340C2F804335D
:10E82000094BBFF35B8F1B68BFF35B8FC340DB07F4
:10E8300042BF064B4FF40032C3F80021704700BFBF
:10E8400094750020001001409075002000E100E068
:10E850000D4B1868010A0006BFF35F8F0B4BD3F80E
:10E860000435181841F10001B3F5801F0AD2084B96
:10E87000D3E90023904271EB030303D210F18070BF
:10E8800041F10001704700BF987500200010014061
:10E89000F00700202DE9F04F85B016461F469DF881
:10E8A00040A00446FFF75EFF0190FFF7D1FFB042A2
:10E8B00071EB070354D23E4B301A67EB01019842CB
:10E8C00071F100014FD23B4B03EB0413D3E9022358
:10E8D0009F4208BF96425ED037494FF4803804F11A
:10E8E000500508FA04F8AD00C1F848832046ADB2DF
:10E8F00003F0D9F826F07F4B05F1804504F5A873A5
:10E9000005F58835DC464FF003090293029A2CF096
:10E910007F4341F82230C1F84483D1F80435274AB7
:10E920006FF00200C01A604420F07F40904232D95C
:10E93000286868B1D1F804350393A3EB0B0020F0ED
:10E940007F40B0F5000F26D9204603F0ACF8039BBA
:10E95000BAF1000F07D109EB030C09F10109D5E762
:10E96000BAF1000F09D06FF0150520460199FFF7A5
:10E9700041FF284605B0BDE8F08F0123104ABFF3E0
:10E980005B8FA34052E8000F184342E800010029C2
:10E99000F8D1BFF35B8F07490E98230101EB0412F6
:10E9A000C8500F9B5360C2E902670025DDE700BF36
:10E9B00001008000D807002000100140FDFF7F000B
:10E9C000907500207FB51C4C1C4BC4F80833C4F86C
:10E9D00048331B4B00254FF0FF304FF0FF31C4F898
:10E9E0000855C3E902014FF48033C4F80433154BD2
:10E9F00002264FF400320121C4F804631120C3F849
:10EA000080212A46F3F714FF1120F3F7E1FE0E4AA6
:10EA10000123A360236013600C4B0D4A0093CDE9E2
:10EA2000015500232846FFF735FF3046FFF7E4F98C
:10EA3000284604B070BD00BF0010014003000F0065
:10EA4000D807002000E100E094750020ADE7000049
:10EA5000FFFF7F002DE9F7432F4CD4F804339907CB
:10EA60000BD5D4F8043143B12C4A0023C4F8043147
:10EA7000D4F80431136801331360D4F80433DA0393
:10EA800029D5BFF35B8F264B53E8002F22F00101FD
:10EA900043E800100028F7D1BFF35B8FD30702D4FF
:10EAA000D4F84031BBB10025C4F84051D4F840310E
:10EAB000FFF7CEFEEFF31182202383F31288BFF31A
:10EAC0006F8F184BD3E90267B042B94106D282F387
:10EAD0001188BFF36F8F03B0BDE8F0834FF0FF38AC
:10EAE0004FF0FF39C3E90289D3E900101D604FF4EC
:10EAF0008033C4F84833C4F84051D4F8403182F32D
:10EB00001188BFF36F8F0029E5D0009032463B4655
:10EB100028468847DFE700BF0010014098750020B5
:10EB200090750020D807002030B5431C124C85B0EA
:10EB300005D08442A8BF0446012CB8BF0124FFF7CA
:10EB400087FE0E4B0C4DD3E90013401AB0F5000FB1
:10EB500010D22218AA4228BF2A4652184FF00000AD
:10EB600007490091CDE9010043F10003FFF792FE50
:10EB700005B030BD2A46F0E7FFFF7F00E807002020
:10EB8000ADE7000008B5FFF763FE024B1B68C01A33
:10EB900008BD00BFE8070020024AD2F80034002B6D
:10EBA000FBD0704700E0014010B54FF08053D3F820
:10EBB00030210D2A55D14FF080410022C1F80C219F
:10EBC000C1F81021C1F83825464AD3F80404C2F828
:10EBD0002005D3F80804C2F82405D3F80C04C2F8C1
:10EBE0002805D3F81004C2F82C05D3F81404C2F891
:10EBF0003005D3F81804C2F83405D3F81C04C2F861
:10EC00004005D3F82004C2F84405D3F82404C2F820
:10EC10004805D3F82804C2F84C05D3F82C04C2F8F0
:10EC20005005D3F83004C2F85405D3F83404C2F8C0
:10EC30006005D3F83804C2F86405D3F83C04C2F880
:10EC40006805D3F84004C2F86C05D3F84434C2F820
:10EC50007035D1F80034DB0709D56FF00103C1F836
:10EC600000344FF08053D3F830310D2B0CD14FF0DE
:10EC70008053D3F834313BB14FF01023D3F808223E
:10EC80004FF08043C3F858254FF01023D3F80022EB
:10EC9000002A03DBD3F80432002B22DA12490123C5
:10ECA0004FF01020C1F804351224FFF775FFC0F8AB
:10ECB0000042FFF771FFC0F80442FFF76DFF002329
:10ECC000C1F80435FFF768FFBFF34F8F0749084BC2
:10ECD000CA6802F4E0621343CB60BFF34F8F00BFFA
:10ECE000FDE710BD00C0004000E0014000ED00E085
:10ECF0000400FA05014B1860704700BF9C750020A6
:10ED000010B5054B1868144602F0DEFE0028A4BFBB
:10ED10002070002010BD00BF9C750020024A012316
:10ED20008340C2F80435704700F00140014B0020D9
:10ED30001B681847A0750020014B1B68184700BFCF
:10ED4000A075002010B50C4C237993B901232371D1
:10ED50000A4B2060002818BF184600F023F850B96D
:10ED600023680748002BBDE8104008BF184600F094
:10ED70005BB86FF0770010BDA07500202DED00008E
:10ED800039ED000008B5064B1B683BB10020F3F7D6
:10ED900041FD18B9BDE80840F3F71ABD08BD00BF32
:10EDA000A0750020054B0246187918B91A60012297
:10EDB0001A7170476FF07700704700BFA875002088
:10EDC0004FF080430022C3F80021D3F80021094905
:10EDD00001221A60096811B1C3F804237047D3F8FF
:10EDE0000021002AFBD00022C3F80021D3F8003113
:10EDF000704700BFA87500204FF08043D3F804236C
:10EE0000D2070DD5D3F8002152B10022C3F800215A
:10EE1000D3F800210122C3F80823024B1B681847CE
:10EE2000704700BFA8750020074A137943B9012134
:10EE3000106011714FF080421846C2F818357047C3
:10EE40006FF07700704700BFB075002010B54FF02D
:10EE500080431D4CD3F81814D3F8182411F4803FC4
:10EE600019D002F00302012A03D00AB102F0B2FE67
:10EE700000224FF08043C3F818250022C3F8042174
:10EE8000D3F8042101229A60226872B9D3F80421D0
:10EE9000002AFBD011E0D3F81424D107E8D5D3F829
:10EEA0001C249207E2D422681AB10222C3F8042378
:10EEB00010BDD3F80421002AFBD00022C3F804219E
:10EEC000D3F80431F4E700BFB0750020F8B54FF077
:10EED0008043194FD3F80443012504F01A04002697
:10EEE00004B9F8BDB4FA84F0C0F11F00830003F543
:10EEF00080739BB203F1804305FA00F2196824EA9B
:10EF000002040029ECD01E601B684FF080430128EA
:10EF1000C3F808230CD1D3F81824D3F81824920787
:10EF200006D10222C3F81805C3F804239860D7E776
:10EF30003B68C0B29847D3E7B0750020036803F080
:10EF40001F025B09026004D0012B034818BF002098
:10EF500070474FF0A040704700030050034A430938
:10EF600000F01F00D35C1844C0B27047B03C0100F1
:10EF7000034611F0010030B5CCB213D1A207C4F39F
:10EF8000400020D5124AD2F8200558604FF0805337
:10EF9000C2F82005D3F830310D2B15D0003818BF3A
:10EFA000012010E04FF0A0414FF08055D1F820250E
:10EFB0001A60C1F82025D5F830510D2D08BFD1F8C1
:10EFC0002015002ADAD030BDD2F82035E6E700BFA0
:10EFD00000030050F7B504460846FFF7BFFF06B22E
:10EFE00004EB46060D46B38ADB072BD5204602F01C
:10EFF000F5FE2946204602F060FE58B1204602F098
:10F0000072FE276800B207EB80030022C3F81025C8
:10F01000C3F810252946204602F08EFE0021B18259
:10F0200001A80195FFF78AFF019B00EB8300074BC6
:10F03000D0F80027134043F00203C0F80037084619
:10F0400003B0F0BD6FF01500FAE700BFF0F8FCFF69
:10F05000014802F057BD00BF5803002010B5044816
:10F060000C4602F031FD0028A4BF2070002010BD26
:10F07000580300202DE9F04F804689B058F804ABC2
:10F08000DAF80413C9B28346082241F00041504621
:10F0900002F07CFE051E2BDA0023032106A8CDE931
:10F0A0000633FFF765FF644B01930DF11809002348
:10F0B000019A009312F8013B60490192DA0803F0CB
:10F0C00007038A5C22FA03F3DA071AD4009B09F1DA
:10F0D0000409A3B14FF000410022504602F056FE51
:10F0E000032106A8FFF744FF0028DCD125F00045E6
:10F0F0000124002D40F08A8009B0BDE8F08F012383
:10F10000D6E7009B4E4A13440293D9F80010002919
:10F11000DCD0029B91FAA1F11C78B1FA81F141EAAD
:10F1200044142046FFF71AFF0BEB40000594878A32
:10F13000C808BB0819F80020039301F00701012358
:10F1400003FA01F122EA010209F8002005A8FFF7FD
:10F15000F5FE059A039B02F5E072C7F3820650F8AC
:10F1600022205B073746C2F3014233D5D6B2404670
:10F170003A46214602F0C1FD05A80594FFF7DEFEE0
:10F18000059B03F5E07350F82330C3F301439E421F
:10F1900007D10021204602F081FD3146204602F0D1
:10F1A0007DFD05A80594FFF7C9FE059B012202FA23
:10F1B00003F3C0F820354FF08053D3F830310D2BD6
:10F1C00001BFD0F82035D0F82035D0F82035D0F860
:10F1D00020359AE7022A0DD10321204602F05EFD78
:10F1E00006F00503012BDCD13A462146404602F0E9
:10F1F00084FDD6E702212046039202F04FFD032E44
:10F20000F2D0039A032ACCD1022EECE795FAA5F3AB
:10F21000B3FA83F304FA03F225EA020503F5A272B6
:10F220000BEB43035AF82220B3F87010C2F30142EB
:10F23000404602F062FD5CE7C03C0100783101000D
:10F24000C03C010038B5EFF31185202383F3128809
:10F25000BFF36F8F064B9C6802F0D2FF85F31188D5
:10F26000BFF36F8F2046BDE83840F3F757BA00BFB1
:10F27000B875002038B50A4B53F82040013053F8D8
:10F280002050A54200D838BD606830B1037EDB074E
:10F2900001D402F08AFF0834F3E723689847FAE7BD
:10F2A0007C31010070B52A4B2A4C2B4D012286B0CF
:10F2B00003201A70FFF7DEFF03F0DFFA0420FFF7E8
:10F2C000D9FF2646AE4204F1300410D300F0E6FD2B
:10F2D000204C224EAC4226D300F0F4FDF2F792FC13
:10F2E0001F4A137B23F00103137306B070BD54F85B
:10F2F0000C3C059354F8103C049354F8143C0393CD
:10F3000054F8183C029354F81C3C019354F8203CE8
:10F31000009354E90A2354E90C0100F089FB54F8E6
:10F32000303C5E65CDE7D4E90A23B3F1FF3F08BF67
:10F33000B2F1FF3F05D052EA0301206803D100F08B
:10F340007DFE3034C6E73146183001F023F8F8E787
:10F35000E5830020742C0100742C0100CF250100EE
:10F36000B008002070B5174E174D184986B0B82365
:10F3700003FB0066164B059301220F23CDE90332F0
:10F380000023CDE90133142303FB005504464FF459
:10F39000C07000FB04110F4B00954FF4A072304673
:10F3A00000F046FB737B0C4AEE6023F0040373739A
:10F3B0004FF4046304FB033313442C746B6006B0F6
:10F3C00070BD00BFF8070020B8750020409B0020EA
:10F3D000C23C01004F22010000930020BFB5002075
:10F3E000FFF748FF284B83F30888284C284F6369B0
:10F3F00043F4007363610025E02384F82230E5774D
:10F4000025766576A57684F82050636A43F4E02378
:10F41000636284F82350F3F7F7F8F3F797FA4FF0A5
:10F42000FF33A362E362F3F759FBF3F7B3FA19482A
:10F43000194C00F09FFB0120FFF71CFF0220FFF793
:10F4400019FF00F073FD154B15495C61154B0593D1
:10F450000123CDE903534FF480623B46CDE90155CA
:10F460000095204600F0E4FA627B064622F0040292
:10F470002046627303F06EF82846FFF773FF3A46A2
:10F4800031462046F3F742FA409B002000ED00E0B1
:10F49000A5F2000068090020B0080020B87500201F
:10F4A000C09C0020C73C010038B5064C064DAC425C
:10F4B00001D3002038BDD4E90112204602F0A3FE9A
:10F4C0001434F4E774030020740300202DE9F341A1
:10F4D000044617461E46EFF31188202383F3128853
:10F4E000BFF36F8FC368334A7BB1806891688842ED
:10F4F00019D057EA060318D188F31188BFF36F8F2C
:10F500006FF00F0002B0BDE8F081916891F90E1024
:10F5100021610133E3609368A36088F31188BFF32E
:10F520006F8F0020EEE72169F2E791F90E1090F954
:10F530000E309942A8BF19466FF07E029142B8BFC3
:10F5400011468B422DDD02F08DFE0546CDE9007699
:10F5500019482246414600F0E7FB0028E1D0EFF3CE
:10F560001186202383F31288BFF36F8FA068D0B178
:10F57000236821699C420AD04BB193F90E3099421D
:10F58000A8BF19466FF07E039942B8BF194602F032
:10F5900069FE40B10848314600F05AFC6FF00A009D
:10F5A000B0E70025D2E7002DF4D186F31188BFF330
:10F5B0006F8FF3E7B8750020E6830020F8B5836805
:10F5C0000546002B40D0234A926893423FD1C3683E
:10F5D000012B03D9013BC3600020F8BDEFF3118775
:10F5E000202383F31288BFF36F8F0169806802F0D4
:10F5F00039FE2C68A54207D10023C5E9023387F301
:10F600001188BFF36F8FE7E7002CF5D0D4E9003203
:10F6100013605A60637B002623F002036373C4E91E
:10F620000066A66004F1180003F04CF8AC6094F991
:10F630000E302B612046C4F8B06002F08BFF064804
:10F64000394600F005FCC7E76FF01500C5E74FF03D
:10F65000FF30C2E7B8750020E683002037B51146B9
:10F66000EFF31185202282F31288BFF36F8F0468B5
:10F670009CB12368426823F003039442036008BFEF
:10F6800043600121204602F07AFE044685F311888A
:10F69000BFF36F8F204603B030BD51EA0302F5D0AF
:10F6A00000F10802CDE900131046294600F03CFBAA
:10F6B0000028EFD1014B9B681C69EBE7B87500206F
:10F6C00070B5EFF31186202383F31288BFF36F8F99
:10F6D0000468A0421BD0D4B1D4E9003213605A6050
:10F6E000637B002523F00203C4E900556373A56022
:10F6F00004F1180002F0E6FFC4F8B050204602F012
:10F7000029FF31460A48BDE8704000F0A1BBD0E9AE
:10F7100002329A4218BF013383600221103003F095
:10F7200086F80028EDD186F31188BFF36F8F70BD86
:10F73000E683002013B5EFF31181202484F31288AF
:10F74000BFF36F8F846844B1013C846081F31188FA
:10F75000BFF36F8F002002B010BD52EA030406D140
:10F7600081F31188BFF36F8F6FF00F00F3E7CDE9DE
:10F7700000230246014800F0D7FAECE7E6830020B8
:10F780002DE9FF414F4E04462027EFF3118887F300
:10F790001288BFF36F8FD4F8BC50F5B9022104F181
:10F7A000D40002F05CFE002868D004F1CC050022F1
:10F7B0000121284602F04CFF0028F8D100230293D3
:10F7C0004FF0FF324FF0FF33CDE90023414604F103
:10F7D000C4023D4800F0FEFCD7E7D4F8C0202B68F7
:10F7E000C4F8BC30954208BFC4F8C030D4F8D43057
:10F7F00043F00203C4F8D430EB6823F0040343F071
:10F800000103EB606B6888F31188BFF36F8F2846A4
:10F810009847EFF3118887F31288BFF36F8FEB6877
:10F82000D80623F0010236D4EA60EB689A0716D5B1
:10F83000306823F00203EB6088B10368002170B1E7
:10F840004268954235D1036869BB72683360824271
:10F8500000D17360002340F8083BFFF731FFD4F874
:10F86000D43023F00203C4F8D43088F31188BFF3F6
:10F870006F8FDB0589D400F061FB86E7D4F8D430C4
:10F88000D9069BD5C4F8D40088F31188BFF36F8FD5
:10F8900004B0BDE8F08123F01103EB6005F1100026
:10F8A000FFF70EFFC1E70B607368834208BF71600A
:10F8B000D0E723B11A68014618461346BFE71A4637
:10F8C000F9E700BFDC750020E6830020F8B5C368C7
:10F8D0009A0704460F46C3F340062ED45B071CD498
:10F8E0000B680BB983680B60E368DD0744BFA3684E
:10F8F0003B603D684CBF02260126002D3CD0204BCA
:10F900009A68D5F8B8309A420AD0D5F8D430D807DA
:10F91000C3F3800214D46FF0120600233B6025E08D
:10F9200002F0D8FDD5F8D4300028F0D1D907C3F3C0
:10F93000C002F0D552B15B0708D46FF00F06ECE7B8
:10F94000002AFAD1C3F3C003002BF6D100232360B1
:10F95000D5F8C03063B9C5E92F44284602F08AFDC6
:10F96000E36843F00403E3603B68A3603046F8BDFE
:10F970001C60C5F8C040F0E76FF01506CDE700BF8A
:10F98000B87500200146014802F08EBD400A0020F3
:10F99000F0B589B004460020C4E92F000E9D04F1A3
:10F9A000C400C4E9310004F1CC00C4E9330055B30C
:10F9B0002879002840F2011008BF0120C4F8D400C3
:10F9C00000204FF0FF364FF0FF37CDE90330CDE98F
:10F9D0000100CDE906670D4B0094204600F09EF82B
:10F9E00055B1296811B1204600F012F86B791BB1AE
:10F9F000237B43F001032373204600F01FFBC4F870
:10FA0000B84009B0F0BD0120D8E700BF81F7000081
:10FA100010B5044608B9054B9C681F2204F1780014
:10FA200002F052FF002084F8970010BDB875002046
:10FA30002DE9F04F073285B022F0070204461E463A
:10FA40007F3200F15803C0E9163322F03F02129BC7
:10FA5000237300200D46119BDDF838A0139FA06092
:10FA600004213F2AC4E906006173A373E07305F122
:10FA70004009A2F1400B05D880F31188BFF36F8FC6
:10FA8000084602DF05EB020841462046F2F79CFBE0
:10FA90000730109B20F00700C4E9269BC4F8A000A3
:10FAA00002930F9BA8EB000BCDE900A35A46334607
:10FAB00029462046F2F7F6FE0F9BE3664FF000085A
:10FAC000109BC4F85480C4E9196A2367EFF31182CC
:10FAD000202181F31288BFF36F8F0F4D296A616770
:10FAE0002C6282F31188BFF36F8F8FB11F223946CA
:10FAF00004F1780002F0E8FE84F89780AB680BB15F
:10FB0000D3F8A430C4F8A430584605B0BDE8F08F4F
:10FB100084F87870F2E700BFB8750020F0B587B0C0
:10FB200000250595109D04950F9D03950E9D02954A
:10FB3000DDE912760D9D01950C9D00950446FFF7B9
:10FB400077FFB6F1FF3F08BFB7F1FF3F05D056EA98
:10FB5000070305D1204600F071FA204607B0F0BD3A
:10FB60003A46334604F11800014900F013FCF4E76B
:10FB7000CF25010040F2011383810023C0E9263321
:10FB8000C0F8A430014B9860704700BFB8750020E2
:10FB90000A4A93686FF00A01C3F8B0100849C3F825
:10FBA000AC004B6843F080534B60002383F3118813
:10FBB000BFF36F8F9368D3F8B0007047B87500201B
:10FBC00000ED00E070B590F90D20437B002A36DB94
:10FBD000D90634D11B4C63F07F032246437352F89D
:10FBE000183FE169934207D1C0E900210860E06154
:10FBF00011E09942F8D01B68002BF5D090F90E5017
:10FC000093F90E60B542F4D0AE42F2DD5968C0E916
:10FC1000003108605860A569954200D005B9E568D3
:10FC2000A3685A7BD20604D1DA897F2A01D9AA694E
:10FC300032B1AB4202D0284600F00EFB656170BDC8
:10FC40006361FCE7B875002038B590F90D20437B5F
:10FC5000002A014604DA03F07F03437302F040FCFC
:10FC60000D4D2A46AB6852F8184F944200D004B9A3
:10FC7000EC688B4207D05A7BD20604D1DA897F2AFE
:10FC800001D9A2692AB1A34202D0204600F0E4FAC9
:10FC900023466B6138BD00BFB8750020B3F1FF3F4C
:10FCA00008BFB2F1FF3F03D00249183000F072BB29
:10FCB000704700BFCF25010038B5194CA168E06935
:10FCC0000B68814214BF1A46002249680B605960D4
:10FCD000A368E1692AB9134AC3E900210B60E36113
:10FCE0000CE093F90E0092F90E50A84214D0854210
:10FCF00012DD5168C3E900210B605360A569094B0F
:10FD00009D4200D005B9E568A3689D4202D028460F
:10FD100000F0A2FA656138BD9142DCD01268D9E7E3
:10FD2000B8750020D0750020F8B50E4B0C46114672
:10FD30000D4A98681060DDE90667EFF31182202212
:10FD400082F31288BFF36F8F9D68284602F0DAFBBA
:10FD5000284632463B46FFF7A1FF2046BDE8F84063
:10FD6000FFF716BFB8750020E4750020F8B504460B
:10FD7000EFF31187202383F31288BFF36F8F437B48
:10FD800003F01F02002A0CBF0126002649B239D118
:10FD900003F07F03437302F0A3FB2C4D437B81737D
:10FDA00063F07F032A46437352F8183F934227D1EA
:10FDB000E869C4E900200460EC610FE09842F8D0E3
:10FDC0001B68002BF5D093F90EC06145F6D08C4529
:10FDD000F4DD5968C4E900310C605C60AC699442A0
:10FDE00000D004B9EC68AB689C4202D0204600F019
:10FDF00033FA6C6187F31188BFF36F8F3046F8BD1B
:10FE0000E869DEE79B071ED5856802F069FB817310
:10FE10002B689D4209D16B68C4E900531C606C607B
:10FE2000E8E76A689342F6D01B68002BF3D093F999
:10FE30000E209142F5D08A42F3DD5A68C4E90032BF
:10FE400014605C60D6E78173D4E700BFB87500200A
:10FE500049B9EFF3058030B9054B5A699B689A425E
:10FE600001D0FFF795BE81F31188BFF36F8F704704
:10FE7000B8750020034648B9EFF3058232B9064A47
:10FE800051699268914201D0FFF782BE83F31188D5
:10FE9000BFF36F8F704700BFB8750020EFF311817B
:10FEA000202383F31288BFF36F8F054B9A68D37BAF
:10FEB000013BD37381F31188BFF36F8F704700BF8D
:10FEC000B875002070B5EFF31186202383F31288F4
:10FED000BFF36F8F144DAB68DA7B0132DA732A46B9
:10FEE00052F8184F944200D004B9EC685A7BD206FD
:10FEF00004D1DA897F2A01D9A2692AB1A34202D0AA
:10FF0000204600F0A9F923466B6186F31188BFF300
:10FF10006F8FEFF31180202383F31288BFF36F8F6D
:10FF2000BDE87040FFF7A6BFB8750020024B03F193
:10FF30001802C3E906227047B875002070B5EFF3C8
:10FF40001186202383F31288BFF36F8F1B4CA168A7
:10FF5000E0690B68814214BF1A46002249680B60B1
:10FF60005960A368E1692AB9154AC3E900210B6009
:10FF7000E3610CE093F90E0092F90E50A84218D0FC
:10FF8000854216DD5168C3E900210B605360A56905
:10FF90000B4B9D4200D005B9E568A3689D4202D095
:10FFA000284600F059F965613046BDE87040FFF71A
:10FFB000EFBD8A42D8D01268D5E700BFB8750020DF
:10FFC000D0750020F8B550EA010306460C4603D16F
:10FFD000FFF7B4FF0020F8BDEFF31187202383F370
:10FFE0001288BFF36F8F124D124BA8681860FFF78D
:10FFF0002BFEA868104923463246183000F0CAF993
:020000021000EC
:10000000AA68537B43F00403537304463846FFF752
:10001000BFFDAB68D3E90A23B3F1004F08BF002A44
:10002000D8D102F077FB201A20EAE070D3E700BFB6
:10003000B8750020E4750020CF25010038B50446CE
:10004000EFF31185202383F31288BFF36F8F437B77
:100050005B070FD5183002F035FB637B23F00403F8
:1000600020466373FFF7AEFD29460548BDE83840DA
:10007000FFF7EEBE85F31188BFF36F8F38BD00BF69
:10008000E6830020014B9868704700BFB8750020D8
:100090002DE9F8430446077BEFF31185202383F312
:1000A0001288BFF36F8F437B190705D585F311883D
:1000B000BFF36F8FBDE8F883D90943F0080260D120
:1000C0004273A36813B1204602F012FA04F118003B
:1000D00002F0F8FAA66D04F15808B04511D04FF0BF
:1000E000000976B1304602F003FA06F1180002F07A
:1000F000E9FAC6F8B0903046FFF764FDA66DB0454A
:10010000EFD1DFF8C480D8F808309C4241D1EFF33A
:100110000589B9F1000918BF4FF00109D8F8186036
:100120002A4A964200D00EB9D8F80C60B34202D0E9
:10013000304600F091F82046C8F8146001F046F807
:10014000204600F0DBF8B9F1000F02D02048FFF79D
:1001500011FDD8F808309C4231D1EFF3058373BB11
:10016000227BD20718D42846FFF712FDFB07A1D542
:10017000002383F31188BFF36F8F0423184602DF37
:1001800098E703F07F0343F00803437302F0A8F9F4
:1001900097E74FF00009C1E785F31188BFF36F8F30
:1001A00083F31188BFF36F8F0423184602DFEFF348
:1001B0001180202383F31288BFF36F8FD4E785F378
:1001C0001188BFF36F8FD1E7B8750020D07500207C
:1001D00068090020D3B5DDE90667089CCDE9006712
:1001E000FFF7A2FD1CB1034B9B681B69236002B0A3
:1001F000D0BD00BFB8750020427B12F01F0203463D
:1002000010D10A4988420DD00949086868B1D989D6
:100210007F2909D893F90E20064B1B689A42B8BF74
:10022000002070470020704710467047F8070020F4
:100230005C030020E8750020044BC01A044BC0107A
:100240005843044B01221A54704700BF200A002073
:10025000ABAAAAAAE683002070B50D4B0D4D1E7CFB
:10026000FFF7CAFF06EB460305EBC3050446284625
:1002700002F028FA084B00229A553CB1621E28462B
:100280000649BDE87040D31700F084B870BD00BFC8
:10029000B8750020200A0020E68300203902010002
:1002A00038B5EFF31185202383F31288BFF36F8FE6
:1002B0000F4B104A9C681068A04206D1FFF7CCFF94
:1002C00085F31188BFF36F8F38BD00211B7C11604F
:1002D000094AD35C002BF3D02046FFF78DFF00289E
:1002E000EED0637BDB0601D1FFF7E6FC2046E5E7B5
:1002F000B8750020E4750020E6830020EFF311813B
:10030000202383F31288BFF36F8F0A4A136A834254
:1003100007D15B6F136281F31188BFF36F8F704752
:100320001346002BF7D05A6F8242F9D1426F5A67B9
:10033000F1E700BFB8750020024B1868984208BF6B
:100340000020704760030020034B1B680BB9FEF7C9
:1003500019BC0020704700BFEC75002030B570B1AB
:100360000B4B5B6898420AD0036843B1D3E9042180
:10037000D0E90445121941EB0501C3E90421D0E994
:10038000003213605A600023C0E9003330BD00BF63
:1003900060030020B3F1FF3F08BFB2F1FF3F2DE93A
:1003A000F84F0446994615461F467AD08160EFF310
:1003B0001188202383F31288BFF36F8FB9F1000FE8
:1003C000DFF8E4A020DBFFF7BFFFDAE90027013503
:1003D00049F100092D1849EBE073C4E90453AD1845
:1003E000064643EB07074FF00109FFF7A5FFDFF8CB
:1003F000BCE0DEF804A00346EBB9C4E900EACAF8A1
:100400000040CEF8044028E0DAE900126FF0010362
:100410005B1A4FF0FF3161EB02025B1B62EB0902DA
:10042000012B72F10001BCBF01230022C0E904329C
:100430004FF00009D9E7D3E9041CD4E904208A422B
:1004400070EB0C0B24DA891A5A686CEB0000C3E9D4
:100450000410C4E9003214605C60FFF76DFF844251
:100460000ED1134B1B685BB9B9F1000F02D1FFF736
:100470006BFF0646304602F00EF90021FEF754FBF2
:1004800088F31188BFF36F8F28463946BDE8F88F8F
:10049000521A60EB0C009A45C4E90420ADD01B68E9
:1004A000AAE700252F46EFE7380A00206003002066
:1004B000EC7500202DE9F047EFF31185202383F33D
:1004C0001288BFF36F8FDFF8A490DFF8A480C9F81B
:1004D0000000FFF731FF00260027D9F80030D8E9E7
:1004E00000ECD91750B1D0E90442A34271EB020AE3
:1004F0001CDAE41A62EB0102C0E9044213EB0E03BA
:100500004FF000044CEB01012046C8E90031C9F866
:10051000004002F0C0F82146FEF706FB85F3118883
:10052000BFF36F8FBDE8F047FFF7BABE14EB0E02C2
:100530004CEBE473C0E90467C8E90023FFF70EFF42
:1005400085F31188BFF36F8F83689847EFF31185A8
:10055000202383F31288BFF36F8FD9F800301B1B61
:10056000C9F80030FFF7E8FEB7E700BFEC750020E0
:10057000380A002010B5EFF31184202383F312888A
:10058000BFF36F8FFFF7E0FE054A0346D2E9000193
:10059000181841EBE37184F31188BFF36F8F10BD1E
:1005A000380A002038B50346EFF31185202282F384
:1005B0001288BFF36F8FC1600121816000688342A0
:1005C00006D185F31188BFF36F8F0024204638BD14
:1005D000D0E9003213605A600023C0E9003302F012
:1005E000E3F8294604460248FFF732FCEEE700BF75
:1005F000E7830020F8B507460C46164601F06AFF6F
:1006000008B10020F8BD0E4B9B68D3F8A450002D14
:10061000F7D0221DF5D2EFF31184202383F3128843
:10062000BFF36F8F47F004012846B04784F3118869
:10063000BFF36F8F0028E4D040F8045BE2E700BF0F
:10064000B87500200146024A0020FFF7D3BF00BF63
:10065000110E010007B5074B0093074907484FF0FB
:10066000FF334FF48062FFF793F9002003B05DF889
:1006700004FB00BF9431010000A10020400A0020CB
:100680000CB430B589B005460C461C22002101A8E7
:1006900002F002F902238DF806300E4B0293059505
:1006A00023462CB1B4F1004F28BF4FF00043013B6B
:1006B0001D440DAA0C99069501A8009200F00CF8B3
:1006C00014B1059B00221A7009B0BDE8304002B099
:1006D000704700BFAF2901002DE9F04F8DB043688E
:1006E0000293837815469A07804640F10D810024D5
:1006F0000E78002E00F00A81252E0BD04B1C0393A0
:100700000134029B4146304698470028C0F2F680EB
:100710000399EDE74E788B1C252E0393F0D000272C
:10072000B946BB46BBF11F0F38D8A6F12003102BEA
:100730000AD8DFE803F02A09093009090921090963
:100740000928092D09091F00A6F13003092B33D907
:100750002A2E37D11BF0400F55F8043B40F0828021
:10076000002BA7BF4BF0200B9946C3F100094BF0BB
:10077000280B01E04BF0010B039B13F8016B039373
:10078000002ECFD130E04BF0020B4BF0040BF3E71F
:100790004BF0080BF0E74BF0100BEDE7BBF17F0FD0
:1007A00019D8A6F13003092BD2D81BF0400F03D083
:1007B0000A2101FB0737DFE70A2101FB09394BF06A
:1007C000200BD9E72E2E06D11BF0400F40F09E8063
:1007D0004BF0400BD0E76C2E31D02BD8682E36D0A2
:1007E0006A2E3CD04C2E3AD0002F46F02003B8BFE2
:1007F0002BF04002A3F16501BCBF1FFA82FB00276A
:10080000022901D9612B2FD1073525F00705DFF823
:10081000ACA2083507271BF0080F66D00AEB070BC0
:1008200056465E4563D1A4EB0A0A06EB0A02A9EB21
:1008300007096FE1742E9FD07A2E9DD0D4E71BF06C
:10084000800F18BF4BF4007B4BF0800B94E71BF438
:10085000807F18BF4BF4007B4BF4807B8CE74BF41C
:10086000207B89E71F4687E7A6F16301122900F282
:10087000F080DFE811F013004F00EE00EE00EE0014
:10088000EE004F00EE00EE00EE00EE00EE00FE0087
:10089000E900EE00EE001B00EE00AF0055F8043B4F
:1008A0008DF8183001270DF1180AB4E755F804AB9C
:1008B000834BBAF1000F08BF9A461BF0400F14BFDC
:1008C00039464FF0FF31504602F00EF80746A2E7D6
:1008D000029B41462020984700280FDB013EB7428B
:1008E000F6D34C44A41BB14698E74E46F7E716F8FA
:1008F000010B029B41469847002892DA98F8023093
:1009000043F0040388F802304FF0FF3420460DB066
:10091000BDE8F08F1BF0800F34D01BF4007F2CD08B
:10092000073525F00705AA4669685AF8080B2BF029
:1009300010050029ADB237DA404261EB410145F4C0
:1009400080650DF1180B0A235A4601F0D9FFA0EB80
:100950000B0301936B0662D5019B25F001019F42B9
:1009600089B240F3A180002E00F0998015F01002AA
:1009700040F09C80BB460D4623E0AA465AF8040B83
:10098000C117D4E7AA461BF4807F5AF8041B01D193
:100990000846F5E71BF4007F15BF48B208B241F3E3
:1009A000C01141F3C031C2E750EA0103C9D11BF0C5
:1009B000400FC6D0002FC4D12BF0110295B2BB4618
:1009C000019740F2064115EA01021CBF0BF1010B31
:1009D00000222CE02BF010021FFA82FB0A231BF0EE
:1009E000800C49D01BF400711DBF073525F00705A9
:1009F000AA46AA461ABF5AF8080B69685AF8040BA7
:100A000050EA010545D12BF016051BF0400FADB2A1
:100A100042D0002F40D12BF0170295B2019715F06C
:100A2000100248D0019B002E42D103F1010B29078F
:100A30005AD4EB0706D5D9456FDD0199A9EB0B0315
:100A40005F18CB465B4649E04BF0100B102378262D
:100A5000C5E7782B04D1C6F1780343F01003BEE755
:100A6000029B4146252098470028FFF647AF0234F5
:100A700047E608230026B2E7AA461BF480715AF81D
:100A8000040BBDD01BF400711ABFC0B2614680B226
:100A9000B6E72BF0060295B20DF1180B54E725F0DE
:100AA0001105ADB2BB468CE70D46B8E73B460D4697
:100AB00003F1020BBBE7DDF804B082E7DC3C010088
:100AC000D53C0100CDE904324146029B20209847E5
:100AD0000028FFF613AF049B059A01339945F1DC1A
:100AE000A4EB0B01CC189B460AB3029B4146302075
:100AF00098470028FFF602AF8EB901342744019BC6
:100B0000391B994224DC1D465DBB019AA9EB0B09F8
:100B1000224455461446914435E0019F92E7023441
:100B200041463046029B98470028E7DAE6E640F265
:100B300006410D42E2D015F0020F14BF2B202020F9
:100B400015F4806F04F10104414618BF2D20E9E738
:100B5000029B414630209847002804F10104CEDA78
:100B6000CCE606AB013D4146585D029B9847002804
:100B7000CADAC3E6029B414620209847002804F1C8
:100B80000104FFF6BBAEA9EB0403002BF2DCBFE5CA
:100B9000704710B50278083A012A0B460CD8447801
:100BA00041681D2C28BF1D241846224601F066FE10
:100BB00003460020185510BD0120FCE700EBC100E2
:100BC000408840087047F8B50346FFF7F7FFB0FAD2
:100BD00080F0C0F11F0003EB800CCA00DCF810604D
:100BE000171D0C4606328DB256B9012101FA00F0EC
:100BF000D9680143D960CCF81040DD539D52F8BD4F
:100C0000F1000431585AD85303EBC0009E52C580FE
:100C10005D52F4E710B500EBC104E388994202F19C
:100C200004010AD1012303FA02F2C36823EA020392
:100C3000C360002340F8213010BDA28840F8213065
:100C400000EBC20100EBC300CB808280F4E708B563
:100C50000346FFF7B3FFB0FA80F2C2F11F02184655
:100C6000BDE80840FFF7D6BF2DE9F843B1FA81F59A
:100C7000C5F11F0900EB89080346D8F810200E467D
:100C8000C2B10327D8F8104018462146FFF796FF57
:100C9000B04206D34A461846FFF7BCFF2046BDE8DF
:100CA000F88303EBC404013FE088C8F8100001D0CA
:100CB0008242E7D1C5F120024FF0FF349440DA6858
:100CC0001440EBD094FAA4F2B2FA82F2111D53F858
:100CD00021402146DFE738B50346FFF76FFF0D4699
:100CE000044611461846FFF769FF03EBC5050444A7
:100CF000600068801846FFF761FF014423F8314027
:100D000038BD38B50346FFF759FF0C46A51A511AEE
:100D100003EBC40405444800608003EBC2006C0090
:100D2000448023F8321018461146FFF747FF01446C
:100D300023F8315038BD38B50546FFF73FFF0C4664
:100D4000014405EBC1035B88DA070AD42846FFF7A4
:100D50007EFF21462846FFF731FF22182846FFF77D
:100D6000BAFF35F83410611A05EBC1035B88DB0765
:100D70000CD42846FFF76BFF35F834102246611A71
:100D80002846FFF7A8FF35F83430E41A21462846F4
:100D9000BDE83840FFF717BF61B100680439091A90
:100DA00021F007030344C9085A8822F001025A803F
:100DB000FFF7C1BF704770B5056809B9002070BD65
:100DC00001F007030B33CC0804EBD304AB689C425F
:100DD00028BF1C4621462846FFF746FF0646002846
:100DE000ECD001462846FFF7E9FEA04207D93219A8
:100DF0002846FFF786FF11462846FFF7E4FE05EB7D
:100E0000C6021046538843F0010353800430D6E7EE
:100E10001146FFF7D0BF043A2DE9F041CC1D114433
:100E200024F0070421F007010E1BF708B7FA87F238
:100E3000C2F12405AD004FF000080735C2F12002D1
:100E4000ED0804604146A760C4F80C80920004F1EC
:100E5000100001F021FD6B0043F00103638004EBFF
:100E6000C5027B1B5900A4F800805180A21924F808
:100E70003550A2F80280A35304EBC70329465A88D1
:100E800042F001025A802046BDE8F041FFF79BBEC8
:100E9000002070470FB407B504A951F8040B019165
:100EA000F0F7E2FF03B05DF804EB04B070470FB455
:100EB00007B504A951F8040B0191F0F7D5FF03B071
:100EC0005DF804EB04B07047092804D83030C0B294
:100ED0000870002070470F2801D85730F7E76FF0EF
:100EE00015007047F8B54E000C46711C994217D892
:100EF000034615460719BB4204D1002302F81430FB
:100F00003046F8BD187829460009FFF7DDFF13F8D1
:100F1000010B691C00F00F00FFF7D6FF0235EAE76E
:100F20000026EDE7036800220BB9184670478B4294
:100F300010D10B6842B942680360914200D143600E
:100F400000230B600120704713604368994208BF7B
:100F50004260F5E71A461B68E6E7038B13F00703C8
:100F600005D10368002B0CBF002003207047022B23
:100F700005D1408BB0FA80F0400980007047012B0A
:100F800005D10368002B0CBF00200520704700200E
:100F9000704710B50C4600B111B96FF0150010BDC7
:100FA000081D00F0D2F80028F9D1A368032BF6D968
:100FB000F3E72DE9F0410D4607461946281D9046F6
:100FC0001E4600F0D6F8044638B13346424629465C
:100FD0003846A446BDE8F0416047BDE8F08110B452
:100FE000EFF31182202484F31288BFF36F8F4161E5
:100FF00010BC0121F0F76ABF38B50C46054658B160
:1010000051B10B6843B14B6833B11C22002101F090
:1010100043FC2C61002038BD6FF01500FBE770B574
:1010200005460E46FFF7B5FF041E14DBEFF31182F1
:10103000202383F31288BFF36F8F6B8B2C8B4FF6BB
:10104000FF718B4204F0070407D182F31188BFF3CC
:101050006F8F6FF00A04204670BD022C0CD1013353
:101060006B8382F31188BFF36F8F002322463146D2
:101070002846FFF79EFFEEE7062C14D8DFE804F0C1
:1010800004131313041A0400002333606B683BB984
:10109000C5E90066ACB902212846F0F717FFDAE788
:1010A0001E606E60F6E782F31188BFF36F8F6FF0FA
:1010B0000404D0E782F31188BFF36F8F6FF08504CB
:1010C000C9E782F31188BFF36F8FC4E710B5EFF360
:1010D0001182202383F31288BFF36F8F048B04F0F7
:1010E0000704022C0AD0012C0CBF6FF004006FF033
:1010F000850082F31188BFF36F8F08E0438B013BBB
:101100009BB2438323B92146F0F7E0FE204610BD91
:101110002046EEE738B5A8B1A1B1EFF31185202242
:1011200082F31288BFF36F8F048BFFF7FBFE30B1A1
:1011300004F0070085F31188BFF36F8F38BD6FF09F
:101140007700F7E76FF01500F8E7034640B1426813
:1011500002F00302022A06D0032A04D0012A05D095
:101160006FF0150070471A68002AF9D000209860C7
:10117000704710B54268816002F00302022A0346FC
:101180004FF0000407D0032A02D05C60002001E089
:1011900018685C6010BD18685C600028F6D0FFF726
:1011A00001FAF3E7704701F077BB01F067BB014636
:1011B0000068F0F7D5BF08B5F1F702F8BDE80840C0
:1011C000F1F722B800210120F0F7CABF6FF08500C7
:1011D000704761B662B680F31188BFF36F8F7047B6
:1011E00072B6002383F31188BFF36F8FBFF34F8F65
:1011F00030BF62B6BFF36F8F704772B6002383F3C0
:101200001188BFF36F8FBFF34F8F20BF80F311881A
:10121000BFF36F8F62B67047202809D9B0F1004F35
:1012200008D80138B0FA80F0C0F11F0040007047C4
:10123000082070473E20704708B5F1F713FD0020E5
:1012400008BD7047002303824369C3607047416A49
:101250008968F1F773BDEFF31182202383F31288BD
:10126000BFF36F8F00230B60436833B9C0E90011EF
:1012700082F31188BFF36F8F704719604160F7E701
:1012800010B50346EFF31181202282F31288BFF3D9
:101290006F8F006828B15C6802681A60A04208BFBE
:1012A0005A6081F31188BFF36F8F10BD027A01324B
:1012B00002727047426810B52AB10B461C465B6843
:1012C000002BFBD16260416010BD10B5044620B90F
:1012D0000B7A01330B72084610BD034618465B6853
:1012E000002BFBD1FFF7E6FF2046F5E710B508B16C
:1012F0004B6843604C68002308464B60F1F79CFD47
:10130000204610BD83680B440360704783880268E1
:1013100019448180D018704730B484880568A318B8
:101320008380281930BC01F0A9BA10B583880268FF
:101330005C1C8480D154D01810BD034600689A8884
:10134000401A11441860998070470268531E036068
:1013500083880133838002F8011C70478288521A07
:10136000034682800068084418607047034600689E
:101370009A88521A01449A801960704710B5036820
:101380001C780121FFF7EAFF204610BD0268806843
:10139000101A7047012310B50621044600F8013BDE
:1013A000F9F7BEF918B9A37963F03F03A37110BD33
:1013B0000B6803608B8883808B798371037823F0BB
:1013C0000203037070470078C0F34000704738B5DF
:1013D0000446807AF1F788FC6169054649B1637A71
:1013E000DB0704D4436A1B6820469B6898470023A8
:1013F000636121462846BDE8384001F016B8F7B5CC
:1014000004460E461746A388012B01D803B0F0BD51
:101410002046FFF7B3FF05460028F7D0A388834294
:10142000F4D32046FFF7AAFF013D23688DF80000A2
:10143000394668468DF801500193B0470028E5D041
:1014400029462046FFF78AFFDDE710B50346BFF3C4
:101450005B8F53E8000F40EA010243E80024002CB0
:10146000F7D1BFF35B8F10BD01210C30FFF77EBFBA
:1014700030B402EBC303044608469A4201D130BCA3
:101480007047114611F8085BA54206D1018A5378CE
:101490009942F4D330BC536818470A46EDE7BFF3CE
:1014A0005B8F50E8003F0B4040E80032002AF8D143
:1014B000BFF35B8F7047033138B5C9B205460E20C4
:1014C000F2F7A0FA032104460C30FFF71FFF0123B7
:1014D0000370A0F80150204638BD70B505460E4691
:1014E0000F200421F2F78EFA042104460C30FFF796
:1014F0000DFF0122067042704580204670BD08B580
:10150000072201F0D1F9B0FA80F0400908BD0028A7
:101510000CBF08460020704707B580B90621684611
:10152000F9F7FEF840B99DF80530684603F03F032F
:101530008DF80530F2F7A6FA03B05DF804FB6FF002
:101540001500F9E70120704710B50C4631B10020B5
:10155000FFF7E2FF08B90123237010BD6FF01500FB
:10156000FBE738B54FF0FF3105464FF0FF30F1F79C
:10157000CFFE044660B102210C30FFF7C7FE0580A4
:1015800021460022BDE8384042F24600F1F75CBF38
:101590006FF0680038BDBFF35B8F0068BFF35B8FEF
:1015A000704708B54B0900EB8300FFF7F4FF01F02B
:1015B0001F01084100F0010008BD0B6803608B8823
:1015C00083808B798371704710B50346BFF35B8FBF
:1015D00053E8000F00EA010243E80024002CF7D191
:1015E000BFF35B8F10BD01F01F0301229A404B092E
:1015F00000EB8300D143FFF7E7BF0023BFF35B8F0E
:1016000050E8002F40E800310029F9D1BFF35B8F8B
:1016100070474A09012301F01F018B4000EB820053
:10162000BFF35B8F50E8002F1A4340E800210029E8
:10163000F8D1BFF35B8F704773B5038A062B2AD9A5
:1016400000F10C0507212846FFF790FE06460088AA
:10165000F2F7F2FE0446F0B104211430FFF7A1FFC7
:10166000C8B996F902308DF8053096F903308DF837
:1016700006303079F1F77EFE227C8DF80700E379A1
:101680008DF804300094737952B933B96A4629460B
:101690002046F2F7E3FE02B070BD01232374FAE79F
:1016A000002BF8D1FAE708B5C3681888F2F7C4FE32
:1016B00020B1BDE808401F21F2F7C6BB08BDBFF34B
:1016C0005B8F0068BFF35B8F084100F0010070473B
:1016D00070B5038A0B2B0D46164602D86FF0150025
:1016E00070BD0C210844FFF741FE04460088F2F764
:1016F000A3FE03460028F1D005211430FFF7DFFFD9
:101700000028EBD0DA7BA179CA40D207E6D5A278CF
:101710002A70B4F903206A8062792A71A1790122C2
:101720008A406A71227AEA71E279AA71B4F80920D2
:101730002A810020E872E27AAA720C34EC603360ED
:10174000CEE70369C9B20C2201FB0233186C00F02A
:101750000700704770B5C9B20369EFF31185202403
:1017600084F31288BFF36F8F0C2606FB0134246CC0
:1017700014F0C00408D0A24206D085F31188BFF34C
:101780006F8F4FF0FF3070BD06FB013301221A64EA
:1017900085F31188BFF36F8F436803EBC1035B6868
:1017A00098470020EFE78022FFF7D4BFF8B5069FE7
:1017B0000469C9B2EFF31186202585F31288BFF3BF
:1017C0006F8F0C2505FB0144256C05F0070CBCF15F
:1017D000010F0CD1276486F31188BFF36F8FC4E922
:1017E0000E23436853F8313098470020F8BD05F0C8
:1017F000C005AF4286F31188BFF36F8F0CBF6FF047
:1018000077004FF0FF30F1E713B580240094FFF725
:10181000CDFF02B010BD10B40069CBB21C2403FB95
:101820000400002110BC10471046FDF749BF00F02E
:10183000EAB9FDF70BBB43685B68D3F810350B6062
:101840000020704743685B6802EA010021EA020158
:10185000C3F80805C3F80C150020704743685B689F
:101860000020C3F80815704743685B680020C3F880
:101870000C15704743685A68D2F8043521EA030012
:101880000B40C2F80805C2F80C350020704710B5AF
:1018900003695868F8B1884219D19C680868586093
:1018A000A14200D19860002008602AB15A680A60FD
:1018B0009A68596002B99960002010E0814206D10F
:1018C0000868206098688142EDD19C60EBE704468F
:1018D00000680028F2D1002AE8D16FF0150010BD91
:1018E000FDF7C8BB30B543681360057A446804EB64
:1018F000C504A34202D36FF0010030BD5C798C4275
:1019000001D00833F0E70020F7E743681B68D3F8FD
:101910008004C3F88004704742681368D3F810014C
:1019200050B1126A002012780A70C3F81001D3F87F
:10193000102101221A6070474FF0FF307047026893
:101940000346D2F8580140B95B68DB0706D4D2F8E9
:101950002001003818BF01207047012070474368FC
:101960001B68D3F80423D20517D5D3F82021A2B1E0
:10197000EFF31182202181F31288BFF36F8FD3F828
:10198000201131B10021C3F82011D3F82011012119
:10199000D96082F31188BFF36F8FD3F85831704745
:1019A00013B501AA0446FFF79DFF002805DB019B44
:1019B000226819791868FCF7AFFD02B010BDF8B5C0
:1019C0000022054601210220F0F732FF0220F0F745
:1019D000FFFE6C680121E068FFF7E2FF6B681968A1
:1019E0002369C1F82435A27D637D207D1343228BBA
:1019F00002431343C1F86C356E68D6E9004313F017
:101A0000010336D02F6904F10C0107F1080204F537
:101A1000907000F094F800282ADB387AFDF77EF900
:101A20000823C4F80035F369C4F844350023C4F82A
:101A300048350123A360D4F85831002BFBD0002196
:101A4000C4F800156D682C68E868FFF7A9FF082343
:101A5000C4F800352A7A52B92B6AC4F83435012308
:101A6000C4F83835C4F81021D4F8102123600020C0
:101A7000F8BD0822C4F80025F269C4F84425C4F86A
:101A800048350123A360D4F82031002BFBD000237C
:101A9000C4F82031D4F820310123E3604FF480737F
:101AA000C4F80433C7E700F150039B009BB203F175
:101AB000804303F5883300221A601B687047034691
:101AC0000020184700F06DBB10B502461168B1B197
:101AD000BFF35B8FB1FA81F3C3F11F000123834091
:101AE00021EA030352E8004F8C4204D142E8003C53
:101AF000BCF1000FF6D1BFF35B8FE7D110BD6FF0E3
:101B00000B00FBE710B50368CB40DB0714D40123BF
:101B10008B400268BFF35B8F43EA020150E8004F3D
:101B2000944204D140E8001CBCF1000FF6D1BFF391
:101B30005B8FEED1002010BD6FF01500FBE770B594
:101B40000C460021054608461646FDF7D9F8002840
:101B50000ADB3378DB0003F1804303F5F833002020
:101B6000C3F81055C3F8144570BD10B1012802D058
:101B70007047FDF76BB9FDF723B918B1012803D100
:101B800000F026B800F03FB8704708B5FDF734F90B
:101B9000BDE80840FDF79AB938B54FF080440123FD
:101BA000C4F8083363600023C4F80031D4F800316E
:101BB00042F21075D4F80C24D4F80C34D20306D5B4
:101BC000DB0704D50120FFF77DFF013DF2D138BDD1
:101BD000FFF7E2BF38B54FF080440223C4F8083362
:101BE0000123E3600023C4F80431D4F8043142F245
:101BF0001075D4F81834DB0304D50120FFF762FF19
:101C0000013DF6D138BDFFF7E5BFF7B5019001A85A
